:100000000C9488110C94F3830C94FEB30C94A711F8
:100010000C94A7110C94A7110C94A7110C94C384F1
:100020000C94A7110C94A7110C94A7110C946A833B
:100030000C94A7110C94A7110C94A7110C94A71160
:100040000C94A7110C94DBAB0C943B290C94052960
:100050000C9453250C943D210C94D7430C94A71178
:100060000C9421650C9438810C94A7110C94A71161
:100070000C94A7110C94A7110C947C290C942B259B
:0C0080000C94A7110C94A7110C94A7116C
:100100005D5D5D5D5D5D5D5D5D5D5D5D5D5D5D5D1F
:100110005D5D5D5D5C5C5C5C5C5C5C5C5C5B5B5B1E
:100120005B5B5B5B5B5A5A5A5A5A5A5A5A5A5A5A2A
:10013000595959595959595959595959595959592F
:100140005959595A5A5A5A5A5A5A5B5B5B5B5B5B0C
:100150005B5B5C5C5C5C5C5C5C5C5D5D5D5D5D5DDB
:100160005D5D5E5E5E5E5E5E5E5E5E5F5F5F5F5FAC
:100170005F5F5F606060606060606061616161617D
:100180006161616161616262626262626262636353
:100190006363636363646464646464646464646523
:1001A00065656565656565666666666666666767F4
:1001B00067676767676868686868686868696969C1
:1001C0006969696A6A6A6A6A6B6B6B6B6B6B6C6C88
:1001D0006C6C6C6C6D6D6D6D6E6E6E6E6F6F6F6F47
:1001E00070707070717171727273737474747575EC
:1001F0007676777878797A7B7C7D7D7D7D7D7D7D57
:10020000FFFFFFFFFFFFFFFFFFFFFFFFFFFFFFFFFE
:10021000FCF9F6F4F1EEEBE8E6E4E1DFDCDAD8D65F
:10022000D4D2D1CFCDCBCAC8C6C5C3C2C1C0BEBD52
:10023000BCBAB9B8B6B5B3B2B2B1B0AFAEADACAB93
:10024000AAA9A8A7A5A4A3A2A1A1A09F9E9E9D9C88
:100250009B9B9A9998979796959493929191908F4A
:100260008E8E8D8D8C8B8B8A8A89888887868685F1
:10027000848383828180807F7E7D7D7C7C7B7B7A92
:100280007A7979787777767675747473727271701B
:10029000706F6E6D6D6C6B6B6A6A696968686766B2
:1002A000666565646363626161605F5F5E5D5C5B40
:1002B0005B5A5959585757565655545453525251E0
:1002C00050504F4E4D4C4B4A494847474645454490
:1002D00043424241403F3E3D3C3B3A38373535345E
:1002E000333231302F2D2C2A2927252322201F1D80
:1002F0001B191613110E0C0804000000000000006A
:10030000FFFFFFFFFFFFFFFFFFFFFFFFFFFFFFFFFD
:10031000FCF9F6F4F1EEEBE8E6E4E1DFDCDAD8D65E
:10032000D4D2D1CFCDCBCAC8C6C5C3C2C1C0BEBD51
:10033000BCBAB9B8B6B5B3B2B2B1B0AFAEADACAB92
:10034000AAA9A8A7A5A4A3A2A1A1A09F9E9E9D9C87
:100350009B9B9A9998979796959493929191908F49
:100360008E8E8D8D8C8B8B8A8A89888887868685F0
:10037000848383828180807F7E7D7D7C7C7B7B7A91
:100380007A7979787777767675747473727271701A
:10039000706F6E6D6D6C6B6B6A6A696968686766B1
:1003A000666565646363626161605F5F5E5D5C5B3F
:1003B0005B5A5959585757565655545453525251DF
:1003C00050504F4E4D4C4B4A49484747464545448F
:1003D00043424241403F3E3D3C3B3A38373535345D
:1003E000333231302F2D2C2A2927252322201F1D7F
:1003F0001B191613110E0C08040000000000000069
:10040000242727272A272D273027FF274A274D274C
:100410005027532756278D2793279627A927FF274D
:10042000C427EF2710281328252828282D283C2802
:100430000029002900290029002900290029002974
:100440000029002900290029002900290029002964
:100450003F284528422848284B284E285128542810
:100460007B288528882893289D28A528A828AB289C
:10047000AE28B128B428B728BA28D628DC28D9282D
:10048000DF28E228E728F228F528F02EF42EF62EB1
:10049000212FF82E232F252F232F252FFA2E272F1C
:1004A000212F232FFC2EFE2E232F272F212F002F2D
:1004B000022F042F062F082F152F172FAC8FE88F30
:1004C000E88FE88FE88FE88FE88F8E8FE88FE88FCE
:1004D000E88FE88FE88FE88FE88FCD8FE88FE88F7F
:1004E000A18FE88FE88FE88FE88FE88FE88FE88F9B
:1004F000E88FE88FE88F468FE88FE88F4E8F588F10
:10050000608FE88F6A8F728F6F94848FE88FE88F87
:100510007C8FE88FD68FE88FB78FC28FE88FE88FF8
:10052000968FE88FE08F99163F1C6E16F615DD1535
:10053000BE1336B0C415C115B1156217A715A015A5
:100540003B3FC91B99158F15F114E6147E14E9136E
:1005500074141AB9C313E313BF13C213EA13C013FD
:10056000C1135BB8C8FAC8C80AC8C83CD21E6464C4
:100570000C3C0EFA3C08101464FFFFFFFF0080558E
:100580005500403333AB2A92240020721C9A19463E
:10059000175515B1134912111100100F0F390E79AB
:1005A0000DCD0C310CA30B210BAB0A3D0AD9097BF5
:1005B000092509D408890842080008C2078807509D
:1005C000071C07EB06BD06900666063E061806F4F5
:1005D00005D105B00591057205550539051F0505BD
:1005E00005EC04D504BE04A80492047E046A0457F2
:1005F0000444043204210410040004F003E103D293
:1006000003C403B603A8039B038E03820376036A25
:10061000035E03530348033E03330329031F0316FA
:10062000030C030303FA02F102E902E002D802D04C
:1006300002C802C102B902B202AB02A4029D029634
:10064000028F02890283027C02760270026A0264CF
:10065000025F02590254024E02490244023F023A2A
:1006600002350230022B02270222021E0219021555
:100670000211020C02080204020002FC01F801F45B
:1006800001F001ED01E901E501E201DE01DB01D745
:1006900001D401D101CE01CA01C701C401C101BE0B
:1006A00001BB01B801B501B201AF01AC01AA01A7BC
:1006B00001A401A1019F019C019A0197019501925A
:1006C0000190018D018B0188018601840182017FE7
:1006D000017D017B01790176017401720170016E67
:1006E000016C016A01680166016401620160015EDA
:1006F000015D015B0159015701550154015201503F
:10070000014E014D014B014901480146014401439D
:1007100001410140013E013D013B013A01380137F1
:100720000135013401320131012F012E012D012B40
:10073000012A012901270126012501230122012186
:10074000011F011E011D011C011A011901180117C9
:10075000011601150113011201110110010F010E03
:10076000010D010B010A010901080107010601053C
:100770000104010301020101017072696D657000DD
:100780007072696D65705F74656D705F7363616CC5
:10079000696E67006177655F74696D655F636F6C33
:1007A00064006177655F74696D655F7761726D0084
:1007B0006372616E6B696E675F74687265730077F0
:1007C00061726D75705F6D61705F7363616C650000
:1007D0006372616E6B696E675F6469760066696CEF
:1007E0006D5F636F656666007368696674637574D0
:1007F0005F706F746C6F770073686966746375748B
:100800005F706F7468690073686966746375745F9C
:1008100072657463757400626F6F73745F6D617479
:1008200064656300626F6F73745F656774646563AA
:10083000006961637265665F6D6174736C6F70658A
:100840000073686966746375745F6D696E72706D4C
:10085000006567745F72696368006B6E6F636B5FDE
:1008600072696368006B6E6F636B5F626F6F737446
:10087000007761726D75705F636C74007761726D83
:1008800075705F72706D5F7363616C650072657126
:100890005F6675656C006469766964657200616C99
:1008A0007465726E61746500696E6A6F70656E0062
:1008B00062617474666163006B7061666163006B92
:1008C00070616F66667300696E6A6F636675656CEA
:1008D00000696E6A72616D7075705F6261747466D2
:1008E000616300696E6A70776D00696E6A70776D1A
:1008F0007400616C735F6C61756E63685F696E70C4
:100900007574006C61756E63685F6D61786B7061A2
:10091000006C61756E63685F6B706172616E6765B4
:1009200000747073646F745F6B7061646F745F6385
:100930006F6E6600747073646F74726174650074B6
:100940007073617100616C735F6375745F6D696E64
:10095000747073007470736173796E630061636D9A
:10096000756C740074707361636F6C64006C617596
:100970006E63685F656E72696368006C61756E6353
:10098000685F726574617264006F76657272756E0D
:100990005F6675656C637574006F76657272756EEF
:1009A0005F6675656C726573756D65007265765FFF
:1009B0006C696D69740061697264656E5F69676E08
:1009C0006F726500636F6E666967313100636F6EC9
:1009D000666967313200636F6E6669673133006242
:1009E0006174745F63616C00696163326C6F616430
:1009F00000616C735F6D61785F6375740062617232
:100A00006F5F6D6F6465007470735F6C6F770074F7
:100A100070735F686967680066616E5F74656D70AA
:100A20000066616E5F687973740066616E5F63680B
:100A3000616E6E656C006961635F737465705F738E
:100A40006571006961635F636F6E66006961635F12
:100A50006D61785F7374657073006961635F747052
:100A6000735F7468726573006961635F636F6C6460
:100A70005F69646C655F74656D70006961635F7761
:100A800061726D5F69646C655F74656D700069614A
:100A9000635F636F6C645F72706D006961635F7741
:100AA00061726D5F72706D006961635F636F6C642A
:100AB0005F73746172745F706F73006961635F77F5
:100AC00061726D5F73746172745F706F73006961DE
:100AD000635F616674657273746172745F72706D66
:100AE000006961635F616674657273746172745FDB
:100AF0006475726174696F6E006961635F737065BC
:100B00006564006961635F6B70006961635F6B6955
:100B1000006961635F6B64006C61756E63685F722E
:100B2000706D006961635F696E74656772616C5FA7
:100B30006C696D69745F646563006961635F696EA8
:100B400074656772616C5F6C696D69745F696E630F
:100B5000006961635F696E74656772616C5F64658B
:100B6000616462616E64006C61756E63685F72657A
:100B7000746172645F6D617267696E00616C735F4E
:100B80006375745F6D617874707300726F61647304
:100B9000706565645F646976696465720069616344
:100BA0005F7265665F706F73006961635F736F6C1E
:100BB0005F6368616E6E656C006961635F69676E33
:100BC0005F736C6F706500736F667472706D5F72C7
:100BD000616E6765006961635F69676E5F61647616
:100BE000616E63655F6C696D6974006961635F69FB
:100BF000676E5F7265746172645F6C696D697400C1
:100C00006961635F69676E5F7468726573686F6C52
:100C1000640065676F5F636F6E660065676F5F6C2A
:100C200061670065676F5F636F6F6C616E7400650D
:100C3000676F5F6D61787470730065676F5F6D617A
:100C4000786D61700065676F5F6D696E72706D00C1
:100C500065676F5F6D617872706D0065676F5F7754
:100C600061726D75700065676F5F6C65616E5F6C5A
:100C7000696D69740065676F5F726963685F6C694D
:100C80006D69740065676F5F7069645F6B700061A8
:100C90006C735F656E726963680065676F5F64653A
:100CA0006C74610065676F5F74617267657400657D
:100CB000676F5F7069645F77696E646F77006967FB
:100CC0006E7265746172645F636C616D7000616CFB
:100CD000735F72656163745F7470730077626F3203
:100CE0005F6162735F6C696D69740077626F325F18
:100CF0006C696D69745F6D6178740077626F325FE3
:100D000066616C6C6261636B0077626F325F726503
:100D10007472795F7400616C735F72657461726480
:100D20005F72706D3100616C735F726574617264C3
:100D30005F72706D320077626F325F72695F7461EB
:100D4000726765740077626F325F6E65726E73747E
:100D500064635F7461726765740077626F325F709D
:100D6000756D705F70775F7A65726F0077626F3252
:100D70005F63616C6962726174696F6E0077626F44
:100D8000325F6865617465725F7069645F6B700083
:100D900077626F325F6865617465725F7069645F06
:100DA0006B690077626F325F6865617465725F704E
:100DB00069645F6B640077626F325F686561746558
:100DC000725F7069645F696C696D69740077626FE6
:100DD000325F70756D705F7069645F6B7000776211
:100DE0006F325F70756D705F7069645F6B690077FB
:100DF000626F325F70756D705F7069645F6B640005
:100E000077626F325F70756D705F7069645F696C77
:100E1000696D697400696E6A5F7374616765325FDA
:100E20006F6666736574006B6E6F636B5F6368619A
:100E30006E006B6E6F636B5F73616D706C696E6774
:100E40005F77696E646F77006B6E6F636B315F669F
:100E500072657175656E6379006B6E6F636B315F80
:100E60006761696E006B6E6F636B315F696E74658D
:100E7000677261746F72006B6E6F636B325F667264
:100E8000657175656E6379006B6E6F636B325F675A
:100E900061696E006B6E6F636B325F696E7465675C
:100EA0007261746F72006B6E6F636B5F74687265F2
:100EB00073686F6C64006B6E6F636B5F6E6F6973EA
:100EC000655F7363616C65006B6E6F636B5F6D6113
:100ED000785F726574617264006B6E6F636B5F64E0
:100EE000656661756C745F726574617264006B6EC7
:100EF0006F636B5F7265746172645F7374657000B9
:100F00006B6E6F636B5F7265746172645F64656C56
:100F10006179006B6E6F636B5F616476616E6365B0
:100F20005F73746570006B6E6F636B5F6164766195
:100F30006E63655F64656C6179006B6E6F636B5F98
:100F40006D696E72706D006B6E6F636B5F6D617853
:100F500072706D0065676F5F64656C6179006567CD
:100F60006F5F6D696E6D617000636F6C645F696760
:100F70006E61646A757374006372616E6B5F76652F
:100F80000066696C6D5F656E6C65616E00696163BA
:100F90005F636C6F73655F64656C61790069616341
:100FA0005F696E74656772616C5F6C6F776D61709D
:100FB000006261726F666163006261726F5F6F668B
:100FC0006673006C63645F6330006C63645F6465C8
:100FD0006C6179006C63645F6261636B6C69676804
:100FE00074006B70615F636F6E6600616C735F6944
:100FF000676E6375745F72706D3200616C735F72DF
:1010000065746172645F6D696E74707300616C7396
:101010005F7265746172645F6D6178747073006C87
:1010200063645F64656661756C745F76696577009B
:101030007072696D6172795F747269676765720059
:101040007365636F6E646172795F747269676765F7
:101050007200746F6F74685F776865656C00747296
:1010600069676765725F746F6F746800616E6F7433
:101070006865725F747269676765725F746F6F74B9
:1010800068006C63645F616E616C696E00746F6FA1
:1010900074685F776865656C5F747769647468000D
:1010A00063616D5F73796E635F725F656467655FCF
:1010B00070686173650063616D5F73796E635F660D
:1010C0005F656467655F706861736500726573650D
:1010D000745F656E6770686173655F616674657281
:1010E0000069676E5F74646364656C617900696749
:1010F0006E5F6477656C6C31340069676E5F64772E
:10110000656C6C6D61700069676E5F6372616E6BB8
:101110005F616476616E63650069676E5F6F7574A9
:101120000069676E63686D617800656E67696E65FA
:101130005F6F66665F64656C61790070756D705F86
:101140006F6E5F6D696E74696D65006675656C7054
:10115000756D705F6368616E6E656C00696E6A5F65
:101160007374616765325F7261746500696E6A5F8E
:101170007374616765325F73746172745F747073E6
:1011800000696E6A5F7374616765325F7374617260
:10119000745F6D617000616C735F69676E63757415
:1011A0005F72706D3100616C735F64656163745F61
:1011B00074696D6500616C735F64656163745F651C
:1011C000677400616C735F72657461726400616C56
:1011D000735F7265765F6C696D6974006D697363C6
:1011E000316F75745F6D696E72706D006D697363D8
:1011F000316F75745F6D617872706D006D697363C6
:10120000316F75745F6D696E747073006D697363AF
:10121000316F75745F6D6178747073006D6973639D
:10122000316F75745F6D696E6D6170006D697363A8
:10123000316F75745F6D61786D6170006D69736396
:10124000316F75745F6368616E6E656C006D697394
:1012500063316F75745F636F6E646974696F6E7309
:10126000006D697363316F75745F636F6E64697469
:10127000696F6E31006D697363316F75745F636F91
:101280006E646974696F6E320073656369676E6F4F
:101290007265006770735F6C6F67006961635F639D
:1012A0006C6F73655F6D696E6D6170006961635F1E
:1012B000636C6F73655F706F73006163745F776FEA
:1012C000745F72706D006163745F776F745F6368E1
:1012D000616E6E656C006163745F72706D5F7270D9
:1012E0006D006163745F72706D5F6368616E6E65DF
:1012F0006C00656774315F63616C00616C735F746F
:101300006B735F6368616E6E656C00626F6F7374A0
:101310005F636F6E6600626F6F73745F6D6F72658F
:1013200000626F6F73745F6D696E70726573737551
:10133000726500626F6F73745F7069645F6B7000D9
:10134000626F6F73745F7069645F6B6900626F6F67
:1013500073745F7069645F6B6400626F6F73745F56
:101360007069645F696C696D697400626F6F737432
:101370005F6368616E6E656C0077617465725F7043
:10138000756D705F74656D700063616D7368616623
:10139000745F65785F6368616E6E656C006E6F6E1A
:1013A00076655F6B70616C6F6F6B75705F6D696E8A
:1013B0006B70610077617465725F70756D705F68E6
:1013C0007973740077617465725F70756D705F63B7
:1013D00068616E6E656C00746F6F746872656C5FC7
:1013E0006E6F726D616C00746F6F746872656C5FA4
:1013F0006D697373696E67006675656C6375745F9C
:101400006D696E5F6B7061006675656C6375745FA6
:101410006D61785F6B706100746163685F636861C0
:101420006E6E656C00746163685F646976007368F2
:101430006966746375745F636F6E665F696E7075FD
:10144000740073686966746375745F74707374682C
:10145000726573680073686966746375745F746934
:101460006D6500736F667472706D5F72706D007978
:101470000780079407A207B007BF07D007DD07E87A
:1014800007F8070708170824083108410851085AC7
:10149000086508710800000000000000000000005E
:1014A000000000000000007C088D0896089E08A837
:1014B00008B008B808BF08C708D108E308EA08F26E
:1014C0000803091109210934090000000000003F48
:1014D00009000000000000450954095D0964096D18
:1014E000097B0989099909AC09B609C409CD09D64E
:1014F00009DF09E809F109FD09070A0F0A180A219D
:101500000A2A0A360A430A4C0A5A0A680A7B0A8ED1
:101510000A9B0AA80ABB0ACE0AE10AF90A030B0AC7
:101520000B110B180B230B3A0B510B670B7C0B8B1E
:101530000B9D0B00000000000000000000000000F8
:101540000000000000A90BB90BC70BD50BEB0B007B
:101550000C120C1B0C230C2F0C3A0C450C500C5B82
:101560000C660C750C840C8F0C9A0CA40CAF0CBE82
:101570000CCE0CDC0CEB0CFB0C090D160D260D36FD
:101580000D450D5A0D6C0D7D0D900DA30DB60DCDB5
:101590000DDE0DEF0D000E150E270E320E480E5902
:1015A0000E650E770E880E940EA60EB60EC80ED9D6
:1015B0000EEE0E000F130F260F3A0F470F540F5E5B
:1015C0000F690F780F810F8D0F9D0FB10FB90FC3EA
:1015D0000FCA0FD40FE20FEB0FFB0F0D101F1030CF
:1015E00010401052105E106C1082108D100000A080
:1015F00010B610CC10E110EE10FA100711191121DD
:10160000112A113B114B115C116C1181119611A61D
:1016100011B511C311CE11DC11EC11FC110C121C0F
:10162000122C123C124D1261127512891293129BE8
:1016300012AC12BA12C612D612E212F212FB120B3E
:101640001316132113331340134D135A136B1379CD
:101650001389139D13B413C413D713E713F8130896
:1016600014181425142E1442145514631400006E1B
:10167000326F5F6D696E747073006E326F5F6D698B
:101680006E72706D006E326F5F6D617872706D009A
:101690006E326F5F726574617264006E326F5F6D7F
:1016A000696E6B7061006E326F5F6D61786B706137
:1016B000006E326F5F696E707574006E326F5F6FAF
:1016C00075747075745F6368616E6E656C006E3200
:1016D0006F5F73657474696E6773006C61756E63B8
:1016E000685F6F75745F6368616E6E656C006C61D6
:1016F000756E63685F6F75745F64656C6179006CAB
:1017000061756E63685F6F75745F70776D6C6F770E
:10171000006C61756E63685F6F75745F70776D687C
:10172000696768006C61756E63685F6F75745F7080
:10173000776D72616D70006C61756E63685F6F7557
:10174000745F6F6E74696D65006C61756E63685F60
:101750006F75745F636F6E66006961635F6D696E5C
:1017600070776D00626F6F737467617567655F6333
:1017700068616E6E656C00626F6F73746761756728
:10178000655F6F666673657400626F6F737467611F
:101790007567655F6D756C006D61705F66696C740F
:1017A00065720073706565645F73656E736F720058
:1017B0006765617273007077636F6D6D6C6F636BDB
:1017C0003000616C735F696163706F7300616E7983
:1017D0007472696D325F696E00616E797472696DE1
:1017E000335F696E0073747269675F76616C6964F8
:1017F0006174696F6E00616E797472696D335F74C4
:1018000079706500626C615F3800626F6F73745F3E
:1018100070776D5F6D617800626F6F73745F707762
:101820006D5F6D696E006961635F636F6E66320044
:101830007761726E696E675F72706D007761726E4C
:10184000696E675F6B7061007761726E696E675F6A
:10185000636F6E66007761726E696E675F61646365
:101860005F76616C7565007761726E696E675F6542
:101870006774007761726E696E675F616672007788
:1018800061726E696E675F636C74007761726E6916
:101890006E675F6368616E6E656C00616E7974720D
:1018A000696D325F7479706500626F6F73745F7415
:1018B00070735F64635F7363616C65006E326F5F4A
:1018C0006D696E676561720063796C696E646572DB
:1018D0005F6F7264657200616C735F7470735F74C4
:1018E000687265730073747269675F6D696E5F61BA
:1018F0006E676C650063616D73686166745F6578BF
:101900005F726566706F73006B6E6F636B5F6761AC
:10191000696E006B6E6F636B5F7265666572656E94
:101920006365006B6E6F636B5F63616C69627261AC
:1019300074696F6E5F6D696E006B6E6F636B5F6372
:10194000616C6962726174696F6E5F6D6178006964
:101950006E6A5F7374616765325F73746172745F1E
:1019600072706D007472616E73625F636F6E666930
:1019700067007472616E73625F696E707574007473
:1019800072616E73625F72706D31007472616E733A
:10199000625F72706D32007472616E73625F647741
:1019A000656C6C31007472616E73625F6477656C34
:1019B0006C32007472616E73625F6368616E6E6533
:1019C0006C00696E6A5F6465616474696D6500735B
:1019D00070656564325F73656E736F720066705F09
:1019E000646976696465720067656172735F6465D6
:1019F0006C617900616E797472696D315F696E0036
:101A00006C61756E63685F737065656431006E321A
:101A10006F5F7269636800616E797472696D315FBE
:101A20007479706500616363656C6C5F7265746185
:101A30007264006372616E6B696E675F636C745F82
:101A400072616E6765006372616E6B5F656E72696D
:101A5000636800616674657273746172745F656E49
:101A60007269636800767674695F636F6C64007690
:101A70007674695F69646C6500767674695F706915
:101A8000645F6B7000767674695F7069645F6B6920
:101A900000767674695F7069645F6B640076767453
:101AA000695F7069645F696C696D697400767674EA
:101AB000695F6368616E6E656C00616363656C5F2E
:101AC00072706D00616363656C5F7363616C650068
:101AD00073747269675F6D61785F616E676C6500D2
:101AE0006D697363326F75745F6D696E72706D00CE
:101AF0006D697363326F75745F6D617872706D00BC
:101B00006D697363326F75745F6D696E74707300A5
:101B10006D697363326F75745F6D61787470730093
:101B20006D697363326F75745F6D696E6D6170009E
:101B30006D697363326F75745F6D61786D6170008C
:101B40006D697363326F75745F6368616E6E656C27
:101B5000006D697363326F75745F636F6E6469746F
:101B6000696F6E73006D697363326F75745F636F55
:101B70006E646974696F6E31006D697363326F757D
:101B8000745F636F6E646974696F6E3200696E6A48
:101B90005F73697A6500636C745F63757276650064
:101BA0006D61745F637572766500636C745F7261FA
:101BB0006E676500626F6F7374616C745F636861F8
:101BC0006E6E656C006F167A16851690169B16A6BB
:101BD00016B116BB16CE16DB16EE16FF161117241D
:101BE000173717491759176417771789179817A3C5
:101BF00017B01700000000000000000000B617C278
:101C000017CD17D917E517F61704180000000000C4
:101C10000000000A181818261830183C18481855E3
:101C200018671873187F188B189B18A918BC18C848
:101C30001800000000D718E518F518081900000072
:101C40000000000000000000000000131900000068
:101C50000000000000000000000000231939194FA7
:101C600019641972197F198B199719A519B319C21B
:101C7000190000000000000000CF19DD19E819F478
:101C800019001A0E1A171A251A331A00000000003C
:101C900000461A000000000000531A000000000077
:101CA00000651A6F1A791A851A911A9D1AAD1ABA17
:101CB0001A000000000000C41A000000000000D05C
:101CC0001AE01AF01A001B101B201B301B401B517E
:101CD0001B651B791B8D1B0000961B00000000007C
:101CE00000000000000000000000000000000000F4
:101CF0000000000000000000000000A01B00000029
:101D000000000000000000000000000000000000D3
:101D100000000000000000000000000000AA1B00FE
:101D200000000000000000000000000000000000B3
:101D300000B41B000070726F68696269745F636F42
:101D40006E6669670070726F68696269745F6800C7
:101D500070726F68696269745F6C00636F6E666948
:101D6000675F73776974636800767473746F726108
:101D7000676500626C616200351D451D501D5B1D6D
:101D8000691D000000000000000000000000731D3D
:101D90000000000000000000000000000000000043
:101DA00056454D532047656E626F617264207633ED
:101DB0002C20006E0D68056909770973017002C156
:101DC000C1E133FFFFFFFFFFFFFFFFE3C104030695
:101DD0000705000102B309E801BC05E9081C04007D
:101DE00000FC04A0092C032C032E020000CC037C71
:101DF000036507AB0600000000FF30EFB7E00010FE
:101E0000134040E0004040909000004455667788C1
:101E1000004E6676838D969EA5ABB1B6BBBFC3C799
:101E2000CBCED1D4D7DADCDEE1E3E5E6E8EAEBEDD0
:101E3000EEF0F1F2F3F4F5F6F7F8F9F9FAFBFBFC42
:101E4000FCFDFDFDFEFEFEFFFFFFFFFFFFFFFFFFAE
:101E500003040506303132333435363738394142E0
:101E60004344454647480080402010080402015082
:101E7000002003401F457272003F3F000D69446817
:101E80004466376653664E6626685866B66784674A
:101E900048678F666B6660664E6549651C6DB670F7
:101EA0000000E16C0000C66DC871E16C9B6DCC75E3
:101EB000E16C916D94710000796D2478E16CC573CB
:101EC0000000746D9F75B46D6F6D6A71000064726F
:101ED000E16C1C6DB6703E6D0B710000C66DC87173
:101EE000E16C4D6F456F00007073966D28740000B3
:101EF000746D9F75B46D3E6D0B7100006472E16C82
:101F00005B6D55715E71E16C0000E16C1C6DB6702B
:101F1000E16C966D287400005B6D4D6DE16CC871CD
:101F20005E7100008B720000916D9471000064720C
:101F3000E16C5571E16C2D71E16C8B720000E16C0C
:101F4000C66DC871B46DE16C8C6D94710000B46D98
:101F5000796D2478B46DC5730000E16C746D9F7564
:101F6000B46DE16CA06DCC750000E16C1C6DB670B9
:101F7000B46DE16C6F6D6A7100003E6D0B71E16CC8
:101F8000396D33720000BF6E0000A46EE470000073
:101F9000816EE16C00003E6D0B71E16CC66DC87125
:101FA0000000396D3372E16C28740000D06D0000C0
:101FB000036B0000386FE16C2B6F0000226FE16C47
:101FC000196F00007A76E16CF37500003076E56CED
:101FD000B96D2B6D0000216DD470C6700000F471D6
:101FE0006F6D8B710000E16CC66DC871B46D8C6D46
:101FF00094710000B46D796D2478B46D3E6D0B71F1
:102000000000E16C746D9F75B46DA06DCC7500001F
:10201000E16C1C6DB670E16C176DA6700000A61E19
:10202000B81EC21ECE1EDC1EE81EF01EFC1EE61FE1
:10203000F41F02200A1F181F241F281F2E1F3E1FD7
:102040004E1F5A1F6A1F7A1F861F8A1F901F961FD6
:10205000A21FAC1FB01FB41FBC1FC41FCC1F9C1EEF
:10206000A21EA21EA21ED61FDE1FA21EA21EE61FB9
:10207000F41F0220102000002076616C3D002070CB
:102080006F733D00746300456774323A00453A004F
:102090004567743A00204D415000626F6F737420A1
:1020A0005467742000656D7074790020643A2000D4
:1020B000206B613A00523A00443A00204C3A0053F7
:1020C0003A004146523D004146523D004F464600CF
:1020D000204F4E0050756D703A00486561743A00AB
:1020E0004E65726E73743A0052693A006477656C9B
:1020F0006C3A004164763A0064633A005645206CBD
:102100006561726E3A00202020202020200020618E
:102110006374697665006961633A006469723A20A4
:1021200000706F733A20006D61780070773A005448
:1021300070733A00436C743A0045676F433A004548
:10214000676F433A004F323A302E004C613A003FFD
:102150003F2E3F004F32253D006B50613A0050004A
:10216000426174743A0054004169723A00202020A0
:1021700020200020200052504D3A0020557064610C
:1021800074696E67204669726D77617265200031EF
:102190002E312E3934004669726D776172653A20AE
:1021A00000562E452E4D2E532E00323031312D301B
:1021B000362D32392030383A3533312E312E3934FC
:1021C0000A0023204669726D7761726576657273C5
:1021D000696F6E3D006A0F6C09790D620E74007AAA
:1021E0000865097500310030004F4B0D0A000D0ADB
:1021F000005965732C206D656E7520616E642063D7
:102200006F6D6D20776F72780D0A004279650D0A47
:102210000048656C6C6F3E0D0A00424144207077A7
:102220000D0A0070774F4B0D0A004F4B0D0A00440A
:102230004BB045E240B23C0539C335DB323F30E5B7
:102240002DC22BD02909286626E5248023362202B8
:1022500021A728AC29AF2AB42BBF2CD52DFD2E40A9
:1022600030AA314633283561370B3A423D2941E9DE
:1022700045B34BC052555B00376C9ECDFAFBFBFC5F
:10228000FCFDFDFEFEFFFFFF400000000095FFFF8C
:10229000FF4100000000D5FFFFFFFF6000000000CD
:1022A000DFFFFFFFFF6600000000A5FFFFFFFF7BD1
:1022B00000000000DFFFFFFFFF4D000000000DFFEA
:1022C000FFFFFF500000020015FFFF66006500647D
:1022D00000630062006100390038003700360035C5
:1022E00000340033003200310030006600650064C5
:1022F00000630062006100390038003700360035A5
:1023000000340033003200310030004750530000E9
:1023100011241FBECFEFD0E1DEBFCDBF11E0A0E0A2
:10232000B1E0E2E4FDE801E00BBF02C007900D92CE
:10233000A831B107D9F71FE0A8E1B1E001C01D92B3
:10234000AC3EB107E1F70E94431D0C949FC60C946C
:102350000000909160018091AF0A981710F450E04E
:102360000FC0809167019091680150E02091C109F0
:1023700048E2249F900111248217930708F051E04E
:10238000852F0895409191018091AE0A85FD4460AA
:1023900084FD40683091940B20E08091930B90E095
:1023A000822B932B90931A058093190540939101EA
:1023B0000895CF93DF93562F40E0C72FD0E09C01C4
:1023C000209789F08FEF4B3F580710F08FEF0DC02B
:1023D000CA01A0E0B0E080509040AF4FBF4FABBF0C
:1023E000FC01879102C0FA0184912827822F8295EF
:1023F0008227082E869586958025082E869580252D
:102400008770022E232F869507948795302D2827D5
:1024100006948795302528274F5F5F4F442309F0A6
:10242000CFCFC901DF91CF910895CF92DF92EF9284
:10243000FF921F93CF93DF9380912C0290912D02F6
:1024400091FDC4C0192F1C7FBC01737020912A021A
:1024500030912B02562F4427C72FDD27209789F074
:102460008FEF4B3F580710F08FEF0DC0CA01A0E06F
:10247000B0E080509040AF4FBF4FABBFFC018791A1
:1024800002C0FA0184912827822F82958227082E84
:10249000869586958025082E869580258770022E44
:1024A000232F869507948795302D282706948795A6
:1024B000302528274F5F5F4F442309F0CFCFAB0172
:1024C0004F5F5F4F4130510571F48EEE97EFA1E001
:1024D000B0E0ABBFFC01879196912817390709F04E
:1024E00067C0146065C04230510571F480EF97EF0A
:1024F000A1E0B0E0ABBFFC018791969128173907A6
:1025000009F056C0186054C04330510571F482EF91
:1025100097EFA1E0B0E0ABBFFC018791969128173F
:10252000390709F045C0106143C04430510571F4CA
:1025300084EF97EFA1E0B0E0ABBFFC0187919691EB
:102540002817390709F034C0106232C08AEF97EFBC
:10255000A1E0B0E0ABBFFC0187919791A791B69144
:102560006C017D018D2D9E2D91704817590779F4CE
:1025700086EF97EFA1E0B0E0ABBFFC0187919691A9
:102580002817390709F4106448EF51E011C082E0C0
:102590004030580779F488EF97EFA1E0B0E0ABBF87
:1025A000FC01879196912817390721F4106802C021
:1025B0002FEF3FEF912F80E0842B952B90932D02EE
:1025C00080932C0230932B0220932A02DF91CF912B
:1025D0001F91FF90EF90DF90CF90089510922D0201
:1025E00010922C028FEF9FEF90932B0280932A0280
:1025F0000895482F4F70807F6827423009F49DC0AE
:10260000433030F4442359F0413009F0B6C053C090
:10261000463009F499C0473009F0AFC099C0862F01
:1026200090E08077907034E0959587953A95E1F742
:10263000E82F67FF2EC030919E01332391F08091E7
:10264000910186FF0EC020918E01822F82958F709E
:10265000831720F4285820938E0107C0295820930F
:102660008E018091520180FF06C0809155018062E9
:10267000809355010895F0E0E851FE4F90818091DC
:10268000A201892B8093A2012BB3892F80958223ED
:102690000DC0F0E0E851FE4F90812091A201892FFA
:1026A000809582238093A2018BB3892B8BBB8AB345
:1026B000982B9ABB0895862F90E08077907024E045
:1026C000959587952A95E1F7382F8230E8F467FFD2
:1026D0000DC02091650081E090E002C0880F991F35
:1026E0003A95E2F7282B2093650008952091650024
:1026F00081E090E002C0880F991F3A95E2F780953B
:10270000822380936500089567FF0BC028B381E0A2
:1027100090E002C0880F991F3A95E2F7282B28BB5A
:10272000089528B381E090E002C0880F991F3A9580
:10273000E2F78095822388BB08958091520181FD44
:102740001CC0E5E6F0E006C08091520182FD15C094
:10275000E2E3F0E085B38F70682B65BB908121E0E8
:1027600030E002C0220F331F4A95E2F7822F809596
:10277000982390838081822B808308950895089503
:1027800008950895089580916501882379F08091D6
:102790002B0580FF0BC0F8948091AC0A60E80E9482
:1027A000F912789480912B058E7F0AC0F89480915D
:1027B000AC0A60E00E94F912789480912B05816048
:1027C00080932B05089580913A05806280933A05A5
:1027D00008950895809140058150809340058F5F52
:1027E00061F49091570992959F708FE0891B8093B7
:1027F00040050E9422B50E9461B48091570982FD74
:1028000020C060915D09862F8F708F3049F08091D4
:10281000BF019091C0014EE223EC31E00E94C2B7AB
:102820006091A40A862F8F708F3009F45CC080916C
:10283000BD019091BE014EE329EB31E00E94C2B789
:10284000089560915D09862F8F708F3019F1809106
:10285000BF019091C00174E0969587957A95E1F754
:10286000807F9F704EE223EC31E00E94C2B78091DE
:10287000BF019091C00164E0880F991F6A95E1F74C
:1028800060915D09605F807F9F704EE423EC31E0D2
:102890000E94C2B76091A40A862F8F708F3019F101
:1028A0008091BD019091BE0154E0969587955A950F
:1028B000E1F7807F9F704EE329EB31E00E94C2B7C1
:1028C0008091BD019091BE0144E0880F991F4A9507
:1028D000E1F76091A40A605F807F9F704EE529EB6D
:1028E00031E00E94C2B708958091FE0982FF03C0C3
:1028F0000E940C5A08950E94FB560895CF93DF93CF
:1029000080916501882391F0909165018091B709CC
:10291000891718F00E94833309C00E94FF3EF89483
:10292000809154018F7E8093540178940E94F237F5
:1029300080916401882389F0809164018031B8F02E
:1029400080913A05806280933A05809110088E5FED
:10295000809310080E944C380AC0F894C09162011C
:10296000D091630178942FE7CD3BD20710F0CCEBE8
:10297000DFE70E9467348091FD088F708F5FE82F3A
:10298000F0E0EE0FFF1FE758FA4F85919491AC01EC
:102990002227D59FD001C49FC001D49F900DA11DB7
:1029A000B21FC59F900DA11DB21F1124CD01AA27F2
:1029B000BB2751E08030950710F480E091E09093C0
:1029C0003D0580933C05DF91CF9108958091630A86
:1029D00086FF06C08091C90A882311F40E94E05F37
:1029E0000895CF92DF92FF920F931F93CF93DF93BF
:1029F00080916A0C80FF89C0F8948091920B90912D
:102A0000930B0CB51DB51093930B0093920B081705
:102A1000190748F48091940B9091950B019690932F
:102A2000950B8093940B7894C090A60CD090A70C33
:102A3000F090A20C6091A10CC091A40CD091A50CB7
:102A40000C151D0520F4962F80E0C81BD90BF61637
:102A5000D9F06F1568F48F2D861B682FC8010E946E
:102A6000921D672F782F892F9927C60FD71F0AC06D
:102A70006F19C8010E94921D672F782F892F9927FF
:102A8000C61BD70BF092A10CD093A50CC093A40C3D
:102A90001093A70C0093A60C8091A30C882349F0F7
:102AA000C8018C199D09C80FD91FD093A50CC093DC
:102AB000A40CC8016F2D0E94921D672F782F892FBB
:102AC0009927C61BD70BD53530F0FF2031F4109273
:102AD000A50C1092A40C80E00FC0DC3A60F4C80191
:102AE0006F2D0E94921D672F782F892F9927709341
:102AF000A50C6093A40C80E88093A30C882319F0A4
:102B00000E94E79902C00E94DF990E94E3B5DF911D
:102B1000CF911F910F91FF90DF90CF9008950E9469
:102B2000A5450E94B94580913A05806980933A0590
:102B300008950E94853F0E9484450E945A45089549
:102B40008091B50D882311F00E9495BC089587E609
:102B500099E00E94364680913A05896080933A0553
:102B600008950E9432B18091630A86FF09C0809166
:102B7000C90A882319F00E94A26008950E94DF7894
:102B800008950E942F4708958091FE08882329F018
:102B900083E597E00E94028604C0109253071092CA
:102BA000A00180914309882329F088E192E00E94E6
:102BB0000286089510921802089580915807843073
:102BC00050F083E597E06091FE080E94CB858091EC
:102BD00053070E948F8580911D02843030F088E178
:102BE00092E0609143090E94CB8508958091FE098F
:102BF00083FF09C08091BC0B882319F00E945557B0
:102C000008950E940059089580917A0A90E080FD0D
:102C100002C040E001C040E830917B0A3F5FBC0148
:102C2000627070703CC03150E32FF0E0E851FE4F0D
:102C30009089292F287785B38F70842B93FF06C046
:102C40009077892B85BB9698969A0CC0822B85BB72
:102C5000809165008B7F8093650080916500846022
:102C60008093650061157105D1F0205195B39F7077
:102C7000822F8F78942B882331F02077922B95BB6D
:102C80009698969A0CC0922B95BB809165008B7F8D
:102C90008093650080916500846080936500332394
:102CA00011F6809177018823C1F08091BF0B86FFD8
:102CB0000EC0409175014295407F80917601482B6E
:102CC00050E056648CE792E262E00E94BD241092CC
:102CD0007601809176018093750108952091940B7F
:102CE0003091950B80917D0A90E082179307B8F49C
:102CF0008091980B9091990BA0919A0BB0919B0B9E
:102D0000CD01AA27BB27281B390B832F9927892B95
:102D100049F4223020F080917C0A821718F00E943A
:102D2000D1350895F8940E9404160E949541789434
:102D3000F6CF8091630A87FF3CC0809118018823F9
:102D400099F08150809318018823F1F4F8948091D0
:102D5000E701877F8093E70185B38F70806B85BB28
:102D60009798979A789410C083E080931801F8940C
:102D70008091E70188608093E70185B38F7080635D
:102D800085BB9798979A78948091E70184FF09C052
:102D9000F89485B38F70806A85BB9798979A7894DA
:102DA00008C0F89485B38F70806285BB9798979A16
:102DB00078948091830A882359F080917201882346
:102DC00039F0F89480917201815080937201789467
:102DD00080912D05815080932D058823A1F48AE0F0
:102DE00080932D0580912E0590912F05019690934B
:102DF0002F0580932E058091F30981FD02C00E946A
:102E000091990E94EA6A0E94BF21809184088823D8
:102E1000D1F08150809384088823A9F4509135081B
:102E20008CE792E261E040E00E94BD2450913908B5
:102E300040E080913A0890E0482B592B8CE792E2D1
:102E400064E00E94BD248091530180FF02C00E9473
:102E500086400E9491330E9401BB0895482F8091C3
:102E6000A309282F30E0C901887A90708038910535
:102E700041F5F901E770F070EE0FFF1FEE5AF24FC7
:102E80000190F081E02D26FD02C021E004C0842FD6
:102E9000411181E0282F8AE0EB3AF80710F020E09A
:102EA00003C0E655F54068F480918C0190E096955A
:102EB0008795969587958170821719F0822F0E94C9
:102EC000FE43089587E89AE00E9436460E942E1736
:102ED0000895CF93DF93EC01653178F4462F50E0ED
:102EE000FA01EC59FA4FE4916DE7E69FB001112425
:102EF000680F791F81E495E0A9C0673109F44EC0DD
:102F0000683130F46531C1F0663109F0A1C056C0B6
:102F10006B3109F47EC06E3109F465C0683109F087
:102F200097C060913C0570913D05680F791F81E461
:102F300095E048E150E08AC08091FE0982FF0EC012
:102F40006091090A70E06F7370706F5F7F4F762F2A
:102F500066276C0F7D1F81E495E01DC06091C60A55
:102F600080912B0581FD60958091090A813F10F0C9
:102F70009AEF02C0982F965F84E6989FC0011124B3
:102F80000E94921D672F782F892F9927C60FD71F70
:102F900081E495E0BE0145E150E058C08091AC0A63
:102FA0008F708F3009F454C00E942048C80FD91F79
:102FB00081E495E0BE0147E150E048C080919B0A62
:102FC00090E0807F907095958795882309F440C0A4
:102FD0006AEF869FB00111246C0F7D1F81E495E09C
:102FE00046E150E033C020919C0A2F70220F81F1FE
:102FF00030E08DE491E0289FB001299F700D389F4B
:10300000700D11246C0F7D1F81E495E04EE150E0BE
:103010001DC08091570990E0807F9070B3E0959536
:103020008795BA95E1F7282F882391F030E08DE459
:1030300091E0289FB001299F700D389F700D1124D9
:103040006C0F7D1F81E495E04BE150E00E94BE6172
:10305000DF91CF9108952F923F924F925F926F929E
:103060007F928F929F92AF92BF92CF92DF92EF9218
:10307000FF920F931F93DF93CF9300D000D0CDB773
:10308000DEB78CEB9FE790933D0580933C0581E490
:1030900095E00E94BB61F8948091920B9091930B04
:1030A000ECB4FDB4F092930BE092920BE816F906A3
:1030B00048F48091940B9091950B01969093950B09
:1030C0008093940B78940FE10150C701602F0E9408
:1030D000691785E191E0E80EF91E0023A9F751E098
:1030E000452E512C4AE0242E38E2332E0E94BF4355
:1030F0008BEC9BE069EF7BE00E94DD9680913905C7
:1031000085FF28C0F8948F7D80933905789480914D
:1031100019010E946DAD80911901882319F498E07E
:103120009093190180911901815080931901909118
:10313000680C913178F08091B00B882311F08150A8
:1031400039F49F3F11F080E003C00E94EF998BE0BB
:103150008093B00B8091680C813108F451C080914C
:103160003A05882309F44CC080913B058823B9F0C7
:10317000809112080E94D720882309F441C0C2011F
:103180000090120802C0880F991F0A94E2F78095F8
:1031900020913A05822380933A0510923B05909145
:1031A0003A0595FF04C0A5E0A093120822C092FF43
:1031B00004C0B2E0B09312081CC094FF04C0E4E065
:1031C000E093120816C097FF04C0F7E0F0931208CE
:1031D00010C093FF04C083E0809312080AC090FFE0
:1031E00003C01092120805C096FF0AC096E09093A3
:1031F0001208809112080E94D220A1E0A0933B0502
:103200000E941FB20E945D9B882341F0F894809138
:10321000390580648093390578941EC28091390500
:1032200086FF0CC00E94239C0E94179DF8948091F9
:1032300039058F7B8093390578940EC284FF06C0D0
:10324000F8948F7E80933905789406C2982F9370F6
:1032500009F4ACC1913021F0923009F0A2C137C01D
:103260008091A50B882319F081508093A50B809144
:10327000B30B882319F081508093B30B9091A60B68
:103280009923A9F08091530182FF11C08091A70B6F
:10329000882351F491509093A60B8091F109829567
:1032A0008F70880F880F8C5F81508093A70B0E94CE
:1032B0006AB180913005882311F00E949A40F894F9
:1032C000809139058F5F809339057894C5C18091CD
:1032D000BF0B86FD06C080917301909174010E941E
:1032E000074F80916501882309F450C19091AE0A7F
:1032F000E92FEF70E83008F0F5C0892F807309F4EA
:10330000F1C0F0E0EE0FFF1FEE5AF24F0190F08196
:10331000E02DB0E1E030FB0708F0E4C084E0F69572
:10332000E7958A95E1F7809191018370833091F55B
:103330008091BB09E81728F08091BC098E1708F02E
:1033400025C140916001809191018150809391014C
:103350008091DB092091AE0A822790E08F709070F7
:10336000892B09F007C28091540186FF03C0809128
:10337000210902C08091000A282F30E0842F90E0BC
:10338000281739070CF4F6C180918C018360809373
:103390008C01EBC1823009F0B7C080919101847833
:1033A00009F44BC0F091B00AFF3F19F426E930E070
:1033B00006C02F2F30E0220F331F220F331F6090E3
:1033C000930B7724B090940BAA24D301AA29BB298C
:1033D0006091190570911A05AD01461B570B4217F4
:1033E000530708F4D3C0C901880F991F84179507A4
:1033F00028F4B0931A05A0931905B0C1260F371F02
:1034000030931A0520931905A9C18091BC09282F72
:103410002A50253F08F0282F9091BB09892F815011
:10342000843F08F4965F2E1708F4B0C0E91708F43B
:10343000ADC0336030939101A9C08091DB0998271A
:10344000892F90E08F709070892BC1F580918C014D
:1034500081FF34C08091BC09282F2A50253F08F0F5
:10346000282F9091BB09892F8150843F08F4965FE3
:103470002E1708F47AC1E91708F477C180918C01FE
:103480008E7F80938C01909160018091540186FF22
:1034900003C08091210902C08091000A282F30E0EA
:1034A000892F90E0281739072CF080918C018D7FAF
:1034B00080938C0180919101815066C08091BC09FC
:1034C000282F2A50253F08F0282F9091BB09892FDB
:1034D0008150843F08F4965F2E1708F44BC1E9171A
:1034E00008F448C18091910188774EC0209167010E
:1034F000309168018091C109839DC0011124281772
:10350000390708F443C03EC1882349F58091B00AC9
:10351000282F30E08090930B9924D090940BCC24EA
:10352000F401EC29FD296091190570911A05AF018C
:10353000461B570B4217530748F1C901880F991FC3
:103540008417950728F4F0931A05E09319051DC117
:10355000260F371F30931A052093190516C1809145
:10356000BC09282F2A50253F08F0282F9091BB092D
:10357000892F8150843F08F4965F2E1738F0E917A1
:1035800028F0809191018360809391010E94F43A28
:10359000F894809139058C7F846080933905789404
:1035A0005BC0F8948C7F80933905789490913905AD
:1035B000892F8C7009F43CC08830B9F08C3009F147
:1035C000843089F5809110088F5F809310080E94E5
:1035D0004C380E940C490E943851F894809139056A
:1035E0008C5F80933905789437C00E941E3A0E9400
:1035F000D4360E949538809139058C5F80933905C7
:103600002BC00E944A3E8091BF0B86FD02C00E94E3
:103610004D4DF8940E944F4180913905837F8093EE
:103620003905789419C0F894937F9093390578946C
:103630008091540180FF1AC0F894809154018E7FCC
:103640008093540178940E94BC33F894809139059A
:10365000816080933905789480913F0581508093F3
:103660003F058F5F09F042CD20923F0586ED9BE03C
:103670006BEC7BE00E946895F8948091920B90919E
:10368000930BECB4FDB4F092930BE092920BE8161E
:10369000F90648F48091940B9091950B01969093C4
:1036A000950B8093940B7894E0914505F091460535
:1036B000FC83EB83CF018E199F0997FF25C01091E2
:1036C0004705E12FF0E0EE0FFF1FEA5DFA4F85910D
:1036D00094919A83898381E495E00E941662A9817E
:1036E000BA81FD010995173111F0FC82EB828B81C3
:1036F0009C81612F0E94691780913F0581508093C2
:103700003F058F5F09F0F2CCB9E0B0933F0580919F
:103710003E058150863008F085E080933E0582307A
:10372000A1F0833030F4882369F0813009F0DECCD9
:1037300006C0833069F0853009F0D8CC0CC00E94F7
:103740008A52D4CC0E94D348D1CC0E945B53CECCB9
:103750000E948850CBCC0E942E4EC8CC3091910153
:103760003877FF3F09F066CE50CE0E940049809323
:10377000A1010CCF909160018091AF0A981708F4D5
:1037800005CFB4CE0E94C21101CF809191018F5F0D
:10379000FBCECF93DF938091F30981FD02C00E949D
:1037A000DD9780913A05846080933A058091770196
:1037B000882359F1F8942091940B3091950B8091C6
:1037C000920B9091930BC92FD22F80916B01909106
:1037D0006C0178949E01281B390B832F9927892B24
:1037E000A1F4223090F0243640F48091BF0B85FD87
:1037F00004C0F8940E9404167894C456D040F894FB
:10380000D0936C01C0936B017894DF91CF910895B0
:103810001F9310915201187F8091A00987FF16C055
:1038200080913508833051F081E70E94E979136077
:103830008091FE0982FD1DC014601BC0F89485B301
:10384000806F85BB9698969A789413C08091A20950
:103850008F3E29F48091A1098E3B39F40AC08E3D38
:1038600021F48091A109843021F081E70E94E97957
:10387000176017FD1760109352011F9108950E9461
:1038800015120E94081C0E947B6080913F0D8E7F64
:103890008C3F51F480914C0D815080934C0D8F5F83
:1038A00019F481EE80933F0D08959FEF9BBB9ABB67
:1038B00081E088BB87EF87BB84E085BB94BB83EE48
:1038C00082BB88EE81BB13B88AE382B91092620092
:1038D000109261008CE18093650087E18093640021
:1038E0000E9404160E94B76180E06BEC7BE00E94AE
:1038F0001D6B1092E7010E9496400E9407650E948E
:10390000E12489EF9BE00E94769486ED9BE00E9483
:1039100076940E94DB4180E00E94FE430E94C3290E
:103920000E94081C809105098E3D11F060E001C0E5
:103930006FEF8BEC9BE00E94088780916A0A90E011
:10394000880F991F880F991F8093C50B0E94A9208B
:103950000E94B2210E94853F0E94F23710925301CB
:1039600084E18093540110925501109265018FEF0C
:1039700080936401109268011092670180910A0A95
:103980008F7080936E0181E080938E0110928F0181
:103990008091DE0980FF1FC02091580130915901AC
:1039A0008091660A8F70823051F487E0283F380793
:1039B00080F4E3E036952795EA95E1F708C083E0C7
:1039C0002C3F380730F43695279536952795822F6A
:1039D00004C08FEF02C080916001809361018091EB
:1039E000790A90E080509F4F909374018093730107
:1039F0000E94CB200E94B89E0E94D2310E94C4999E
:103A00000E94B6560E946E4D0E9486400E94EC793C
:103A10000E94BE830E94EDAE0E949BA10E94B4B0A2
:103A20000E94DEB00E94CCB08AE080932D0581E038
:103A300080932C050E94BBB70E9499B683E38093C4
:103A40007C088091630A82FF03C080E48093B50DF7
:103A50000E94EFBE83E295E069E579E00E94189F3D
:103A60000E94ECB38CE095E069E579E00E94189F34
:103A700010922D0210922C028FEF9FEF90932B0249
:103A800080932A0208950E941A6A0E94551C0E947F
:103A9000C8630E94203678940E946D20882331F0FC
:103AA00081E08093BC0B88E28093C30B0E942B18AB
:103AB00080E090E00895FC018FEF9FEF9183808379
:103AC000138212821482158216821782108608953C
:103AD000FC01828193818617970728F473836283A0
:103AE0000097F9F0BC01808191816817790738F45B
:103AF000718360832FEF8F3F920799F0BC01CB0158
:103B0000A0E0B0E02481358146815781280F391F1C
:103B10004A1F5B1F248335834683578380858F5FCD
:103B20008087089555274427869F9001969F300DE2
:103B3000411D1124B901CA0108950F93382F801730
:103B400050F5061710F0422F26C0681BE62FF0E054
:103B5000EE0FFF1FE758FA4F85919491031BBC01AC
:103B6000BB27AA27609FC001709F900DA11D112443
:103B7000892F9A2FAB2FBB27982F421738F0842F0D
:103B8000821B989FC0011124491B05C0241B829FE2
:103B9000C0011124490F842F0F9108950F93982F7E
:103BA000342F681718F00E949D1D06C0862F692FBC
:103BB000422F232F0E949D1D0F9108950F93782F60
:103BC000801708F048C0061710F0A90144C0681B10
:103BD000E62FF0E0EE0FFF1FE758FA4F8591949122
:103BE000071BBC01BB27AA27609FC001709F900DD7
:103BF000A11D1124BC0142175307C0F0CA01821B4A
:103C0000930BFC0122277F9FD0016E9FC0017E9FF6
:103C1000900DA11DB21F6F9F900DA11DB21F112409
:103C2000CD01AA27BB27481B590B15C0241B350BF8
:103C3000EE27739FD001629FC001729F900DA11D5E
:103C4000BE1F639F900DA11DBE1F1124CD01AA2789
:103C5000BB27480F591FCA010F910895282F8417B9
:103C600010F080E00895461710F08FEF0895681B5C
:103C7000E62FF0E0EE0FFF1FE758FA4F8591949181
:103C8000421B9C01BB27AA27249FC001349F900D93
:103C9000A11D1124892F9A2FAB2FBB270895FC015A
:103CA000D901615020E002C02F5F3196261718F429
:103CB00080814817C8F78081481728F011966C93C7
:103CC00011976C930895222329F411961C92119751
:103CD0001C92089511962C93119721502C930895BE
:103CE000CF92DF92EF92FF920F93DF93CF9300D0AA
:103CF000CDB7DEB77C01042F69019E012F5F3F4FD6
:103D00000E944F1EA981B0E0EA812E2F30E0C7014A
:103D10008A0F9B1FE20EF31EAC0DBD1D2C0D3D1D29
:103D2000FC018081F70160814C91F90120810E94A2
:103D30009D1D0F900F90CF91DF910F91FF90EF900D
:103D4000DF90CF900895CF93DF93DC01E9016150BC
:103D500090E002C09F5F1196961720F4FD018491B8
:103D60004817C0F7992319F41982188203C0998360
:103D700091509883DF91CF91089599E2899FC00176
:103D80001124AC012227579FD001469FC001569FA6
:103D9000900DA11DB21F479F900DA11DB21F1124B0
:103DA0009295A295B29580EFBA27B823BA27A92792
:103DB000A823A9279D01C90108959DEC899FC001F1
:103DC0001124EE27979FA001869F9001969F300DAA
:103DD000411D5E1F879F300D411D5E1F11246BE04A
:103DE00056954795379527956A95D1F7C901089556
:103DF000E9E2552744278E9F90019E9F300D411D7B
:103E00001124BB27AA276E9FC0017E9F900DA11D84
:103E10001124232F342F452F5527892F9A2FAB2F6D
:103E2000BB27F9016627F99FA001E89F9001F89F41
:103E3000300D411D561FE99F300D411D561F1124A5
:103E4000232F342F452F5527C901089520E8E22F4D
:103E5000552744278E9F90019E9F300D411D1124B0
:103E60008CEDF82FBB27AA276F9FC0017F9F900D75
:103E7000A11D1124232F342F452F5527892F9A2F29
:103E8000AB2FBB27F9016627F99FA001E89F90019E
:103E9000F89F300D411D561FE99F300D411D561FE3
:103EA0001124232F342F452F5527C901089520E1D0
:103EB000E22F552744278E9F90019E9F300D411D74
:103EC000112489E2F82FBB27AA276F9FC0017F9F8B
:103ED000900DA11D1124232F342F452F5527892FF5
:103EE0009A2FAB2FBB27F9016627F99FA001E89F06
:103EF0009001F89F300D411D561FE99F300D411D67
:103F0000561F1124232F342F452F5527C9010895FB
:103F1000FC0181818283908191836083691708F419
:103F2000692F8281891708F4892F861708F4682F72
:103F3000862F0895FC019B01861797072CF49A01A0
:103F40004E175F070CF49F01C9010895681724F00C
:103F5000642F48170CF4682F862F0895681720F0F7
:103F6000642F481708F4682F862F0895861708F4E1
:103F7000682F862F0895681708F4682F862F0895F4
:103F800050E070E09B01429FB001439F700D529F33
:103F9000700D112420E130E0241B350B90E0AC01C2
:103FA000249FC001259F900D349F900D1124860FF2
:103FB000971FA4E096958795AA95E1F70895FC01CF
:103FC000CB01642F442321F155274427869F90017C
:103FD000969F300D411D11246195BB27AA27E69FAE
:103FE000C001F69F900DA11D1124820F931FA41FE5
:103FF000B51F292F3A2F4B2F552787FD02C0F901F6
:1040000007C0C901019619F4EFEFFFEF01C0FC01F1
:10401000CF010895FC01842F82958F70A82FB0E006
:10402000262F30E0C9010197A817B9072CF0E20F3D
:10403000F31F3197808108954F70642F70E0EA0F6D
:10404000FB1F818190E0869FA001879F500D969F66
:10405000500D1124208130E080E190E0861B970B09
:10406000BC01269FC001279F900D369F900D112403
:10407000480F591F34E0569547953A95E1F7842F3C
:104080000895FC01842F82958695877011F48081B4
:1040900008954F7150E0E80FF11D808190E0849FFA
:1040A000B001859F700D949F700D11243197208170
:1040B00030E080E290E0841B950BAC01249FC001AE
:1040C000259F900D349F900D1124860F971F45E07A
:1040D000969587954A95E1F7089580EF9FEFA1E0C7
:1040E000B0E0ABBFFC018791863751F481EF9FEFC1
:1040F000A1E0B0E0ABBFFC01879190E0833309F011
:1041000091E0892F08950F93082FFB0182958F70FE
:10411000682F6295607FE80FF11D862F615F4081F7
:1041200021810E949D1D0F910895282FFB01E90F09
:10413000F11D3081882359F08181289FC00111240D
:104140002195329F90011124820F931F392F832FC5
:10415000089587E886B9E3E1F8E020E0822F8770D0
:10416000806487B9369A349BFECF349A84B195B176
:10417000880F991F819391932F5F203179F70895CC
:104180008770806487B9369A349BFECF349A24B105
:1041900035B1C90108951092120880E487B987EFFC
:1041A00086B908958770806487B9349A0895349BDE
:1041B00007C0E0911A01E81729F0349A80931A0198
:1041C00080E00895E530A9F440910F08403478F478
:1041D00084B195B120910D0830910E08820F931F84
:1041E00090930E0880930D084F5F40930F0881E075
:1041F0000895F0E024B135B1EE0FFF1FED5EF74FEB
:104200008081918196958795820F931F91838083FA
:1042100081E0089580910F08882309F42DC0E82FCC
:10422000F0E0EE0FFF1FE758FA4F2591349180918F
:104230000D0890910E08BC014427739FD001629F26
:10424000C001729F900DA11DB41F639F900DA11D11
:10425000B41F11246FE0B695A795979587956A9539
:10426000D1F790931E0880931D0810920E081092AB
:104270000D0810920F0881E008951F920F920FB65B
:104280000F920BB60F9211242F933F938F939F930E
:10429000AF93BF93EF93FF932091680CE22FF0E070
:1042A00084B5DF01AB5CB34F92968C9384B195B12A
:1042B000EE0FFF1FEB5CF34F918380832F3039F4B7
:1042C000809112088770806487B9349A03C02031C6
:1042D00008F033982F5F2093680C8EB79DB7382F66
:1042E00020E0892F90E0822B932B2091E80D3091D4
:1042F000E90D2115310519F08217930720F49093E9
:10430000E90D8093E80DFF91EF91BF91AF919F91DF
:104310008F913F912F910F900BBE0F900FBE0F907A
:104320001F901895282FE82FEF70E63011F480E0E9
:104330000895F0E0EE0FFF1FED5EF74F8081918151
:10434000B3E096958795BA95E1F7E82F24FF05C06D
:1043500080E0E61730F481E0089580E06E1708F4FD
:1043600081E008958091A00986FF08C085E08093D0
:10437000350880913A05806480933A05089520912C
:10438000A00927FF4AC080913508833009F445C051
:10439000853099F480913A0586FD3FC080911F08D1
:1043A0009091200833E0969587953A95E1F781340E
:1043B000910588F41092350808958230C9F49091DF
:1043C000A10980913A08981779F49091A2098091F7
:1043D0003908981749F426FF05C08091620080646F
:1043E0008093620083E001C084E0809335080895E3
:1043F00080913608882389F41092350881E08093F3
:10440000360810923708EFEBFDE1E491E0939C0051
:1044100080919A00806280939A000895823130F4EE
:10442000E82FF0E0E056F24E8491089582518630F4
:1044300030F4E82FF0E0E050FF4F8081089587309E
:1044400011F080E008958EE5089580912E0508957D
:10445000883070F4E82FF0E0EE0FFF1FEE5AF24FB5
:10446000808191812FEF8F3F920711F0892F08955E
:1044700080E00895883060F4E82FF0E0EE0FFF1F31
:10448000EE5AF24F808191812FEF8F3F920709F40E
:1044900080E00895282F30E08031E0F48695E82F01
:1044A000F0E020FF0BC0EE0FFF1FEE5AF24F8081AD
:1044B00091812FEF8F3F920799F00895EE0FFF1F24
:1044C000EE5AF24F808191812FEF8F3F920741F09A
:1044D000892F0895E2E3F8E0E21BF30B8081089551
:1044E00080E008958F3F11F480E00895E82FF0E018
:1044F000ED54F64F80810895982FE0913B08F0E04D
:10450000A3E0EE0FFF1FAA95E1F7E05CF74F2081D3
:104510008181992329F0913011F08AE70895822F43
:104520000895E0913B08F0E0B3E0EE0FFF1FBA956D
:10453000E1F7E05CF74F0190F081E02DE80FF11D0D
:1045400080810895282F882339F48FEF9FEF90936F
:10455000800880937F080AC0803240F0803219F4CE
:10456000E0917F083CC0E091800839C0822F90E044
:1045700020FF03C0E0911D0113C0E0913B08F0E073
:1045800023E0EE0FFF1F2A95E1F7E05CF74F019063
:10459000F081E02DE80FF91F818180931D01E081FA
:1045A00080917F08909180088E27282F22952827B8
:1045B000022E269526952025022E26952025277049
:1045C000082E892F269507942795902D82270694EB
:1045D0002795902582279093800880937F088E2FBF
:1045E0000895E0913B08F0E033E0EE0FFF1F3A95AD
:1045F000E1F7E05CF74F0190F081E02DE80FF11D4D
:10460000E4918E2F0895E0913B08F0E043E0EE0F37
:10461000FF1F4A95E1F7E05CF74F20813181280FB9
:10462000311D40E050E041604BBFF9018791089592
:10463000823108F08FEF8093B70B0895E9EFFDE129
:10464000E80FF11DE4918E2F0895E82FF0E0EE0FB2
:10465000FF1FEB52F24E25913491C9010895FB01E1
:104660008C3028F48A3050F5883090F11BC08E30A1
:1046700081F08F3018F48C3059F51AC08F3019F052
:10468000803131F506C08CE0858384838BE397E02D
:1046900005C08CE08583848385EF97E093838283D4
:1046A0000C961EC088E0858384838CE693E015C059
:1046B00088E0858384838CE094E00FC080E185836B
:1046C0008EE084838EE093E093838283409608C0DB
:1046D00088E0858384838CEB93E0938382830896C0
:1046E0009183808308951F93DF93CF9300D000D0F0
:1046F00000D0CDB7DEB7823110F010E012C0E82F45
:10470000F0E0E750F24E1491112359F0883048F050
:10471000BE016F5F7F4F0E942F238D819E81890F85
:10472000180F812F26960FB6F894DEBF0FBECDBFAF
:10473000CF91DF911F9108950F931F93DF93CF9334
:1047400000D000D000D0CDB7DEB7282F823108F0DE
:104750007AC0482F50E0CA01880F991F8B52924EA1
:10476000FC01A591B4914750524EFA013491109733
:1047700009F469C090E00FEF1FEF19C08D91082771
:10478000802F82958027082E869586958025082E75
:10479000869580258770002E012F86950794879532
:1047A000102D082706948795102508279F5F9317DB
:1047B00028F3283008F449C0822FBE016F5F7F4F75
:1047C0000E942F232E81EB81FC8190E019C0819102
:1047D0000827802F82958027082E8695869580252C
:1047E000082E869580258770002E012F86950794C8
:1047F0008795102D082706948795102508279F5F19
:10480000921728F32D81E981FA8190E019C08191F6
:104810000827802F82958027082E869586958025EB
:10482000082E869580258770002E012F8695079487
:104830008795102D082706948795102508279F5FD8
:10484000921728F302C00FEF1FEFC80126960FB68C
:10485000F894DEBF0FBECDBFCF91DF911F910F91B6
:104860000895CF93DF93AC0180919E08C82FD0E0CC
:1048700021969E0127703070219780913B08821706
:1048800011F48FEF18C0F3E0CC0FDD1FFA95E1F7BC
:10489000DE01A45CB74F11965C934E93FE01E25C7F
:1048A000F74F608313961C92C05CD74F1982188211
:1048B00020939E0880E0DF91CF910895CF93DF93FE
:1048C000FC01922F80919E08C82FD0E021969E0176
:1048D00027703070219780913B088217D1F073E0E8
:1048E000CC0FDD1F7A95E1F7DE01A45CB74F11967E
:1048F000FC93EE93FE01E25CF74F608313961C92EB
:104900001397C05CD74F5983488316969C93209386
:104910009E08DF91CF910895CF93DF93FC01962FEE
:10492000B90180919E08C82FD0E021969E01277082
:104930003070219780913B088217E1F0A3E0CC0F03
:10494000DD1FAA95E1F7DE01A45CB74F1196FC9339
:10495000EE93FE01E25CF74F908313961C9213973F
:10496000C05CD74F5983488317967C936E931697F4
:1049700020939E08DF91CF91089520E00E945E244D
:104980000895FF920F931F93CF93DF938C01F62E20
:10499000F801849131960E5F1F4FE491D82FC0E04B
:1049A000AE014E0F511D82EE9DE26FEF20E00E949E
:1049B0005E24FA9469F7DF91CF911F910F91FF90D8
:1049C000089510927C0810927D0888E98AB986E0E3
:1049D000809395001092900083E389B910923B0870
:1049E00010929E088FEF9FEF9093800880937F082E
:1049F000109283080895282F909137089F5F923076
:104A000029F48333C1F41092380822C09A3051F44B
:104A100080913808821711F482E001C081E0809310
:104A2000350816C0943019F48093390804C09530C5
:104A300011F480933A0880913808822728E03CE8F6
:104A400080FB86950EF483272A95D1F7809338084A
:104A50009093370808951F920F920FB60F920BB6DE
:104A60000F9211248F93EF93FF93E09136088E2FCE
:104A70008F5FF0E0E154F24EE491E0939C008E30C1
:104A800031F480919A008F7D80939A0080E080932A
:104A90003608FF91EF918F910F900BBE0F900FBED4
:104AA0000F901F9018951F920F920FB60F9211241E
:104AB0002F938F939F9355990FC020917C082223A9
:104AC00061F090919E0880913B08981731F4109204
:104AD000900029B910927C0856989F918F912F9140
:104AE0000F900FBE0F901F9018955D9BFECF8CB955
:104AF000089590E0875B9F4F68E40E94921D47E015
:104B000096958795779567954A95D1F7E62FF0E0CA
:104B1000EE0FFF1FE758FA4F8591949168E40E94C9
:104B2000921DDC01CB0127E0B695A7959795879557
:104B30002A95D1F7885C0895DF92EF92FF920F9348
:104B40001F93DF93CF9300D000D000D0CDB7DEB756
:104B5000182F062F8091B70BE82EFF24F701E7509E
:104B6000F24ED4908F3FC1F11D15D8F4823039F444
:104B7000183058F0E12FF0E0E454FA4F2CC089309F
:104B800021F4862F0E947925082FC701880F991FCD
:104B90008B52924EFC01A591B491A10FB11D0C93C3
:104BA0001BC08830C8F0BE016F5F7F4F0E942F236B
:104BB000812F8D199E81891728F4EB81FC81E80FE4
:104BC000F11D09C0891B982F8D81981728F4E98160
:104BD000FA81E90FF11D008326960FB6F894DEBF27
:104BE0000FBECDBFCF91DF911F910F91FF90EF903E
:104BF000DF90089590E088539F4F68E40E94921DD3
:104C0000E7E09695879577956795EA95D1F7E62F32
:104C1000F0E0EE0FFF1FE758FA4F8591949168E49A
:104C20000E94921DDC01CB0167E0B695A795979590
:104C300087956A95D1F789540895FF920F931F9332
:104C4000DF93CF9300D000D000D0CDB7DEB7082FD0
:104C500080913B08482F50E0FA0173E0EE0FFF1FF0
:104C60007A95E1F7E05CF74F2081818190E0892B14
:104C700019F462E0F62E01C0FF24822F90E0FC01BF
:104C8000E750F24E14912F3F11F460E083C00117FA
:104C900008F042C0880F991F8B52924EFC0165911B
:104CA0007491A02FB0E06A0F7B1FFB016081293057
:104CB00029F4862F0E94FA25682F6CC0223031F427
:104CC000083038F0A454BA4F6C9103C0283008F073
:104CD00061C0202F30E0812F90E00197281739071D
:104CE0000CF458C093E0440F551F9A95E1F7DA0190
:104CF000A45CB74F8FEF13968C931397FA01E25C85
:104D0000F74FF0821D921C92405C574F8FE798E05E
:104D1000DA018D939C933EC0822FBE016F5F7F4F5F
:104D20000E942F23202F211B8E81281730F4EB8126
:104D3000FC81E20FF11D60812DC0281B8D81281799
:104D400010F060E005C0E981FA81E20FF11D608199
:104D500030E090E0019728173907E4F0E0913B0834
:104D6000F0E013E0EE0FFF1F1A95E1F79F01245CBE
:104D7000374F8FEFD90113968C93DF01A25CB74FA9
:104D8000FC92D9011D921C92E05CF74F8FE798E0EE
:104D900091838083862F26960FB6F894DEBF0FBED0
:104DA000CDBFCF91DF911F910F91FF900895262FD6
:104DB000982F98519031D0F5E92FE695F0E0E35324
:104DC000F24E349190FD1BC1662319F0AEE7B8E0B6
:104DD0000BC080913B08A82FB0E043E0AA0FBB1F97
:104DE0004A95E1F7AE5BB74F383068F4E32FF0E057
:104DF000EE0FFF1FEE5AF24F0190F081E02D2FEFE2
:104E0000EF3FF20709F4E0E0EC93383008F0F8C126
:104E1000E32FF0E0EE0FFF1FEE5AF24F6081718139
:104E20008FEF6F3F780709F0D3C0EAC1E82FF0E0B9
:104E3000E534F10508F0E4C1E050FE4FEE0FFF1F2E
:104E40000590F491E02D099460912E05DCC16091EC
:104E50009A01D9C160915301D6C160916601D3C155
:104E6000662319F0EEE7F8E00BC080913B08E82FCD
:104E7000F0E083E0EE0FFF1F8A95E1F7EE5BF74F5E
:104E800080915801909159018083809158019091AF
:104E9000590178C060915B01B6C160915A01B3C1FC
:104EA00060916001B0C160915701ADC18091F3097B
:104EB00081FF20C06091800C7091810CB5E07695E7
:104EC0006795BA95E1F721E06333720708F498C15A
:104ED00082E06630780710F4625395C16F557040D8
:104EE000769567956F3F710509F008F48CC16FEFF7
:104EF00070E089C18091240A85FF05C08091210856
:104F00009091220804C08091150890911608F3E052
:104F100096958795FA95E1F771C18091A1089091D6
:104F2000A20864E60FC06091A3086DC18091A40837
:104F30009091A50825E08F3F920708F063C1865E37
:104F4000904062E30E94921D672F782F892F992746
:104F50005AC1662319F0EEE7F8E00BC080913B08D8
:104F6000E82FF0E073E0EE0FFF1F7A95E1F7EE5BBC
:104F7000F74F80916701909168018083809167016C
:104F800090916801692F3FC1662319F0EEE7F8E0C0
:104F90000BC080913B08E82FF0E063E0EE0FFF1FAD
:104FA0006A95E1F7EE5BF74F8091690190916A0194
:104FB000808380916501882369F48091C00B81FF13
:104FC00009C06091850C7091860C6115710511F016
:104FD000672F19C18091690190916A01D3CF8091A7
:104FE0006501882361F48091C00B81FF08C0609146
:104FF000850C7091860C6115710509F004C122239E
:1050000019F060917E08FFC0E0913B08F0E053E0AA
:10501000EE0FFF1F5A95E1F7E45CF74F6681F3C08E
:105020006091A608F0C08091A7089091A80864E458
:105030000E94921D272F382F492F5527832F90E04C
:10504000892B09F0DFC0622FDEC06091A908DBC0A8
:1050500080917A0190917B01CCC0809173019091F5
:1050600074018E5F914008F0CDC0809173019091E2
:10507000740196958795C2C06091B70AC4C06091CB
:10508000AB08C1C060911802BEC06091740DBBC076
:105090006091760DB8C06091750DB5C06091770DC7
:1050A000B2C06091780DAFC08091540186FF02C0FC
:1050B00060E801C060E08091550181FD61608091F0
:1050C0008C01837009F0606480919101847809F00B
:1050D00060628091550187FD606180918C0182FD45
:1050E00068608091540183FD64608091D60182FFE5
:1050F0008AC0626088C0809131059091320525E0B8
:10510000969587952A95E1F779C0609199017BC0C2
:1051100080913505909136058050904C880F892FED
:10512000881F990B6BC08091B80A9091B90A892F9A
:10513000990F990B682F605866C0809154018F7742
:105140008093540160918F015EC060911B055BC02C
:1051500060911C0558C060911D0555C060911E05E9
:1051600052C060911F054FC0609120054CC06091F6
:10517000210549C080915401806880935401809139
:10518000C00B87FF05C087ED96E268E30E943124DB
:105190006091AC087091AD0887E0683F780790F5A2
:1051A000F3E076956795FA95E1F72DC060916F0170
:1051B0002AC06091A00127C06091530724C060916C
:1051C000C10121C08091BF019091C00112C08091A6
:1051D000560190E08F709070892B91F0609156018C
:1051E000607711C06091BC010EC08091BD019091AB
:1051F000BE01E4E096958795EA95E1F7682F03C034
:1052000060E001C06FEF862F08951F920F920FB6D6
:105210000F920BB60F9211242F933F934F935F93EE
:105220006F937F938F939F93AF93BF93EF93FF936E
:1052300086ED9BE00E942095292F30E0232B39F04A
:10524000559880917C08882319F0569A01C08CB932
:10525000FF91EF91BF91AF919F918F917F916F914E
:105260005F914F913F912F910F900BBE0F900FBE0A
:105270000F901F9018951F920F920FB60F920BB6BA
:105280000F9211242F933F934F935F936F937F93CC
:105290008F939F93AF93BF93EF93FF938BB18871DD
:1052A00011F08CB105C06CB189EF9BE00E947B943A
:1052B000FF91EF91BF91AF919F918F917F916F91EE
:1052C0005F914F913F912F910F900BBE0F900FBEAA
:1052D0000F901F90189586ED9BE06DE20E947B94E5
:1052E0008CE792E264E045E75BE20E94BD24559AB8
:1052F00084E68093840808951F920F920FB60F9250
:105300000BB60F9211241F932F933F934F935F93EC
:105310006F937F938F939F93AF93BF93EF93FF937D
:1053200010919C0080919B008871C9F48091840841
:10533000882331F086ED9BE0612F0E947B94559A83
:105340008091A00987FF04C0812F0E94FB2407C021
:105350008091F20981FF03C0812F0E9457BFFF9106
:10536000EF91BF91AF919F918F917F916F915F91DD
:105370004F913F912F911F910F900BBE0F900FBE39
:105380000F901F9018958091A00987FF0CC088E9A5
:1053900080939A0086E080939D001092980087E6A3
:1053A0008093990008958091F20981FF12C0809145
:1053B000920A87FD0EC088E980939A0086E0809368
:1053C0009D00109298000E9419BF8093990010923E
:1053D0009A0808950E941D26682F86ED9BE00E9482
:1053E000D59484E40895982F80913B08A82FB0E0CD
:1053F000FD0163E0EE0FFF1F6A95E1F7E05CF74FF8
:10540000808161819330A0F4992369F0913011F487
:10541000682F09C053E0AA0FBB1F5A95E1F7A45C9F
:10542000B74F16966C9186ED9BE00E94D5941BC0F9
:10543000953070F086ED9BE06EE70E947B948FEFD5
:105440009FEF9093800880937F08109283080BC091
:10545000933019F460917F0802C06091800886ED56
:105460009BE00E94979484E50895282F81E0809323
:10547000830880913B08A82FB0E0FD0183E0EE0F88
:10548000FF1F8A95E1F7E05CF74F8081618123304F
:10549000D0F4222399F0213011F061E00FC0682F81
:1054A00090E08F779070892B49F473E0AA0FBB1FAF
:1054B0007A95E1F7A25CB74F86E08C9386ED9BE08E
:1054C0000E94D5941BC0253071F486ED9BE06EE7F9
:1054D0000E947B948FEF9FEF9093800880937F08CA
:1054E000109283080BC0233019F460917F0802C02A
:1054F0006091800886ED9BE00E94979480E5089576
:10550000873360F5863311F468E723C08432E8F40A
:1055100080FD0FC086950E949C23E0913B08F0E03F
:1055200023E0EE0FFF1F2A95E1F7E45CF74F968327
:105530000FC0E0913B08F0E093E0EE0FFF1F9A955B
:10554000E1F7E45CF74F668104C084520E94732344
:10555000682F86ED9BE00E94D59419C0893360F0D6
:1055600086ED9BE06EE70E947B948FEF9FEF909318
:10557000800880937F080BC0873319F460917F08FF
:1055800002C06091800886ED9BE00E94979483E4BE
:105590000895682F80913B08A82FB0E0FD0143E0FB
:1055A000EE0FFF1F4A95E1F7E25CF74F808190E034
:1055B000AC0143505040262F30E024173507BCF48F
:1055C00004972817390711F462E30CC033E0AA0FDF
:1055D000BB1F3A95E1F7A05CB74FED91FC91862F88
:1055E0000995682F86ED9BE00E94D5941CC0019719
:1055F0002817390764F086ED9BE06EE70E947B94E4
:105600008FEF9FEF9093800880937F080CC0241742
:10561000350719F460917F0802C06091800886ED1B
:105620009BE00E94979483E70895982F823FB8F5F6
:10563000813F11F465E72EC0803F61F4E0913B08A3
:10564000F0E073E0EE0FFF1F7A95E1F7E05CF74FB3
:10565000608120C08091D60182FF02C060E01AC044
:10566000E0913B08F0E063E0EE0FFF1F6A95E1F781
:10567000E05CF74F0190F081E02DE199FECF54E01E
:10568000EE0FFF1F5A95E1F7E90FF11DFFBBEEBBCF
:10569000E09A6DB386ED9BE00E94D5941FC0843FD5
:1056A00060F086ED9BE06EE70E947B948FEF9FEFAA
:1056B0009093800880937F0811C08091D60182FF6B
:1056C00002C060E007C0923F19F460917F0802C0F9
:1056D0006091800886ED9BE00E94979480E0089599
:1056E000863468F4853411F460E204C060E00E94FE
:1056F000D726682F86ED9BE00E94D59419C0883488
:1057000060F086ED9BE06EE70E947B948FEF9FEF49
:105710009093800880937F080BC0863419F46091C1
:105720007F0802C06091800886ED9BE00E949794FC
:1057300080E00895282F80913B08A82FB0E0FD015C
:1057400083E0EE0FFF1F8A95E1F7E25CF74F80815F
:105750008150281760F086ED9BE06EE70E947B94F5
:105760008FEF9FEF9093800880937F0834C0982F2D
:10577000921B933008F1E3E0AA0FBB1FEA95E1F713
:10578000A05CB74FED91FC91963040F0309711F44A
:1057900061E00DC0E20FF11D608109C0933011F48A
:1057A00067E705C0943011F46E2F01C06F2F86EDAE
:1057B0009BE00E94D5940FC030E090E0029728173C
:1057C000390719F460917F0802C06091800886ED66
:1057D0009BE00E94979480E50895CF93DF93682F14
:1057E00090917D08913021F0923009F08FC006C071
:1057F00080931C0182E080937D08BDC180911B01D4
:105800008E3409F44EC08F34B8F4883409F442C0A1
:10581000893448F4853409F44CC0873489F18932DD
:1058200009F071C042C08A34D1F18A3408F443C00F
:105830008C3409F068C037C08835C1F0893540F430
:10584000843551F18735C9F18F3409F05CC015C03A
:105850008D35A9F18E3520F4893509F054C027C063
:105860008338B1F0873F09F04EC02BC080911C01F6
:105870008093C20B6093C10B46C01092B70B03C05C
:1058800083E08093B70B80911C010E949C253BC054
:1058900087E0F7CF81E0F5CF9093B70BF4CF8AE0A4
:1058A000F0CF8EE0EECF89E0ECCF88E0EACF8FE05A
:1058B000E8CF84E0E6CF8CE0E4CF8DE0E2CF86E075
:1058C000E0CF20911C01C62FD0E02F3F89F4AE011C
:1058D0005F6F8AEE99E26FEF0E94BD24FE01EE0F2A
:1058E000FF1FEB52F24E85919491AC0160E006C02F
:1058F000922F80E0AE01482B592B60E26A5F8AE963
:105900009BE20E94BD2410927D0835C18B3509F4BD
:105910001CC18C35A0F58C3409F422C18D34C8F437
:10592000823409F477C0833450F4893209F418C101
:10593000813409F469C0883209F01DC1D9C08434AA
:1059400009F46FC0843408F468C08B3408F013C1C4
:1059500007C1833509F476C0843550F48E3408F4D9
:105960000AC1803508F4FCC0813509F004C165C066
:10597000863508F4F5C0873508F4FDC0F1C08F36D0
:1059800009F46DC08037E0F4883609F484C08936A4
:1059900050F4853609F4BEC0873609F46AC08D35E7
:1059A00009F0E9C0DDC08A3609F487C08A3608F4F8
:1059B000BAC08C3609F493C08E3609F0DCC086C0BC
:1059C000823809F45FC0833880F4863709F440C018
:1059D000873720F4843709F0CEC066C0873709F4D2
:1059E000ABC0893709F0C7C08CC0803A01F1813A59
:1059F00020F4833809F0BFC0B3C0873F09F4B0C0BA
:105A0000883F09F0B8C0B2C01092B50D87ED96E29C
:105A100068E3AFC00E94E943AEC085E292E261E074
:105A2000A8C01092B50D87ED96E267E4A2C010926F
:105A3000B50D80E79BE269E49CC01092B50D82EE43
:105A40009EE204C01092B50D8EE092E26AE191C030
:105A50004091B70B8DE196E26FEF50E07EC010925F
:105A6000B50D1092B70B8DE196E26FEF40E050E07C
:105A700074C083E08093B70B8DE196E26FEF43E053
:105A800050E06BC087E08093B70B8DE196E26FEF3B
:105A900047E050E062C081E08093B70B8DE196E271
:105AA0006FEF41E050E059C082E08093B70B8DE189
:105AB00096E26FEF42E050E050C08AE08093B70B6F
:105AC0008DE196E26FEF4AE050E047C08EE08093B0
:105AD000B70B8DE196E26FEF4EE050E03EC089E0FB
:105AE0008093B70B8DE196E26FEF49E050E035C04F
:105AF00088E08093B70B8DE196E26FEF48E050E0CD
:105B00002CC08FE08093B70B8DE196E26FEF4FE0F2
:105B100050E023C084E08093B70B8DE196E26FEFF5
:105B200044E050E01AC08CE08093B70B8DE196E220
:105B30006FEF4CE050E011C08DE08093B70B8DE12A
:105B400096E26FEF4DE050E008C086E08093B70B1F
:105B50008DE196E26FEF46E050E00E94BD240BC05D
:105B600081E080937D0860931B0105C080E89AE284
:105B70006AE30E943124DF91CF910895E0913B08C0
:105B8000F0E023E0EE0FFF1F2A95E1F7E05CF74F0E
:105B900090812181813051F0813030F0823051F09C
:105BA000833061F08AE70895892F05C0892F0E940C
:105BB000675B0895822F0E945E5B0895822F0E948A
:105BC000675B08951F93782F80913B08A82FB0E062
:105BD000FD0113E0EE0FFF1F1A95E1F7E05CF74FB0
:105BE00020813181E32F703F58F063E0AA0FBB1F83
:105BF0006A95E1F7A45CB74F13961C92832FE0C01F
:105C0000122FF22FF295FF703C3611F13D3684F4DD
:105C1000383651F1393634F4323651F1353609F02F
:105C20004AC033C03936D1F13A3609F044C014C005
:105C30003337C1F134372CF43E3691F03037D9F593
:105C400035C03937F1F03A3721F13437A1F515C0B5
:105C500088E04CE253E032C08EE04EE252E01CC0DD
:105C60008CE045E657E007C08FEF48EE51E026C0D4
:105C70008EE044EC55E06CE022C08FEF4CEB55E039
:105C80001DC08CE04BEA56E0F6CF88E04CE154E0D2
:105C900015C088E04CE654E060E111C088E04CECAF
:105CA00053E00CC082E04CEF54E008C083E048E7CA
:105CB00056E061E104C088E04CE753E068E07530ED
:105CC00000F5723091F0733028F4772361F0713071
:105CD000C1F407C0733019F0743099F410C08DE529
:105CE0006FC08BE56DC08E2F6BC0F81710F48F2F2F
:105CF00065C0F81711F08BE663C082E761C08DE3E1
:105D00005FC0EA3621F4FF3011F49EE001C0962F07
:105D100083E0989F802D11248B5F781751F51F70B9
:105D2000F11791F053E0AA0FBB1F5A95E1F7FD015F
:105D3000E05CF74F205F3F4F31832083A45CB74F77
:105D40008FEE13968C9313C0E53629F483EB9DE117
:105D500066E00E94C124E0913B08F0E033E0EE0FE2
:105D6000FF1F3A95E1F7E45CF74F8EEF83838AE0FB
:105D700027C0272F30E090E001972817390711F44A
:105D80008DE01EC06F9FF0011124E40FF51F272F37
:105D90002450822F63E00E940BC6E80FF11D982F5C
:105DA000990F980F291B213021F0223031F080E229
:105DB00007C080810E945E5B03C080810E94675B98
:105DC0001F91089590E0FC013197E931F10550F4FD
:105DD000EB5BFD4FEE0FFF1F0590F491E02D099452
:105DE00085E4089586E508958DE4089583E5089592
:105DF00086E7089589E3089586E3089588E708957E
:105E00008BE6089580E7089581E608958DE308956F
:105E10009091660A892F82958F708F3011F482E3FA
:105E20000895892F0E945E5B08958CE208959091F9
:105E3000660A892F8F708F3031F0892F0E94675B3F
:105E4000089580E2089581E308958EE2089584E341
:105E50000895EF92FF921F93CF93DF93282F8091A5
:105E60003B08A82FB0E0FD0183E0EE0FFF1F8A95ED
:105E7000E1F7E05CF74FC081D181FD0113E0EE0F47
:105E8000FF1F1A95E1F7E45CF74F3681333439F49C
:105E9000BE01660F771F6B53744E16EB0EC0CE011A
:105EA000880F991F333729F4BC016858724E12E1EC
:105EB00004C0BC0161597B4E1EEF90E003C06250EC
:105EC00070409F5FFB01E590F490E114F104B9F399
:105ED000283F58F5E20EF11CF7018491882309F060
:105EE00076C0992359F4FB01329685919491892BC0
:105EF00089F4812F90E0C817D90760F443E0AA0F16
:105F0000BB1F4A95E1F7A45CB74F87EF13968C93BC
:105F10008BE55DC033E0AA0FBB1F3A95E1F7A45CA7
:105F2000B74F8AEF13968C931EC0333419F4E9EE01
:105F3000F8E007C0333719F0E3EBF9E002C0E0EA1C
:105F4000F9E02B3FC1F02C3F38F4293F71F02A3F94
:105F500050F4283FD9F50BC02D3FC9F02D3F88F0F4
:105F60002E3FA1F516C08DE332C08DE530C0892FDC
:105F70000E94705B2CC0EC0FFD1F80810E945E5B55
:105F800026C0EC0FFD1F80810E94675B20C08DE062
:105F90001EC0CE010196FD0123E0EE0FFF1F2A95E2
:105FA000E1F7E05CF74F91838083212F30E02817E1
:105FB000390750F083E0AA0FBB1F8A95E1F7A45C74
:105FC000B74F8FEF13968C938AE001C08AE7DF9179
:105FD000CF911F91FF90EF900895482F4F70807FD1
:105FE0006827423009F49DC0433030F4442359F00F
:105FF000413009F0B6C053C0463009F499C047306B
:1060000009F0AFC099C0862F90E08077907034E09F
:10601000959587953A95E1F7E82F67FF2EC0309167
:106020009E01332391F08091910186FF0EC0209153
:106030008E01822F82958F70831720F42858209329
:106040008E0107C0295820938E018091520180FF54
:1060500006C0809155018062809355010895F0E05B
:10606000E851FE4F90818091A201892B8093A2017B
:106070002BB3892F809582230DC0F0E0E851FE4FAD
:1060800090812091A201892F809582238093A20183
:106090008BB3892B8BBB8AB3982B9ABB0895862F21
:1060A00090E08077907024E0959587952A95E1F7A8
:1060B000382F8230E8F467FF0DC02091650081E041
:1060C00090E002C0880F991F3A95E2F7282B2093A1
:1060D000650008952091650081E090E002C0880F7E
:1060E000991F3A95E2F78095822380936500089581
:1060F00067FF0BC028B381E090E002C0880F991FB2
:106100003A95E2F7282B28BB089528B381E090E068
:1061100002C0880F991F3A95E2F78095822388BBC9
:1061200008958091520181FD1CC0E5E6F0E006C0B3
:106130008091520182FD15C0E2E3F0E085B38F70DB
:10614000682B65BB908121E030E002C0220F331F35
:106150004A95E2F7822F8095982390838081822B45
:1061600080830895CF92DF92EF92FF920F931F9357
:10617000CF93DF937C0190936A01809369019091A2
:10618000DA09993C28F489E1989FC001112407C0DD
:10619000985C8DE7989FC001112488579C4E90937E
:1061A0008B0180938A01E091800AEF3F09F493C04C
:1061B00020915801309159018091660A8F70823088
:1061C00051F487E0283F380780F4A3E036952795FF
:1061D000AA95E1F708C083E02C3F380730F43695E4
:1061E000279536952795622F01C06FEF809160014A
:1061F000F09165017091810A50913609F8944091AF
:10620000550147FF1FC08B3F38F490E005962E2FB5
:1062100030E082179307A4F0552341F02F2F30E090
:10622000852F90E001972817390754F0772389F0DC
:10623000262F30E0872F90E00197281739074CF47C
:106240004F7707C0E81728F45F1718F4761708F49B
:10625000406840935501789447FF44C080917F0A7D
:106260008F3D18F021E031E009C0805EE82FF0E0BA
:10627000EE0FFF1FE758FA4F259134914427F39E04
:10628000D001E29EC001F29E900DA11DB41FE39EBD
:10629000900DA11DB41F11246BE0B695A79597959D
:1062A00087956A95D1F79C018091470A90E0880F05
:1062B000991F880F991F280F391F82E02130380756
:1062C00018F4EE24FF240EC0E12C4EEFF42EE20E63
:1062D000F31EA70109C0F894809155018F77809330
:1062E0005501789440E050E00091D209602F70E0B1
:1062F0006770707018E01150C12FD0E0C617D70733
:1063000009F4A7014115510519F420E030E021C03E
:10631000FE01E851FE4F80A190E080589E4F6C0135
:1063200022275D9DD0014C9DC0015C9D900DA11D5B
:10633000B21F4D9D900DA11DB21F112429E0B695ED
:10634000A795979587952A95D1F79C0180A5280F49
:10635000311DF894CC0FDD1FCC0FDD1FC754D74F74
:10636000398328837894112309F0C5CF902F977033
:10637000E92FF0E0E851FE4F208107C09150E92F4E
:10638000F0E0E851FE4F8081282B9923B9F7209344
:106390009001DF91CF911F910F91FF90EF90DF90CF
:1063A000CF90089580E091E09093A2088093A10897
:1063B00024E62093A3089093A5088093A40880E87E
:1063C0008093A60810923408109233088DE791E06C
:1063D0009093A8088093A70888E38093AB08109255
:1063E000AD081092AC082093AE081092AF0810923E
:1063F000B0081092B1081092B60880E090E00E94B8
:10640000B2308091980B9091990BA0919A0BB0911A
:106410009B0BBF6F8093980B9093990BA0939A0B53
:10642000B0939B0B08959091710980917209282F68
:10643000392FC90108952091580130915901809157
:10644000660A8F70823051F487E0283F380778F46D
:1064500043E0369527954A95E1F70AC083E02C3F43
:10646000380728F4369527953695279501C02FEFE4
:106470008091AA0A281720F48091AF0884609BC0FD
:1064800030E090E002968217930734F48091AF08D1
:106490008B7F8093AF0804C08091AF0882FDD1C08C
:1064A000309165019091ED092091EE098091A60B44
:1064B000882319F4892F422F0CC09D3F10F08FEFD5
:1064C00002C0892F8E5F2D3F10F04FEF02C0422F88
:1064D0004E5F381720F08091AF08816005C04317E8
:1064E00028F08091AF088E7F8093AF08692F70E00D
:1064F000621B7109CB018E7F90700A9709F067C00B
:10650000209167013091680136952795369527953A
:1065100089E1489FC0011124281B390B37FD3AC07F
:10652000B4E036952795BA95E1F7522F9091600126
:106530008091540186FF03C08091210902C080919F
:10654000000A8917A0F4981B892F60FF09C0909159
:106550006E01282F26952917E8F4592F521B18C0D1
:106560009531C0F4880F8517A8F4581B11C04091CD
:106570000A0A252F30E0842F90E08F7090708217E8
:10658000930734F042954F70541710F050936E01FA
:10659000552361F4809191018F7B809391018091CB
:1065A000AF088D7F8093AF0820E00EC0503130F0EF
:1065B0008091AF0882608093AF0833C080919101D1
:1065C000806480939101252F20939E0138C0909183
:1065D00060018091540186FF03C08091210902C0AF
:1065E0008091000A282F30E0892F90E02817390782
:1065F0008CF410929E01809191018F7B8093910188
:106600008091BF0B81FD1DC08091AF088D7F80936D
:10661000AF0815C09091AF0890FF05C092609093AD
:10662000AF0881E0089510929E01809191018F7BC7
:106630008093910191FF03C09D7F9093AF0880E00C
:10664000089581E00895CF93DF93AC01762F662300
:1066500011F420E054C0809157012091D8098D3366
:1066600010F46FEF10C090E0CC9730E0FC01E29F97
:10667000C001E39F900DF29F900D1124892F990F77
:10668000990B682F6095679FC0011124692F7727A8
:1066900067FD7A95262FC62FD0E08AE290E0FC01B4
:1066A000CE9FC001CF9F900DDE9F900D1124F4E08E
:1066B00095958795FA95E1F74817590700F5CA01AE
:1066C000880F991F840F951F73E0880F991F7A9583
:1066D000E1F770E00E9417C6E62FF0E0E05FF14EB0
:1066E000E4918E2F90E09C012C9FC0012D9F900D76
:1066F0003C9F900D1124892F990F990B282F822FE1
:10670000DF91CF910895F8948091530182608B7F3F
:106710008093530180915401806180935401789457
:1067200008958091BF09282F30E043E0220F331FE6
:106730004A95E1F780915C0190915D012817390736
:10674000C0F480915C0190915D01821B930B60917C
:10675000C2090E94921D272F382F492F5527832FBA
:1067600090E0892B11F06FEF01C0622F6093B408A5
:1067700008951092B4080895DF92EF92FF920F935C
:106780001F93CF93DF93D09064018FE08D1550F469
:10679000F8948AE090E09093680180936701789480
:1067A00081E088C0C0916201D0916301C439D105F4
:1067B000B8F4CD2B61F08FEF80936501F8948CE9EC
:1067C00093E69093680180936701789478C0109263
:1067D0006501F894109268011092670178946FC077
:1067E0008091F10982958F708F5FE82FF0E0EE0FB6
:1067F000FF1FE758FA4F859194916FE20E94921D16
:10680000672F782F892F992724EC39E04427739F2D
:106810008001629F7001729FF00C011D141F639F25
:10682000F00C011D141F1124DD20E1F0F89480917B
:1068300064012091620130916301789490E0A0E0BE
:10684000B0E0DC019927882740E050E0820F931FD9
:10685000A41FB51F74E0B695A795979587957A956F
:10686000D1F7EC019E0140E050E0C801B7010E9461
:106870002BC6C901DD2029F064E0969587956A95BD
:10688000E1F7F8949093680180936701789469E246
:106890000E94921D72958295929560EF982796239B
:1068A00098278727862387279C01832F9927892B61
:1068B00021F08FEF8093650102C020936501DF9185
:1068C000CF911F910F91FF90EF90DF900895E0918D
:1068D000F709E7FD2CC08091330890913408892B8B
:1068E00009F07FC080915801909159019C01220FBD
:1068F000331F3093340820933308969587959695E7
:106900008795482F873608F041C050E02E2F30E0A1
:106910002F703070220F331F220F331F84E690E058
:10692000821B930B481759070CF05BC02FC0F0E097
:10693000E077F070A3E0F695E795AA95E1F7EE5AB7
:10694000F24F808191816091610A0E94921DF9E06D
:106950009695879577956795FA95D1F78091620A14
:10696000680F711D6138710518F460E070E006C0B1
:106970006058704083E06D3F780740F4CB019695F6
:10698000879596958795482F873618F080E293E093
:1069900018C08091F70990E08F709070880F991F50
:1069A000880F991F24E630E0281B390B842F90E0D4
:1069B0008217930784F4C90143E0880F991F4A9511
:1069C000E1F79093340880933308809154018260FA
:1069D0008093540106C0660F771F7093340860934C
:1069E00033088091F30983FD02C080E80FC08091D5
:1069F0003308909134089695879568E70E94921D18
:106A0000672F782F892F99278CE3861B8093A60800
:106A1000089580915701873710F080E008958D33F5
:106A200010F48CEF0895E82FF0E0EE0FFF1FE75809
:106A3000FA4F8591949167E70E94921D672F782FF6
:106A4000892F9927862F08951F93182F0E940935A3
:106A5000189FC0011124892F9927810F911D90FD46
:106A60008FEF1F9108957F928F929F92AF92BF9266
:106A7000CF92DF92EF92FF920F931F93CF93DF930A
:106A8000EC0170901E01072D10E0F801EE0FFF1FC2
:106A9000E05EFE4F40815181D183C0838091BA096D
:106AA00090E0880F991F9E0120503048241B350B21
:106AB0004427399F5001289F4001389F900CA11C0A
:106AC000B41E299F900CA11CB41E112460E80E94E2
:106AD000921D6B017C018091D20990E087709070CB
:106AE0000817190714F000E002C0072D0F5F00938C
:106AF0001E018091540184FF03C010921F0140C009
:106B000080911F01882389F155274B2D3A2D292D7E
:106B10002C193D094E095F09F901C9018C0F9D1F10
:106B200018161906ECF41216130664F110915E0A99
:106B3000C90180509048612F0E94921D672F782FC5
:106B4000892F9927212F30E03695322F222737952C
:106B50002795EE27FF27E21BF30BE60FF71F12C066
:106B6000EE27FF27EC1BFD0B0DC0E0E2F1E0C19327
:106B7000D19381E0E033F807D1F781E080931F01E2
:106B8000E0E0F0E0CF01DF91CF911F910F91FF90F6
:106B9000EF90DF90CF90BF90AF909F908F907F90BD
:106BA0000895EF92FF920F931F93E090A901F09048
:106BB000AA010091AB011091AC0187EC9BE16091BF
:106BC00053070E94921D672F782F892F99276E0DEA
:106BD0007F1D801F911F6093A9017093AA0180936C
:106BE000AB019093AC012091A9013091AA01409191
:106BF000AB015091AC016091AD017091AE018091FB
:106C0000AF019091B0019A014427552740E050E030
:106C10000E942BC6DA01C901892F9A2FAB2FBB27FF
:106C200064E60E94921D672F782F892F9927709311
:106C3000A8016093A7011F910F91FF90EF90089515
:106C4000CF92DF92EF92FF920F93CF93DF938091D9
:106C5000520180FDA1C04091B309442309F49CC0B6
:106C600080916001833B08F097C0493C28F489E19A
:106C7000489FE001112407C0485C8DE7489FE00170
:106C80001124C857DC4ECE016091B4090E94921DB8
:106C900000915A01C72ED82EE92EFF248CE36EEA0C
:106CA000AE0196010E94DE1DEC018091D9090E947F
:106CB000243581BF209709F46FC0CE010E94B23005
:106CC0008091920B9091930B2CB53DB53093930B23
:106CD0002093920B2817390748F48091940B9091D8
:106CE000950B01969093950B8093940BE091B908C6
:106CF000F091BA08309709F44DC04CB55DB550938A
:106D0000930B4093920B4217530748F48091940BD6
:106D10009091950B01969093950B8093940B809195
:106D2000A20180959091E8018923C9F080915201D8
:106D300080FF06C0809155018062809355010FC08D
:106D4000209190018091A201822B8093A2019BB39C
:106D5000822F809589238BBB8AB3822B8ABBBA0191
:106D60006E0F7F1F7093BC086093BB0820918A014F
:106D700030918B01C90143968E179F0710F04BE2AB
:106D800004C0B901640F751F4BE181E39BE050E043
:106D90000E94BE610E946364DF91CF910F91FF90CA
:106DA000EF90DF90CF900895FF920F931F93E091A3
:106DB000DB09E295EF70EF3019F4819928C025C006
:106DC000E83010F480E00CC0EC3009F1EF3019F03D
:106DD000E83021F41AC080991AC017C0E77081E02A
:106DE000F0E0EE0FFF1FEE5AF24FE181E43010F4B5
:106DF00090E005C0E83010F490E401C090E88823EA
:106E000039F080E8891B982F03C090E001C090E81A
:106E1000F89480915401992311F4806403C0903850
:106E200009F48F7B809354017894F0906001482F8F
:106E3000407486FD03C0109272010BC08091340A29
:106E40008F1538F48091830A882309F48FEF80939B
:106E500072019091650120915C0130915D014423A4
:106E600009F18091530181FD1DC04091820A941760
:106E700020F48091390A9817A8F08091830A88231A
:106E800021F080917201882369F08091840A88231F
:106E9000C9F090E0B3E0880F991FBA95E1F7821727
:106EA000930780F48091540185FF51C0F89480913C
:106EB00054018F7D8093540178941092B008109201
:106EC000B60845C010916501141710F420E017C0F2
:106ED0004091F6094F718091E7096091120A20E014
:106EE0000F2D0E949D1D282F6091670A161738F4F8
:106EF0008091820A40E0012F0E949D1D282F20933F
:106F0000B6088091680A6091690A40912F0A20E0D2
:106F10000F2D0E949D1D8093B0088091540185FD26
:106F20000EC0F8948091540180628093540178944B
:106F30008091830A882309F48FEF809372018091F6
:106F4000820A80FD06C08091690A8F1510F460E006
:106F500001C060E8F89480919A0A0E94ED2F78941D
:106F60001F910F91FF9008950F939C0180916701ED
:106F7000909168019695879596958795281739077A
:106F800010F080E011C0FC01E21BF30BCF01807018
:106F9000892B11F080E108C080E06091200A40E078
:106FA00020E10E2F0E949D1D0F9108950F93809157
:106FB000D3092091D409482F50E0420F511D4F3F73
:106FC000510511F008F04FEF281710F020E002C033
:106FD000821B282F009157018CE362EA0E949D1DBD
:106FE0000F9108950F931F9300911708109118089F
:106FF00053E0169507955A95E1F78091F80960914D
:10700000F90940E02FEF0E94CE1D8093600120918E
:1070100013083091140843E0369527954A95E1F717
:107020008091F409829FC0011124909357018091AF
:107030005A0D90915B0D2FEF8F3F920729F410921C
:107040005D0110925C010CC06091990A0E94921D32
:10705000672F782F892F992770935D0160935C01CA
:107060008091580D9091590D2FEF8F3F920729F481
:1070700010925F0110925E010CC06091990A0E940B
:10708000921D672F782F892F992770935F01609346
:107090005E011F910F9108958091FD0882958F7078
:1070A00090911008981730F00E940A21882311F05F
:1070B000109210086091D509662319F480E991E0D7
:1070C0002FC080911D0890911E080E94921D209152
:1070D000660A22952F70243011F427E005C0213074
:1070E00011F028E001C029E004C0969587957795B6
:1070F00067952A95D2F72091D609422F213808F0BA
:1071000040E830E0240F311D260F371F81E0213089
:10711000380718F480E090E003C0C9018050914026
:10712000909359018093580108959F92AF92BF9216
:10713000CF92DF92EF92FF920F931F93CF93DF9343
:10714000F8948091DE0980FF1DC020915801309194
:1071500059018091660A8F70823051F447E0283FD0
:10716000340798F413E0369527951A95E1F708C08F
:1071700053E02C3F350748F43695279536952795EB
:10718000122F04C01091600101C01FEF78949090FD
:107190003001A92CBB24F501EE0FFF1FE05DFE4F6F
:1071A0006091E8096C776068818592850E94921DE4
:1071B000672F782F892F9927EB01F501E05DFE4FAE
:1071C0004181141708F48AC0812F841B482F8093B3
:1071D0006F018091DF09481708F49AC08FED99E09C
:1071E00064E022E639E00E94701EC82E40916501DD
:1071F0008EE599E064E023EE39E00E94701EE82EEF
:1072000000915A014091E90950E0405C5F4F8CE3E6
:107210006EEA20E430E00E94DE1DEC9C7001112437
:10722000A7012227599F7001489F6001589FD00CE9
:10723000E11CF21E499FD00CE11CF21E1124CD2C42
:10724000DE2CEF2CFF2400915A014091EA098CE3D7
:107250006EEA50E020E030E00E94DE1D76E0880F0C
:10726000991F7A95E1F7C80ED91EC60160914A09A7
:107270000E94921D9B01AC0132954295529520EFE0
:10728000542752235427432742234327CA0180937C
:107290006D018091D00929E1829FC0011124AC01C8
:1072A0002227D59ED001C49EC001D49E900DA11D61
:1072B000B21FC59E900DA11DB21F11249295A295DB
:1072C000B29580EFBA27B823BA27A927A823A92700
:1072D0009D01C217D307E0F4E9011AC0842F90E0A2
:1072E000811B91090E9794F4909160018091540153
:1072F00086FF03C08091210902C08091000A282FD7
:1073000030E0892F90E02817390714F0C0E0D0E072
:10731000F501EE0FFF1FE05DFE4FD287C187F5013B
:10732000E05DFE4F11838091D20990E087709070EC
:10733000A816B90614F080E002C0892D8F5F8093F3
:107340003001D093AD08C093AC08CD2B69F4F8940C
:10735000809153018F7C80935301789484E68093CD
:10736000AE0810926D010CC0F894809153018061B9
:1073700080935301809153018F7D809353017894C2
:1073800010936101DF91CF911F910F91FF90EF90CA
:10739000DF90CF90BF90AF909F900895EF92FF92B3
:1073A0000F931F93E090B709F0906501EF1480F4FC
:1073B0008091A60B882319F023E539E00BC0F894DF
:1073C000809153018B7F80935301789410E030C0FB
:1073D0002FE439E000915A018BE499E064E0402FFA
:1073E0000E94701E182FEF1418F58CE36EEA40917E
:1073F000B5092091B6090E949D1D893010F460E006
:1074000002C0682F6850212F30E00091A60BF901CF
:10741000F695E795601728F080E040E050E09F0186
:1074200004C0061B80E067E0AF010E94DE1D182F3C
:10743000812F1F910F91FF90EF900895EF92FF928F
:107440000F931F93CF93DF930E94CE39C82FD0E0C4
:10745000E4E0CC0FDD1FEA95E1F7C050DF4F9091DB
:107460005A0180919E09981728F0D093A508C093DF
:10747000A40852C0E091B708F0E0A091B808B0E0CD
:1074800000915A019F012D54364F73EBE72E79E09E
:10749000F72EEA0EFB1EEB56F64F8081AB56B64F29
:1074A0006C91F9014289F70122890E949D1D482FA4
:1074B0002091CF09829F90011124232F330F330B8A
:1074C0000091650180910E0360911D030E949D1D36
:1074D000482F2091B809829F90011124232F330F48
:1074E000330B009158011091590133E0169507951F
:1074F0003A95E1F78FE062E30E949D1D682FCE016F
:107500000E94921D672F782F892F99276C0F7D1F5E
:107510007093A5086093A408DF91CF911F910F91FC
:10752000FF90EF900895EF92FF920F931F93CF93E8
:10753000DF937B018F71883029F4C0915801D0917D
:10754000590147C0803119F48091530704C081313B
:1075500051F480911802C82FD0E004E0CC0FDD1F59
:107560000A95E1F736C0E82FF0E0E770F070EE0F13
:10757000FF1FEE5AF24FC081D181893050F1009146
:10758000580110915901C80164E60E94921D672FAD
:10759000782F892F9927060F171FCE016EE00E94C2
:1075A000921DFE01E457FF4F672F782F892F9927EF
:1075B000E60FF71F0E171F0718F0C0E0D0E009C054
:1075C000EF01C01BD10B80E1C030D80710F0CFEF26
:1075D000DFE0CE01B7010E949520DF91CF911F918E
:1075E0000F91FF90EF9008950F931F938091520198
:1075F00081FD15C10091B10A2091DB098091AE0A8D
:10760000822790E08F709070892B09F460C0E22F80
:10761000EF70E83010F480E00DC0EC3059F1EF303D
:1076200019F0E83021F41DC0809924C01AC0E22F5F
:10763000E77081E0F0E0EE0FFF1FEE5AF24FE181BC
:10764000E43010F450E005C0E83010F450E401C01C
:1076500050E8882319F080E8851B582F552341F402
:1076600001C050E080918C01816080938C0108C042
:10767000503831F480918C018E7F80938C0150E8DA
:107680008091650190E020910D0A30E02A50304051
:107690004091110A241B3109281739079CF45523FE
:1076A00031F480918C01826080938C0106C08091BE
:1076B0008C0181FF0CC0503829F00E940049809352
:1076C000A10105C080918C018D7F80938C018091F8
:1076D0008C0181FD37C0F8948091F20860E00E942F
:1076E000ED2F78941092B10889E1089FA001112430
:1076F0008091FE0987FF6FC080917201882309F095
:107700006AC0909160018091540186FF03C080910E
:10771000210902C08091000A282F30E0892F90E0D3
:10772000281739070CF457C09091BE0A85E0989F3E
:10773000C0011124969587958417950708F04BC0D2
:10774000AC0149C0F8948091F20860E80E94ED2FE6
:1077500078948091120985FF03C04091180202C0FD
:10776000409153074A3E20F480910B05841728F47A
:1077700080918C018D7F80938C01809104058823FA
:1077800021F4423008F051C003C0841708F44DC002
:1077900010910D0A80914909807F803819F080E0AE
:1077A00090E007C08091460968E776E00E94933A2E
:1077B00090E080938D019C01210F311D832F99272B
:1077C000892B19F4201708F4022F89E1089FA001E2
:1077D000112400939F01CA010E94B4379091B6080A
:1077E000582F891708F4592F809191018C70A9F0B6
:1077F00080916701909168012091C10948E2249F1E
:10780000900111248217930740F08091BD098F7079
:107810008F5F581710F4582F03C0513108F050E112
:1078200050938F011F910F91089584E095E068E0D7
:107830002CEF34E00E94701E182FACCF1F93CF9313
:10784000DF93109165016091BB0B662339F070E006
:1078500014E0660F771F1A95E1F717C28091910126
:1078600087FD11C28091540185FF03C08091860A73
:1078700002C08091EF09282F30E0412F50E02417FB
:10788000350708F400C28091AE0A86FF09C0225075
:1078900030402417350720F480919101886003C09F
:1078A00080919101877F809391019091AB0A209103
:1078B0005801309159018091660A8F70823051F4DD
:1078C00047E0283F340780F4B3E036952795BA9512
:1078D000E1F708C053E02C3F350730F43695279583
:1078E00036952795822F01C08FEF981708F4CBC1EA
:1078F0008091540185FD05C00E941B32882309F048
:10790000C2C14091A4085091A5088091AE0829E118
:10791000829FC0011124EA012227D99FB001C89F8C
:10792000A001D89F500D611D721FC99F500D611D90
:10793000721F11242091A30830E0205F3E4F8091F8
:10794000A60890E0805F9E4FEC01EE273D9FD0019E
:107950002C9FC0013C9F900DA11DBE1F2D9F900D1F
:10796000A11DBE1F1124892F9A2FAB2FBB27452F96
:10797000562F672F7727FC012227F59FD001E49F20
:10798000C001F49F900DA11DB21FE59F900DA11D98
:10799000B21F11249295A295B29580EFBA27B82311
:1079A000BA27A927A823A9279D018091B709811784
:1079B00028F080916001833B08F065C180915401FB
:1079C00084FF21C08091D20984FF1DC08091B90934
:1079D000E82FF0E0EE0FFF1FE758FA4F85919491E2
:1079E000BC014427379FD001269FC001369F900DD0
:1079F000A11DB41F279F900DA11DB41F1124CD01FF
:107A0000AA27BB279C018091A1089091A208EC01B4
:107A100044273D9FD0012C9FC0013C9F900DA11D8C
:107A2000B41F2D9F900DA11DB41F1124892F9A2FD3
:107A3000AB2FBB279C018091B108882399F090E07F
:107A400080509F4FFC0144273F9FD0012E9FC001D3
:107A50003E9F900DA11DB41F2F9F900DA11DB41F1F
:107A6000112414C08091B00890E080509F4FBC0159
:107A70004427379FD001269FC001369F900DA11D3E
:107A8000B41F279F900DA11DB41F1124892F9A2F79
:107A9000AB2FBB27BC018091F10880FF19C08091FA
:107AA000B50890E080589F4FEC0122277D9FD001C0
:107AB0006C9FC0017C9F900DA11DB21F6D9F900D0A
:107AC000A11DB21F1124892F9A2FAB2FBB27BC01F8
:107AD0007093A8086093A7088091A9089091AA08BC
:107AE000EE27799FA001689F9001789F300D411D7E
:107AF0005E1F699F300D411D5E1F112486E0569563
:107B00004795379527958A95D1F78091AB0890E0F6
:107B100088539F4FFC0166273F9FD0012E9FC001D5
:107B20003E9F900DA11DB61F2F9F900DA11DB61F4A
:107B30001124892F9A2FAB2FBB27EC018091490983
:107B4000807FE9F48091460968E776E00E94933AE5
:107B500090E088539F4FAC012227D59FD001C49F4E
:107B6000C001D49F900DA11DB21FC59F900DA11DF6
:107B7000B21F1124892F9A2FAB2FBB27EC018091C4
:107B80001B09807FE9F48091070969E876E00E948B
:107B9000933A90E088539F4FBC012227D79FD00192
:107BA000C69FC001D69F900DA11DB21FC79F900D0B
:107BB000A11DB21F1124892F9A2FAB2FBB27EC01D7
:107BC0008091F30982FD08C080915801909159017C
:107BD000BE010E94261F3BC080910B04882311F434
:107BE0006CEA2DC020915801309159018091F20921
:107BF00082FF0AC08091330890913408969587954A
:107C00002817390708F49C0144273D9FD0012C9F79
:107C1000C0013C9F900DA11DB41F2D9F900DA11D73
:107C2000B41F1124892F9A2FAB2FBB27EC010E9480
:107C3000684A853F10F06FEF02C0682F665FCE0183
:107C40000E94921D672F782F892F9927CB01609171
:107C5000D0090E94921D44E0969587957795679587
:107C60004A95D1F78091540184FF06C09091650137
:107C70008091B709891748F48091AC089091AD08BC
:107C8000680F791F02C060E070E0CB01DF91CF91F7
:107C90001F910895CF92DF92EF92FF920F931F935F
:107CA000DF93CF9300D0CDB7DEB70E941E3C8C018E
:107CB0000E9433357C01E00EF11E90917109809194
:107CC0007209092F182F812F902FAC012227F59EC2
:107CD000D001E49EC001F49E900DA11DB21FE59E4F
:107CE000900DA11DB21F11244091AD015091AE0124
:107CF0006091AF017091B001892F9A2FAB2FBB27F4
:107D00002EE43BE18C01EE27319FD001209FC00182
:107D1000309F900DA11DBE1F219F900DA11DBE1F64
:107D200011248C019D0112952295329500EF322786
:107D300030233227212720232127C901A0E0B0E0EA
:107D4000840F951FA61FB71F8093AD019093AE01BE
:107D5000A093AF01B093B001E114F10409F43CC069
:107D60008091F10981FD0CC0C7016091D7090E9483
:107D70002333182F0E94D63790E0810F911D26C023
:107D8000409157018BE09EE165E09E012F5F3F4FE0
:107D90000E94A31EA981B0E0FD01E55FF14E849130
:107DA000EA81CE2EDD249601255F314EF9016491E2
:107DB00000915701A25CB64F2EE339E0C20ED31EEC
:107DC0004C91F60120810E949D1D90E0880F991F23
:107DD000880F991FE80EF91EC7010E94B2308091EA
:107DE000D9090E94243581BF0F900F90CF91DF9168
:107DF0001F910F91FF90EF90DF90CF9008950F9318
:107E00008091530181FF1EC0F894809153018D7FB2
:107E1000846080935301789400915A018CE36EEA58
:107E20004091B5092091B6090E949D1D8093A60B33
:107E300087E18093A70B8091630A83FF03C081E0F1
:107E40000E9462610F91089540915B012091600151
:107E5000809164048F3F39F08CE194E0642F422FCD
:107E60000E94CD4B08958CE594E068E02CE134E06D
:107E70000E94701E08958091F30987FF10C08091C1
:107E80001B0890911C0863E0969587956A95E1F729
:107E900064E879E00E94832080935B0131C04091C7
:107EA0001B0850911C08CA0153E0969587955A9576
:107EB000E1F7282F30E0F901E050FE4F94918F3F19
:107EC00051F02F5F3D4FF90164914770440F892FA6
:107ED0000E94C01F982FE0E0F2E0E491EF3F29F00C
:107EE000EFEFF2E0E491EF3F49F48EE8989FC00194
:107EF0001124892F990F990B982F945C90935B0113
:107F00000E94243F8093A30808958091F30986FF7F
:107F10000FC08091190890911A08B3E09695879543
:107F2000BA95E1F763E779E00E948320482F1FC0EC
:107F3000E0911908F0911A08A3E0F695E795AA9543
:107F4000E1F7E050FD4F4491E0E0F3E0E491EF3FD2
:107F500029F0EFEFF3E0E491EF3F49F48EE8489F1A
:107F6000C0011124892F990F990B482F445C40932D
:107F70005A0185E999E06AE027EB38E00E944F1E3C
:107F80000895482F4F70807F6827423009F49DC0C4
:107F9000433030F4442359F0413009F0B6C053C0A7
:107FA000463009F499C0473009F0AFC099C0862F18
:107FB00090E08077907034E0959587953A95E1F759
:107FC000E82F67FF2EC030919E01332391F08091FE
:107FD000910186FF0EC020918E01822F82958F70B5
:107FE000831720F4285820938E0107C02958209326
:107FF0008E018091520180FF06C080915501806200
:10800000809355010895F0E0E851FE4F90818091F2
:10801000A201892B8093A2012BB3892F8095822303
:108020000DC0F0E0E851FE4F90812091A201892F10
:10803000809582238093A2018BB3892B8BBB8AB35B
:10804000982B9ABB0895862F90E08077907024E05B
:10805000959587952A95E1F7382F8230E8F467FFE8
:108060000DC02091650081E090E002C0880F991F4B
:108070003A95E2F7282B209365000895209165003A
:1080800081E090E002C0880F991F3A95E2F7809551
:10809000822380936500089567FF0BC028B381E0B9
:1080A00090E002C0880F991F3A95E2F7282B28BB71
:1080B000089528B381E090E002C0880F991F3A9597
:1080C000E2F78095822388BB08958091520181FD5B
:1080D0001CC0E5E6F0E006C08091520182FD15C0AB
:1080E000E2E3F0E085B38F70682B65BB908121E0FF
:1080F00030E002C0220F331F4A95E2F7822F8095AD
:10810000982390838081822B80830895F8948091B6
:108110007E0A60E80E94C13F78940895F8948091A7
:108120007E0A60E00E94C13F7894089583B7896712
:1081300083BF08950895EF92FF920F931F93CF93FB
:10814000DF93582FF62EE42EA82FB0E0AA0FBB1F06
:10815000AA0FBB1FA754B74F0D911C911197011582
:10816000110509F495C08091920B9091930BCCB5B9
:10817000DDB5D093930BC093920BC817D90748F481
:108180008091940B9091950B01969093950B809311
:10819000940BE52FF0E080E2F81621F58091A20122
:1081A000E851FE4F80959081892349F080915201DA
:1081B00080FF08C0809155018062809355014BE09B
:1081C00081E049C0209190018091A201822B80938F
:1081D000A2019BB3822F809589238BBB8AB3822B0C
:1081E0008ABBEDCFE851FE4F20818091A20180959E
:1081F000822371F130919E01332391F0809191019E
:1082000086FF0EC090918E01892F82958F70831703
:1082100020F4985890938E0107C0995890938E013E
:108220008091520180FF06C0809155018062809349
:1082300055010DC08091A201822B8093A2019BB3B6
:10824000822F809589238BBB8AB3282B2ABB81E0A0
:10825000452F4295407F9E01200F311F13963C937E
:108260002E93129760918A0170918B01882349F0B7
:10827000CB0143968017910720F46C0F7D1F4E0DA4
:1082800002C04F0DB90181E39BE050E00E94BE6146
:10829000DF91CF911F910F91FF90EF9008951F9361
:1082A00080916C0A84FF04C08091550183FF3BC01C
:1082B0009091D109913049F08091A40B8150809325
:1082C000A40B882381F59093A40B8091530181FF27
:1082D00008C08091D20984FF04C080E060E240E1E0
:1082E0001EC01091A3010E943C7A8091550187FF26
:1082F00018C08091D209282F30E0277030702630C6
:1083000031057CF4243031052CF0112311F01330A9
:1083100041F4117087708F5F810F6AE049E00E941D
:108320009B400E9463641F91089580E091E09093C8
:10833000A2088093A1081092530180915401846196
:10834000809354018FEF8093A80B1092A301809328
:10835000640110926501109268011092670180918A
:10836000790A90E080509F4F90937401809373013D
:108370000E94CCB0F8940E948E4078940000F8944B
:108380008091E7018F738093E701789480E090E01B
:108390000E94B2300E9438510E941E3C90936A01A4
:1083A0008093690108959C01E199FECF3FBB2EBBEC
:1083B000E09A8DB308951092D60108959091D60158
:1083C00092FF02C080E00895823008F080E09F7044
:1083D00096608295807F982B9093D60181E00895D6
:1083E0004091CE015091CF01E091D001F091D101A7
:1083F000A091D201B091D30111972091D401309175
:10840000D501E199FECFCA01820F931F9FBB8EBB9E
:10841000E09A7DB3E20FF31F60812F5F3F4FCA01E7
:10842000820F931F215030400BC02F5F3F4FE199C7
:10843000FECF9FBB8EBBE09A7DB3618101963196E2
:10844000761721F42A173B0780F315C0E199FECF78
:10845000420F531F5FBB4EBB6DBB0FB6F894E29A41
:10846000E19A0FBE8091D60181608093D601E39A94
:108470002A173B0730F03093D5012093D40181E0D7
:1084800008952F5F3F4F3093D5012093D40180E0B2
:1084900008958091CD01833009F497C0843038F479
:1084A000813009F441C0823008F072C00EC08530BE
:1084B00009F4F3C0853008F4BCC0863009F421C14A
:1084C000883009F451C181E008959091D601892F37
:1084D000807F91F092959F70892F90E0019723E023
:1084E00037E0AC01429FC001439F900D529F900D19
:1084F00011248058974F02C080E091E09093CF0103
:108500008093CE0183EB99E09093D1018093D001C9
:108510008FEF90E09093D3018093D2011092D50118
:108520001092D40181E025C10E94F041882309F412
:1085300024C19091D601892F807F91F092959F70F0
:10854000892F90E0019723E037E0AC01429FC00102
:10855000439F900D529F900D11248158964F02C059
:108560008FEF91E09093CF018093CE0189EE98E058
:108570009093D1018093D00187EB90E09093D30149
:108580008093D2011092D5011092D40182E0F1C003
:108590000E94F041882309F4F0C080E090E09093BD
:1085A000CF018093CE0180EA99E09093D10180932E
:1085B000D00183E190E09093D3018093D201109297
:1085C000D5011092D40183E0D4C00E94F0418823E9
:1085D00009F4D3C09091D601892F807F91F09295B4
:1085E0009F70892F90E0019723E037E0AC01429F14
:1085F000C001439F900D529F900D11248A5C954FAE
:1086000002C086EB92E09093CF018093CE018EE280
:1086100092E09093D1018093D0018EED92E09093FF
:10862000D3018093D2011092D5011092D40184E03D
:10863000A0C00E94F041882309F49FC09091D60108
:10864000892F807F91F092959F70892F90E00197FC
:1086500023E037E0AC01429FC001439F900D529F41
:10866000900D11248C5E924F02C084E995E09093A6
:10867000CF018093CE0185E697E09093D10180935E
:10868000D00188EA90E09093D3018093D2011092B8
:10869000D5011092D40185E06CC00E94F04188237E
:1086A00009F46BC09091D601892F807F91F092954B
:1086B0009F70892F90E0019723E037E0AC01429F43
:1086C000C001439F900D529F900D11248D5A904FE1
:1086D00002C083ED97E09093CF018093CE0188EEA6
:1086E00091E09093D1018093D00180E390E090934A
:1086F000D3018093D2011092D5011092D40186E06B
:1087000038C00E94F0418823C1F19091D601892F91
:10871000807F91F092959F70892F90E0019723E0E0
:1087200037E0AC01429FC001439F900D529F900DD6
:1087300011248454924F02C08CE396E09093CF01B1
:108740008093CE018CEB95E09093D1018093D00182
:1087500087E991E09093D3018093D2011092D501E3
:108760001092D40188E005C00E94F041882329F0CE
:108770008DE08093CD0180E0089580E00895909190
:10878000D60192FF13C091FF06C09D7F9093D60142
:108790001092CD01089590FD09C00E94494288239E
:1087A00029F08091D6018B7F8093D60108951F9286
:1087B0000F920FB60F9211248F938091D6018E7F66
:1087C0008093D601E3988F910F900FBE0F901F906A
:1087D00018950E946E4D80918C012091D60122FD4A
:1087E0000CC02F70266090E0880F991F880F991F8A
:1087F00080719070282B2093D60108951F93182F15
:1088000080EA99E060E070E043E150E023ED31E47C
:108810000E94D0C5113009F040C083EB99E060E8B8
:1088200078E04FEF50E023ED31E40E94D0C589EEAF
:1088300098E06FE779E047EB50E023ED31E40E94E8
:10884000D0C588EE91E063E57FE040E350E023EDA2
:1088500031E40E94D0C58EE292E066E37AE04EED0C
:1088600052E023ED31E40E94D0C585E697E064E153
:108870007DE048EA50E023ED31E40E94D0C58CEB66
:1088800095E06CEB7DE047E951E023ED31E40E9497
:10889000D0C580918C0184603FC083EB99E060E09B
:1088A00071E04FEF50E023ED31E40E94D0C589EE36
:1088B00098E06FEF71E047EB50E023ED31E40E9468
:1088C000D0C588EE91E063ED77E040E350E023ED22
:1088D00031E40E94D0C58EE292E066EB72E04EED8C
:1088E00052E023ED31E40E94D0C585E697E064E9CB
:1088F00075E048EA50E023ED31E40E94D0C58CEBEE
:1089000095E06CE376E047E951E023ED31E40E9425
:10891000D0C580918C018B7F80938C0180917B0AE4
:10892000877080937B0A1F910895482F4F70807F36
:108930006827423009F49DC0433030F4442359F095
:10894000413009F0B6C053C0463009F499C04730F1
:1089500009F0AFC099C0862F90E08077907034E026
:10896000959587953A95E1F7E82F67FF2EC03091EE
:108970009E01332391F08091910186FF0EC02091DA
:108980008E01822F82958F70831720F428582093B0
:108990008E0107C0295820938E018091520180FFDB
:1089A00006C0809155018062809355010895F0E0E2
:1089B000E851FE4F90818091A201892B8093A20102
:1089C0002BB3892F809582230DC0F0E0E851FE4F34
:1089D00090812091A201892F809582238093A2010A
:1089E0008BB3892B8BBB8AB3982B9ABB0895862FA8
:1089F00090E08077907024E0959587952A95E1F72F
:108A0000382F8230E8F467FF0DC02091650081E0C7
:108A100090E002C0880F991F3A95E2F7282B209327
:108A2000650008952091650081E090E002C0880F04
:108A3000991F3A95E2F78095822380936500089507
:108A400067FF0BC028B381E090E002C0880F991F38
:108A50003A95E2F7282B28BB089528B381E090E0EF
:108A600002C0880F991F3A95E2F78095822388BB50
:108A700008958091520181FD1CC0E5E6F0E006C03A
:108A80008091520182FD15C0E2E3F0E085B38F7062
:108A9000682B65BB908121E030E002C0220F331FBC
:108AA0004A95E2F7822F8095982390838081822BCC
:108AB0008083089580915A015091FA0990E0252F02
:108AC00030E04091FB09241B31092817390744F491
:108AD0008091530181FD04C0809157018E3540F48F
:108AE000F8948091FC0960E00E9495447894089580
:108AF00080915A01581738F4F8948091FC0960E885
:108B00000E9495447894089580915A012091A30A77
:108B1000281740F4F8948091A70A60E80E949544D1
:108B20007894089580915A0190E030E04091A60A2F
:108B3000241B3109281739073CF0F8948091A70AC3
:108B400060E00E9495447894089580916001873E8A
:108B500040F0909165018091950A891710F460E8C2
:108B600001C060E0F8948091960A0E949544789440
:108B70000895209165018091970A821710F460E8AA
:108B800007C090E0019730E0281739073CF460E017
:108B9000F8948091980A0E949544789408958530BD
:108BA00079F1863070F4823001F1833020F4813025
:108BB00009F059C017C08330D9F0843009F053C090
:108BC0001BC0883009F440C0893030F4863041F150
:108BD000873009F048C034C08930D1F18A3009F0BB
:108BE00042C03CC080915B0105C080915B0106C022
:108BF00080915A0140E02FC080915A0140E031C07D
:108C000020915C0130915D0140E0862F90E063E0AF
:108C1000880F991F6A95E1F72817390728F123C0B3
:108C200020915C0130915D0140E0862F90E053E09F
:108C3000880F991F5A95E1F782179307A8F013C080
:108C400040E08091530707C040E08091530709C07E
:108C500040E080911802861738F005C040E080910E
:108C60001802681708F041E0842F08951F93CF93EE
:108C7000DF93EC0140916501509160012091580112
:108C8000309159018091660A8F70823051F487E0EB
:108C9000283F380780F4E3E036952795EA95E1F719
:108CA00008C083E02C3F380730F436952795369579
:108CB0002795922F01C09FEF8881481700F1898185
:108CC0008417E8F08A815817D0F08B818517B8F0A7
:108CD0008C819817A0F08D81891788F08F818F7013
:108CE00068850E94CF45882351F08F8182958F70CF
:108CF00069850E94CF45882311F010E801C010E07B
:108D0000F8948E81612F0E9495447894812FDF9191
:108D1000CF911F9108951F9340916501509160017B
:108D200020915801309159018091660A8F708230EC
:108D300051F487E0283F380778F413E036952795FB
:108D40001A95E1F70AC083E02C3F380728F43695DE
:108D500027953695279501C02FEF8091EF08E82FD2
:108D6000EF70E83010F480E00EC0EC3009F462C01F
:108D7000EF3019F0E83021F41DC080995BC01AC0B3
:108D8000E82FE77081E0F0E0EE0FFF1FEE5AF24FA0
:108D9000E181E43010F490E005C0E83010F490E494
:108DA00001C090E8882319F080E8891B982F992347
:108DB00009F040C08091F108982F81FF04C0809194
:108DC0008C0181FD37C080918F01882399F58091B6
:108DD0009E01882379F580919101847811F092FDAC
:108DE00029C08091EA08481728F18091EB08841780
:108DF00008F18091E9085817E8F08091ED082817EC
:108E0000C8F08091EE088217A8F09091A00180919F
:108E10001D09981778F01091EC088091480980930B
:108E2000B508F8948091550182608093550178943B
:108E300060E80CC080E88093B508F89480915501F3
:108E40008D7F80935501789460E010E0F8948091D4
:108E5000F0080E9495447894812F1F910895EF9215
:108E6000FF920F931F938091B9089091BA08892BB4
:108E700041F080915301807321F48091540182FF6D
:108E800003C01092490107C0809149018A3018F44B
:108E90008F5F809349019091650180911309981724
:108EA00008F491C020915801309159018091660ACF
:108EB0008F70823051F487E0283F380780F4F3E068
:108EC00036952795FA95E1F708C083E02C3F3807DF
:108ED00030F43695279536952795922F01C09FEF50
:108EE00080911409981708F46EC020915C013091AC
:108EF0005D018091170990E073E0880F991F7A95C2
:108F0000E1F78217930718F460E8E62E01C0EE241B
:108F1000F09015090091800C1091810C0E946499C9
:108F200080179107F0F40091800C1091810C0E9441
:108F30006499081B190B8091180924E6829FC001CF
:108F400011248017910768F4F294F694F69453E094
:108F5000F522F394FF0C80914901F81610F440E8D3
:108F6000E42E2091150925FF24C09091540A809188
:108F7000770D9817E0F080917E0D9817C0F08091E2
:108F8000850D9817A0F080918C0D981780F0809136
:108F9000930D981760F080919A0D981740F080918A
:108FA000A10D981720F08091A80D981710F430E8C3
:108FB000E32E822F609116090E949221882321F0CE
:108FC00020E8E22E01C0EE2490915A018091190907
:108FD000891710F490E8E92E20911209809154012C
:108FE00084FF04C027FF02C080E8E82E809156016C
:108FF00090E08F709070892B59F024FF02C000E838
:10900000E02EF894809156018F5F809356017894FA
:10901000F89480911A096E2D0E949544789400006E
:10902000F89480915301EE2011F0886001C0877F91
:109030008093530178941F910F91FF90EF900895C2
:109040008091C20B813061F48091C10B682F70E078
:109050006F5F7F4F85E0660F771F8A95E1F738C015
:109060008091A80B87FD32C080916401882371F53F
:10907000F894209162013091630178946091AD0A77
:10908000663038F480912B0580FF03C080E2861B98
:10909000682FC9010E94921D9B01AC01BB27A92F1B
:1090A000982F872F885F9F4018F06CEB7FE710C0E8
:1090B000A5E05695479537952795AA95D1F7B9011B
:1090C000203D310528F460ED70E002C060E070E6FC
:1090D000CB010895982F662311F403C0961B9617B1
:1090E000E8F730916D0A262F291B213011F122302B
:1090F00021F480916B0A84FF1CC03E3031F466304D
:1091000021F480E09230B1F412C0683139F43A337E
:1091100029F480E09E7F9A3069F409C0303211F062
:1091200080E00895223029F080E0253019F481E0B4
:10913000089581E008958091F30985FD30C0209164
:109140005801309159018091660A8F70823051F434
:1091500047E0283F340780F493E0369527959A95A9
:10916000E1F708C053E02C3F350730F436952795DA
:1091700036952795922F01C09FEF8091A50A9817E9
:1091800080F48091600190E022E330E0AC01429FE6
:10919000C001439F900D529F900D112402C09091E9
:1091A0006601892F089520917C0130917D01809185
:1091B000840190918501822B932B892B01F590914D
:1091C000800180918201892BD1F4F89480918301F0
:1091D000809382018091860190918701909385010F
:1091E00080938401809181018093800180917E0130
:1091F00090917F0190937D0180937C0178940895F4
:109200008091930B82958695869583709091940BAF
:10921000990F990F892B08958091580190915901C8
:1092200040915801509159018091660A8F708230A7
:1092300051F487E0483F580778F463E05695479526
:109240006A95E1F70AC083E04C3F580728F4569529
:1092500047955695479501C04FEF8091F30982FFDE
:1092600019C0409160018091FE0983FF13C0909165
:10927000F5098091B70A989FC0011124892F992779
:10928000869586958695840F911D90FF02C04FEFBD
:1092900001C0482F409366018EE193E06EE022EB1F
:1092A0003AE00E944F1E08952F923F924F925F9294
:1092B0006F927F928F929F92AF92CF92EF92FF9296
:1092C0000F931F93DF93CF9300D000D0CDB7DEB7BD
:1092D0004B015C834B833A832983602F0E94921D4C
:1092E0001B012C01C4016E2D0E94921D3B014C01FB
:1092F0008B819C816C2D0E94921D7B018C01898148
:109300009A816A2D0E94921DA4019301220D331DA2
:10931000441D551D2E0D3F1D401F511F260F371F89
:10932000481F591F203080E838078EEF480780E03B
:10933000580710F08FEF07C0205030484F4F5F4F55
:10934000CA01AA27BB270F900F900F900F90CF91C3
:10935000DF911F910F91FF90EF90CF90AF909F9072
:109360008F907F906F905F904F903F902F900895D7
:109370002F923F924F925F926F927F928F929F9225
:10938000AF92BF92CF92DF92EF92FF920F931F9313
:10939000DF93CF9300D000D00F92CDB7DEB7FC01A2
:1093A0006B01DA017C91E79E702D1124D601FC90AF
:1093B0001196BC91B983DA0111968C91E89EE02C4C
:1093C00011248827139F4001029F3001129F700CC7
:1093D000811C981E039F700C811C981E1124C901CA
:1093E000809590954427199F6001089F5001189F10
:1093F000B00CC11CD41E099FB00CC11CD41E11247A
:10940000009510951C014427139DD001029DC001B9
:10941000129D900DA11DB41F039D900DA11DB41FA1
:10942000112429016627159DA001049D9001149D1A
:10943000300D411D561F059D300D411D561F112435
:109440001D01442455242A823B824C825D829A016C
:10945000442755275601CC24DD243401882499243F
:10946000672F6F0D8F01060F111D3980730D1F01BE
:10947000270E311CFE0C2F014F0C511C8981E80E68
:10948000EE0DF11D8A819B81B901A5019301D801DF
:109490000C91D101EC90D201CC90A0800E94544953
:1094A0000F900F900F900F900F90CF91DF911F9121
:1094B0000F91FF90EF90DF90CF90BF90AF909F9073
:1094C0008F907F906F905F904F903F902F90089576
:1094D0003F924F925F926F927F928F929F92AF9244
:1094E000BF92CF92DF92EF92FF920F931F93DF9381
:1094F000CF9300D000D0CDB7DEB7E0906701F090F9
:109500006801009158011091590193E01695079553
:109510009A95E1F7A02E409165018CE094E068E017
:109520009E012D5F3F4F0E944F1E84E194E068E052
:10953000402F9E012F5F3F4F0E944F1E4B8069803E
:10954000660C660C660C3C805A80550C550C550C0C
:10955000E42DF0E0E45FFB4F908189E1989F80016A
:109560001124F694E794F694E7940E151F0518F06D
:10957000CC24DD242FC0E32DF0E0E45FFB4F80819D
:10958000891BE82FF0E0EE0FFF1FE758FA4F859197
:10959000949163EA0E94921D72958295929560EF74
:1095A0009827962398278727862387279C01C7011A
:1095B000801B910BBC014427379FD001269FC0011F
:1095C000369F900DA11DB41F279F900DA11DB41FA4
:1095D00011246C01E981F0E0EC5EFB4F00810A157B
:1095E00018F020E030E02FC0EA81F0E0EC5EFB4FA5
:1095F0008081801BE82FF0E0EE0FFF1FE758FA4F45
:109600008591949163EA0E94921D7295829592953C
:1096100060EF9827962398278727862387279C0122
:109620008E2D801B90E0FC0144273F9FD0012E9F90
:10963000C0013E9F900DA11DB41F2F9F900DA11D35
:10964000B41F11249C0188273D9D50012C9D400191
:109650003C9D900CA11CB81E2D9D900CA11CB81E09
:109660001124C601809590954427399F8001289F39
:109670007001389FF00C011D141F299FF00C011D73
:10968000141F112420953095BC014427379FD00129
:10969000269FC001369F900DA11DB41F279F900DDE
:1096A000A11DB41F1124F9016627FD9DA001EC9DA9
:1096B0009001FC9D300D411D561FED9D300D411D4B
:1096C000561F1124CD01AA27BB279A0144275527ED
:1096D0007801002711274501AA24BB24062D040D7B
:1096E000A02FB0E0A453BC4F630C77246CEC73E064
:1096F000660E771E450CC42CDD24C60ED71E530CF7
:10970000E52DF0E0E60FF71FB901A70194010C91D8
:10971000D301EC90D601CC90A0800E9454490F90C8
:109720000F900F900F90CF91DF911F910F91FF90AD
:10973000EF90DF90CF90BF90AF909F908F907F90F1
:109740006F905F904F903F900895CF93DF93282FB5
:10975000DB01EA018981FB01E80FF11DE0812E1791
:1097600018F06FEF7FEF15C08881A80FB11D6C91C5
:10977000621718F060E070E00CC0E61BF0E0EE0F3E
:10978000FF1FE758FA4F85919491261B622F0E9484
:10979000921DCB01DF91CF9108956F927F928F92AE
:1097A0009F92AF92BF92CF92DF92EF92FF920F9370
:1097B0001F93DF93CF9300D000D0CDB7DEB75C010D
:1097C000762E642EA0E48A2E912C880E991EC40158
:1097D00068E0472D6E010894C11CD11C96010E94BF
:1097E0004F1E8501085B1F4FF3E0EF2EF12CEC0EAE
:1097F000FD1EC80168E0462D97010E944F1E872D6F
:10980000B401A6010E94A54B4C01862DB801A70109
:109810000E94A54B8C01C501B601A7019401E8E0A7
:10982000EE2E0E94B8490F900F900F900F90CF919D
:10983000DF911F910F91FF90EF90DF90CF90BF903D
:10984000AF909F908F907F906F9008950F931F938C
:1098500020918D0180910D0A90E0820F911D29E1E8
:1098600030E0829FA001839F500D929F500D1124E4
:109870008091110A481B51092091670130916801BC
:109880003695279536952795C90182509F4F4817E1
:10989000590708F088C08091120985FF03C08091A4
:1098A000180202C08091530790910405992321F476
:1098B000823008F078C003C0981708F474C0009193
:1098C000EB091091EC092417350708F5842F821B4A
:1098D000282F209530E0812F90E0AC01249FC0011B
:1098E000259F900D349F900D1124892F990F990B6E
:1098F000182F802F90E0AC01249FC001259F900D70
:10990000349F900D1124892F990F990B082F809166
:1099100058019091590123E0969587952A95E1F792
:109920006091DC09681798F5861B682F8091DD0926
:10993000681718F010E000E02AC0E82FF0E0EE0F02
:10994000FF1FE758FA4F859194910E94921D6095F0
:109950007095272F30E0812F90E0AC01249FC0014B
:10996000259F900D349F900D1124892F990F990BED
:10997000182F802F90E0AC01249FC001259F900DEF
:10998000349F900D1124892F990F990B082F8091E6
:10999000F80883FF03C00093B10808C08091EB0969
:1099A0008093B10803C01092B10810E0812F1F917D
:1099B0000F9108956091F10970E0607F7070E3E0AD
:1099C00075956795EA95E1F76E5F0E94921D9B0180
:1099D000AC018091720A843111F066EB01C069EB31
:1099E000C9010E94921D9B01AC01232F342F452FEA
:1099F0005527C90108950E94DA4CFC0120916201AB
:109A00003091630140916401442309F01EC088270E
:109A10003F9FB0012E9FA0013E9F500D611D781FFA
:109A20002F9F500D611D781F1124872F803108F062
:109A300030C052956295729540EF76277423762751
:109A40006527642365279B0126C0403110F5A4E0FB
:109A500036952795AA95E1F7942F9295907F80E00F
:109A6000822B932B66279F9FA0018E9F90019E9F24
:109A7000300D411D561F8F9F300D411D561F112463
:109A8000852F882331F4BB27A52F942F832F9C018A
:109A900002C02FEF3FEFC90108952091A4012223B6
:109AA00029F41092A6011092A501089530E083E0F8
:109AB000220F331F8A95E1F78091760A90E0880F94
:109AC000991F820F931F0E94FB4C97FF02C08FEFDC
:109AD0009FE79093A6018093A5010895CF92DF920E
:109AE000FF920F931F93CF93DF9350916D0A809154
:109AF0006B0A81FD15C0503211F454E211C084FF8D
:109B000003C0952F9F5F02C0952F9E5F80916C0AC6
:109B100084FD04C0543010F0592F02C0592F550F46
:109B200010917B0A012F0150F52E612F43C0E62FC3
:109B3000F0E0E851FE4F40894877A0EFB1E07FEFB9
:109B400098E0C92ED12CCE0EDF1EC02FD0E0CA0F58
:109B5000DB1F2CC0242F30E018968C91189790E0D2
:109B60008877907028173907F9F49C91F601808165
:109B7000903859F4803849F4E72F171708F4E12F8B
:109B8000F0E0E851FE4F90858881292F250F281B92
:109B9000521708F4251B2F1508F4F22E452F421BEF
:109BA00019F04F1508F4F42E11967F5F701791F697
:109BB00061500150662309F0BACF812F87708F5F03
:109BC00010E08150E82FF0E0E851FE4F908D19171A
:109BD00008F4192F8823A9F79091710A8091720ACD
:109BE000F92F282F822F9F2F6F2D0E94921D812FDA
:109BF00090E08617970718F080E090E004C0FB0122
:109C0000E81BF90BCF010E94DA4C90937901809305
:109C10007801DF91CF911F910F91FF90DF90CF904E
:109C20000895682F809158019091590121E0893160
:109C3000920710F480E00895885191400E94921D8F
:109C400026E096958795779567952A95D1F764369E
:109C5000710510F084E60895862F08956F927F9223
:109C60008F929F92AF92BF92CF92DF92EF920F931B
:109C70001F93DF93CF9300D000D0CDB7DEB74091D4
:109C8000650185EF97E06CE09E012F5F3F4F0E94DA
:109C90004F1E0E949B48482F81E098E06CE09E0197
:109CA0002D5F3F4F0E944F1EE981F0E0EB50F84FCF
:109CB000408129E1429F9001112480916701909198
:109CC000680196958795969587952817390788F4A2
:109CD000EA81F0E0EB50F84F8081841BE82FF0E040
:109CE000EE0FFF1FE758FA4F8591949163EA0E94A7
:109CF000921DEB81F0E0EF5FF74F208160916601EC
:109D0000261788F4EC81F0E0EF5FF74F8081821B2B
:109D1000E82FF0E0EE0FFF1FE758FA4F859194917E
:109D2000621B0E94921D0091580110915901A3E0FD
:109D300016950795AA95E1F7409165018CEE94E0A0
:109D400068E05E010894A11CB11C95010E944F1EA1
:109D5000F3E0CF2ED12CCC0EDD1E84EF94E068E032
:109D6000402F96010E944F1E809165016CEE74E0B9
:109D7000A5010E94A54B3C01802F64EF74E0A60171
:109D80000E94A54B4C018CE694E0B501A60193011D
:109D90008401E8E0EE2E0E94B8498093C2018CEA6B
:109DA00094E0B501A60193010E94B8498093BB01DC
:109DB000409165018CE696E06CE020E636E00E947A
:109DC000701E8093A4010F900F900F900F90CF9171
:109DD000DF911F910F91EF90DF90CF90BF90AF90E8
:109DE0009F908F907F906F900895409165012CE631
:109DF00036E0C9016CE0285130400E94701E90E0AE
:109E00000E94FB4C909389018093880108958F9262
:109E10009F92AF92BF92CF92DF92EF92FF920F93F9
:109E20001F93CF93DF936C018091760AC82FD0E007
:109E3000CC0FDD1FC050DF4F00916E0A9091710A68
:109E40008091720A882E992E0E94F54EB0906D0A6C
:109E500080916B0A81FD18C090E2B91619F434E2C2
:109E6000B32E12C084FF03C09B2D9F5F02C09B2DA9
:109E70009E5F80916C0A84FD05C083E08B1510F411
:109E8000B92E02C0B92EBB0C023008F04DC0809133
:109E9000760A813508F048C0CC15DD0548F400236A
:109EA00011F000E002C00B2D0150C80DD91D3CC0BF
:109EB000909165018091B709891708F446C0E09038
:109EC0007A01F0907B01CE018C199D090E94FB4C18
:109ED000E816F906D0F1F8941092870110928601E5
:109EE00080918601909187019093850180938401F0
:109EF0000093830180918301809382017894F89488
:109F0000F0927F01E0927E0180917E0190917F012D
:109F100090937D0180937C01009381018091810168
:109F2000809380017894E7C0CC15DD0570F48091B2
:109F3000760A90E0880F991F80509F4F909374018C
:109F400080937301C0E0D0E002C0CC19DD09811418
:109F5000910439F409C00F5F0B1508F000E0C8192F
:109F6000D9098C169D06B8F380916B0A282F30E032
:109F7000C901827A9070823A910539F480916D0A14
:109F80008C3018F4AA24A39402C0A0906F0A21FF79
:109F900009C010C0002311F0015001C0012FC80DED
:109FA000D91D02C01B2D1150802F6A2D0E946A48B6
:109FB000882381F7CE010E94FB4C9C0180916401B3
:109FC000803120F49FEF2F3F390751F4F89480E857
:109FD00080938301809183018093810178948BC069
:109FE00069018FE72D3B380720F08CEBC82E8FE7F7
:109FF000D82EC4010E94FB4C7C0180917A01909183
:10A000007B018C159D0518F0E114F10429F4E6019B
:10A01000C81BD90B102F3FC09C012C193D09802F64
:10A020009B2D915007C0882311F0815001C0892FCA
:10A030002E193F092E153F05B0F7882311F0182F70
:10A0400001C01B2D1150E701C21BD30B90916B0A6D
:10A0500091FF09C010C0112311F0115001C01B2D38
:10A06000CE0DDF1D01C0BA94812F6A2D0E946A486F
:10A07000882389F710C0809165018E3160F096FFCA
:10A080000AC080918101181731F4CE0DDF1D112314
:10A0900009F41B2D1150F89480918201811721F44D
:10A0A000D0938501C093840110938301D0938701DD
:10A0B000C093860180916D0A8A3360F480916501B6
:10A0C000853040F420917A0130917B012C0F3D1FA7
:10A0D000912F02C0902F96019093810130937F01C0
:10A0E00020937E0180918001891721F430937D01B6
:10A0F00020937C017894DF91CF911F910F91FF9075
:10A10000EF90DF90CF90BF90AF909F908F90089589
:10A11000AF92BF92CF92DF92EF92FF920F931F9375
:10A12000DF93CF9300D000D0CDB7DEB7409165016B
:10A130008CE693E068E06E010894C11CD11C960186
:10A140000E944F1E0E949B48182FF3E0EF2EF12C27
:10A15000EC0EFD1E84E793E068E0412F97010E941A
:10A160004F1E809165016CE673E0A6010E94A54B2D
:10A170005C01812F64E773E0A7010E94A54B8C016D
:10A180008CE293E0B601A7019501E8E0EE2E0E9473
:10A19000B849082F10E008531F4F8091B408882356
:10A1A000B9F090E080509F4FAC012227159FD0015D
:10A1B000049FC001149F900DA11DB21F059F900D1B
:10A1C000A11DB21F1124892F9A2FAB2FBB278C0101
:10A1D00080914909807F803129F48091460968E7A0
:10A1E00076E01DC080911B09807F803179F48091D9
:10A1F000070969E876E00E94933AA801480F511DCB
:10A20000CA0151E08834950780F113C080910A0992
:10A21000807F803189F4809108096AE976E00E94A4
:10A22000933A9801280F311DC90131E08834930712
:10A23000E0F08C010058104041E0073C140718F48E
:10A24000802F885C01C08FEF8093AB080F900F9038
:10A250000F900F90CF91DF911F910F91FF90EF9092
:10A26000DF90CF90BF90AF90089508EC10E0E8CF5A
:10A270008F929F92AF92BF92CF92DF92EF92FF9216
:10A280000F931F93CF93DF938091540184FF48C0B5
:10A2900010915D0A80914909807F803329F4809173
:10A2A000460968E776E013C080911B09807F803300
:10A2B00029F48091070969E876E009C080910A09CC
:10A2C000807F803351F5809108096AE976E00E9429
:10A2D000933A482F50E0212F30E0CA0163E0880F05
:10A2E000991F6A95E1F7841B950BBC014427379FA2
:10A2F000D001269FC001369F900DA11DB41F279F3E
:10A30000900DA11DB41F1124892F9A2FAB2FBB27AD
:10A310009093AA088093A908F0C01093A908EBC0F5
:10A32000409165018EE093E060E124EB3AE00E9409
:10A330004F1EE091B40AF0E0E25FFC4F908189E1AA
:10A34000989F80011124C0916701D0916801D69532
:10A35000C795D695C7950C171D0718F0C0E0D0E03B
:10A3600031C0E091B50AF0E0E25FFC4F8081891BCB
:10A37000E82FF0E0EE0FFF1FE758FA4F8591949118
:10A3800063EA0E94921D9B01AC0132954295529561
:10A3900020EF542752235427432742234327CA013F
:10A3A000C01BD10BAC0122275D9FD0014C9FC00187
:10A3B0005C9F900DA11DB21F4D9F900DA11DB21F5E
:10A3C0001124EC014E0180949094E091B20AF0E0E7
:10A3D000E25EFC4F208160916601261718F020E0B4
:10A3E00030E013C0E091B30AF0E0E25EFC4F808100
:10A3F000821BE82FF0E0EE0FFF1FE758FA4F859120
:10A400009491621B0E94921D9B0188273D9F6001D1
:10A410002C9F50013C9FB00CC11CD81E2D9FB00C2E
:10A42000C11CD81E11248827399D8001289D7001E8
:10A43000389DF00C011D181F299DF00C011D181FDF
:10A440001124209530954427399DD001289DC001C5
:10A45000389D900DA11DB41F299D900DA11DB41F05
:10A460001124F9016627FD9FA001EC9F9001FC9F3C
:10A47000300D411D561FED9F300D411D561F1124FB
:10A480007091B20A7295707FF091B40A6091B50A2A
:10A49000E091B30AE295E07FCD01AA27BB279A019C
:10A4A000442755277801002711275601CC24DD24A5
:10A4B000072F0F0F10E0025D1D4F760FC72FD0E062
:10A4C000C25DDD4FFE0FAF2FB0E0A25DBD4FE60FC6
:10A4D0008E2E99246EE272E0860E971EB901A701B6
:10A4E0009501F8010081E880CC90F401A0800E94E1
:10A4F00054498093A9081092AA08DF91CF911F9127
:10A500000F91FF90EF90DF90CF90BF90AF909F9012
:10A510008F9008951F9380917A0A86FD2DC06091D7
:10A52000730170917401CB0188968150914018F4A9
:10A5300060E070E011C0685D70408AE991E00E94BF
:10A54000921D672F782F892F992781E0683A780725
:10A5500018F0E9E1F0E004C0E0ECF1E0E61BF70BF5
:10A56000809165018B3008F045C080917A0A83FFA5
:10A5700041C0E050FE4F3EC01091780A112389F18E
:10A580000E940935982F1230C8F0812F0E94114E79
:10A59000182F0E940935189F90011124232F33276B
:10A5A000482F50E0410F511D420F531FCA018070C8
:10A5B000892B19F4942F413E08F090EE8091770A90
:10A5C000989FF001112490E034E0F695E7953A95D4
:10A5D000E1F724E0880F991F2A95E1F7E80FF91FAA
:10A5E00009C08091770AE82FF0E084E0EE0FFF1FAA
:10A5F0008A95E1F7A0917801B091790160916201AB
:10A600007091630120916401222309F01EC0882704
:10A610007B9FA0016A9F90017A9F300D411D581FBA
:10A620006B9F300D411D581F1124852F803108F07C
:10A6300032C032954295529520EF54275223542729
:10A64000432742234327CA0122C0203120F514E0CA
:10A65000769567951A95E1F7922F9295907F80E015
:10A66000862B972B66279B9FA0018A9F90019A9F1C
:10A67000300D411D561F8B9F300D411D561F11245B
:10A68000852F882341F4BB27A52F942F832F853650
:10A69000910528F002C08FEF9FEF84569040E81795
:10A6A000F90708F4CF01F89490937B0180937A0125
:10A6B00078941F910895AF92BF92CF92DF92EF925C
:10A6C000FF920F931F93DF93CF9300D000D0CDB7AD
:10A6D000DEB74091650113E0C12ED12CCC0EDD1EFA
:10A6E00085EF97E06CE096010E944F1E0E949B4808
:10A6F000182F81E098E06CE0412F7E010894E11C66
:10A70000F11C97010E944F1E8091650165EF77E073
:10A71000A6010E94A54B5C01812F61E078E0A701B2
:10A720000E94A54B8C0185E697E0B601A701950133
:10A73000BCE0EB2E0E94B849082F10E000501048F2
:10A7400080918C0181FF05C00E94264C081B1109D5
:10A750003BC08091540185FF33C0C090650180915A
:10A76000390AC81688F18091850A87FF02C040E047
:10A7700002C040E8481BE12CA1E8FA2EE00EF11ED1
:10A78000F694E794009160018091680A6091690AEB
:10A790002E2D0E949D1D282F60913A0AC61638F46E
:10A7A0008091390A4E2D0C2D0E949D1D282FE22EDE
:10A7B000FF24EE0CFF1C20E03FE7E20EF31E2DC04D
:10A7C000C8010E94025B8C018091750190917B0A07
:10A7D0008150981708F4892F90E0FC0173E0EE0F88
:10A7E000FF1F7A95E1F7E81BF90BED58F24F8481D2
:10A7F000081B11098091F30984FD0AC060915B0177
:10A80000409160018CE793E00E94CD4B081B110939
:10A8100080916D017801E81AF1088091F10880FFBC
:10A8200004C00E948B46E81AF10880910A09807FD3
:10A83000803261F4809108096AE976E00E94933AD7
:10A8400020E830E0E20EF31EE81AF10880915C0A7D
:10A8500087FF04C0482F4058CC2404C040E8481B60
:10A86000CC24C39400915A0184E66EEA20E00E9451
:10A870009D1D482F009158011091590163E01695D4
:10A8800007956A95E1F783E266E420E00E949D1D4A
:10A89000282F30E0CC2029F0C701821B930B9C01AC
:10A8A00002C02E0D3F1D8091C30B882329F0282F55
:10A8B00030E02050304826C0009165018091B709F2
:10A8C000801738F08091790A282F30E020503048E6
:10A8D00020C06091F507061748F44091790A50E0CE
:10A8E000405050480E94DE1D9C010CC08091910197
:10A8F000847841F08091BD09807F20E030E8281BFA
:10A90000310907C09FE72130390718F420E030E013
:10A9100002C020503F478091330A682F70E026170D
:10A92000370708F49B01F894309374012093730166
:10A93000809175018093700D78940F900F900F9017
:10A940000F90CF91DF911F910F91FF90EF90DF90CB
:10A95000CF90BF90AF900895482F4F70807F6827A9
:10A96000423009F49DC0433030F4442359F0413063
:10A9700009F0B6C053C0463009F499C0473009F019
:10A98000AFC099C0862F90E08077907034E09595A5
:10A9900087953A95E1F7E82F67FF2EC030919E0129
:10A9A000332391F08091910186FF0EC020918E019A
:10A9B000822F82958F70831720F4285820938E0160
:10A9C00007C0295820938E018091520180FF06C054
:10A9D000809155018062809355010895F0E0E8511F
:10A9E000FE4F90818091A201892B8093A2012BB30D
:10A9F000892F809582230DC0F0E0E851FE4F9081B1
:10AA00002091A201892F809582238093A2018BB38C
:10AA1000892B8BBB8AB3982B9ABB0895862F90E025
:10AA20008077907024E0959587952A95E1F7382FE7
:10AA30008230E8F467FF0DC02091650081E090E06E
:10AA400002C0880F991F3A95E2F7282B20936500E2
:10AA500008952091650081E090E002C0880F991F61
:10AA60003A95E2F78095822380936500089567FF09
:10AA70000BC028B381E090E002C0880F991F3A957F
:10AA8000E2F7282B28BB089528B381E090E002C0AC
:10AA9000880F991F3A95E2F78095822388BB089525
:10AAA0008091520181FD1CC0E5E6F0E006C0809176
:10AAB000520182FD15C0E2E3F0E085B38F70682B90
:10AAC00065BB908121E030E002C0220F331F4A9520
:10AAD000E2F7822F8095982390838081822B808358
:10AAE00008958091530187FD15C08091FE0982FD74
:10AAF0000AC080915F0A2AE0829FC00111249093CE
:10AB0000C50A8093C40AF8948091530180688093A9
:10AB1000530178940895482F8BE0489F90011124A9
:10AB200076956795260F371F54E0369527955A95E9
:10AB3000E1F7C9018070892B11F08FEF01C0822FDE
:10AB4000481710F0842F11C09091BE0A891768F43D
:10AB50008FE0989FC0011124840F911D44E09695C9
:10AB600087954A95E1F790FD8FEF8093BE0A08958F
:10AB70008091080A8093BF0A8091070A8093C00AD7
:10AB800008958091080A2091070A82239091030A70
:10AB900089239091040A892380FD02C080E00895F2
:10ABA00080E02B50253108F481E008953091C00AEF
:10ABB000332331F14091080A2091070A822F842320
:10ABC0009091030A89239091040A892380FF03C08E
:10ABD0002B50253180F08091BF0A882341F003C0BB
:10ABE0004093BF0A04C081508093BF0A089531503A
:10ABF0003093C00A08958091BF0A8823A1F7F0CF4F
:10AC00000895BC018091F209482F84FF04C080910F
:10AC10005307882321F520915801309159018091E3
:10AC2000660A8F70823051F487E0283F380780F43D
:10AC300093E0369527959A95E1F708C083E02C3F7D
:10AC4000380730F43695279536952795922F01C011
:10AC50009FEF8091600A981738F443FD05C0109269
:10AC6000B90A1092B80A08959B0177FF04C0222701
:10AC70003327261B370B8091100A90E028173907DD
:10AC80000CF473C077FF07C09091B70A8091F90860
:10AC9000891758F008956115710539F09091B70A38
:10ACA0008091FF09981708F060C08091B80A9091D0
:10ACB000B90A805090489C0140E050E02050304854
:10ACC0004F4F5F4F60507048CB01A0E0B0E0280FBD
:10ACD000391F4A1F5B1FCA01AA27BB27882319F403
:10ACE00040E050E006C0823019F44FEF5FEF01C042
:10ACF000A90180910E0A90E09695982F8827979544
:10AD0000879520E030E8281B390B4217530700F1E4
:10AD100080910F0A282F30E03695322F2227379561
:10AD20002795205030482417350798F45091080A89
:10AD30004091070A842F85239091030A89239091DB
:10AD4000040A892380FF04C0842F8B50853140F092
:10AD5000A901405050485093B90A4093B80A089549
:10AD60005093BF0A4093C00AF3CF08958091FE0923
:10AD700082FD07C01092B60A1092B70A1092C60A56
:10AD800009C080E48093B60A8091FF098093B70AD6
:10AD90001092C70AF8948091520182FD02C090E897
:10ADA00001C090E085B38F708067892B85BB969832
:10ADB000969A0895813059F0813030F0823051F008
:10ADC000833069F0E0E011C0E091FD090DC0E09131
:10ADD000FD0908C0E091FD09E295EF7005C0E09122
:10ADE000FD09E295E695E695E370F0E0E05BF14E53
:10ADF000E4918E2F08950F931F9300911E0A202F28
:10AE000030E02F7030702F30310509F44BC0809145
:10AE1000FE0983FF12C082FD10C08091C60A8823FC
:10AE2000D1F080912B0581FF04C08D7F80932B058D
:10AE300010C0826080932B050EC090915A018091C2
:10AE4000020A981740F490915A018091010A9817CC
:10AE500048F510E801C010E09091B70A2E30310596
:10AE600071F4802F82958F708630E0F4E82FF0E047
:10AE7000EE0FFF1FE654F24F1082918313C0F89437
:10AE8000802F612F0E94AC548091FE0985FF09C07C
:10AE900078940000F8941058802F805F612F0E94F2
:10AEA000AC5478941F910F9108959091F9088917E7
:10AEB00008F4892F9091FF09282F981708F4292F5B
:10AEC0008091FE0982FF12C08091B60A86FF0BC0F6
:10AED00080916701909168018038910598F01092F7
:10AEE000B60A1092B70A2093C70A08952093B70AAA
:10AEF000822F0E9424359091FF09981708F4892F1A
:10AF00008093C60A08958091540186FF03C09091F2
:10AF1000210902C09091000A953F28F480916001B8
:10AF2000965F981790F48091B70A833010F480E010
:10AF300001C082508093B70A0E9424359091FF0986
:10AF4000981708F4892F8093C60A08950F93982FB5
:10AF50008091540186FF03C08091210902C0809135
:10AF6000000A2091FF098F3EA0F4682F605F0091D6
:10AF70006001601730F04091C10A292F0E949D1D89
:10AF800007C0862F6FEF492F0E949D1D8093C10A35
:10AF9000282F822F0F910895EF92FF920F93E09147
:10AFA000B708F0E0A091B808B0E000915A019F0105
:10AFB0002C5E354F64E1E62E6AE0F62EEA0EFB1EAB
:10AFC000EB56F64F8081AB56B64F6C91F90140813C
:10AFD000F70120810E949D1D482F9091C0099F700C
:10AFE000E9F020915B01253610F480E006C02A3A92
:10AFF00010F086E402C0822F8456899F90011124AC
:10B0000055E0369527955A95E1F7240F311D832F8A
:10B010009927892B11F04FEF01C0422F842F0F91F8
:10B02000FF90EF9008958091FE0982FD12C020915B
:10B03000C40A3091C50A2115310539F0215030403C
:10B040003093C50A2093C40A04C081FD02C00E9447
:10B0500083578091530187FF18C08091FE0982FFBA
:10B060000DC08091120982FF09C00E94CC57982F11
:10B070008091B70A891710F49093B70AF8948091D9
:10B0800053018F7780935301789408950F93009123
:10B090005A018091010A6091020A4091030A2091AD
:10B0A000040A0E949D1D0F9108950E94921D9B010C
:10B0B000AC0174E056954795379527957A95D1F769
:10B0C000DA01C90180709078B0700097A105B105D0
:10B0D00019F06FEF7FE701C0B901CB010895AF927E
:10B0E000BF92CF92DF92EF92FF920F931F93CF9375
:10B0F000DF936C01C091BC0AD091BD0A8091FE091A
:10B1000086FF1CC01C141D04CCF480E3C816D104B7
:10B1100014F000E402C00C2D005FC601602F0E94F5
:10B1200055586C011C161D064CF4CE01602F0E9470
:10B130005558EC019093BD0A8093BC0AF0900C0A1C
:10B14000CE01805090486F2D0E94921D672F782F5E
:10B15000892F99270F2D10E01695102F002717958E
:10B160000795109501951F4F060F171FB0900A0AFB
:10B17000C601805090486B2D0E94921D6B017C018E
:10B18000A0900B0A8091B80A9091B90A805090481B
:10B190006A2D0E94921DCD2CDE2CEF2CFF244B2D0E
:10B1A00050E05695542F4427579547955095419513
:10B1B0005F4F4C0D5D1D400F511F672F782F892F5A
:10B1C00099272A2D30E03695322F2227379527955B
:10B1D000309521953F4F260F371F420F531FE4E054
:10B1E00055954795EA95E1F7CA01DF91CF911F91F7
:10B1F0000F91FF90EF90DF90CF90BF90AF900895A8
:10B20000EF92FF920F931F93CF93DF93809153019F
:10B2100080FF04C08091530181FF4DC0F89480915C
:10B2200053018F778093530178941092B90A10924A
:10B23000B80A1092C30A1092C20A8091080A809339
:10B24000BF0A8091070A8093C00A9091030A282FB1
:10B2500030E0290F311D30FF02C08FEF01C0822F77
:10B260008093BE0A8091FE0982FD0EC08091530139
:10B2700081FD0AC080917D0A90E02091940B30916D
:10B28000950B2817390758F400915A018CE36EEAA0
:10B290004091050A2091060A0E949D1DB4C080912C
:10B2A0005F0A2AE0829FC00111249093C50A80930F
:10B2B000C40A80E0A8C0C0916701D0916801809164
:10B2C000BA0A9091BB0A8C1B9D0B9093BD0A809388
:10B2D000BC0AD093BB0AC093BA0A00915A0180916C
:10B2E000010A6091020A4091030A2091040A0E9417
:10B2F0009D1D182F0E94D6558091C00A90E0810FA5
:10B30000911D90FD8FEFBE010E948B559AE0899FA1
:10B3100070011124EC1AFD0A909160018091540192
:10B3200086FF03C08091210902C08091000A282F66
:10B3300030E0892F90E0281739071CF41E141F04F1
:10B34000D4F48091530187FD18C08091FE0982FDDD
:10B350000AC080915F0A2AE0829FC0011124909365
:10B36000C50A8093C40AF894809153018068809341
:10B370005301789402C00E9413588091540185FFB4
:10B3800004C0809106098823F1F5809158019091BD
:10B39000590153E0969587955A95E1F72091930AC4
:10B3A000281718F48091940A2EC08091FE0982FF1C
:10B3B00006C08091690190916A01892B31F10E9448
:10B3C000CC57182F8091530187FF14C0C7010E94EA
:10B3D0006F58810F911D992311F4182F05C0192F53
:10B3E000111F1127111F1150C7010E940156109300
:10B3F000C10A08C08091FE0981FF07C0812F0E9409
:10B40000A657182F812F0E945557DF91CF911F917A
:10B410000F91FF90EF9008950F931F938091120961
:10B4200081FF34C080914D01882349F08150809381
:10B430004D01882321F482E060E00E94AC548091A9
:10B440004C01882349F0815080934C01882321F4DA
:10B4500082E760E00E94AC5480914B01882349F060
:10B46000815080934B01882321F481E560E00E94A4
:10B47000AC5480914A01882349F0815080934A015D
:10B48000882321F481E660E00E94AC548091B60AE2
:10B4900090E0AC014074507086FD07C08091690156
:10B4A00090916A01892B09F4AAC08091B70A909102
:10B4B000C70A891709F47AC02091C80A981720F0A2
:10B4C000122F1F5F8F5F03C0122F11508150809386
:10B4D000B70A891731F41092B60A452B11F00E9471
:10B4E0000059012F03708091120981FF38C0802F0D
:10B4F0000E94DA568430A9F0853020F4833009F0B8
:10B5000051C006C08530B9F0863009F04BC01DC06F
:10B5100082E080934D01F89460E80E94AC547894E6
:10B5200041C082E080934C01F89482E760E80E9479
:10B53000AC54789437C082E080934B01F89481E555
:10B5400060E80E94AC5478942DC082E080934A0158
:10B55000F89481E660E80E94AC54789423C080FDA2
:10B5600002C010E801C010E0F894802F0E94DA5663
:10B5700095B38295807F9F70892B812B85BB969890
:10B58000969A78940000F8948091C80A0E94DA563E
:10B5900095B38295807F9F70982B1058192B15BBFF
:10B5A0009698969A78940093C80A29C01092B60A81
:10B5B0008091FE0980FF23C0F89485B38F7080636B
:10B5C00085BB9698969A78940000F89485B38F700E
:10B5D000806485BB9698969A78940000F89485B319
:10B5E0008F70806585BB9698969A78940000F89441
:10B5F00085B38F70806685BB9698969A78941F91D4
:10B600000F910895CF93DF93EC018091FE0984FFA1
:10B6100048C08091530187FF44C020916701309159
:10B620006801909165018091EE09891708F442C084
:10B630009091BE0A8AE0989FC0011124281739070B
:10B64000B8F4821B930B60911F0A0E94921D672F12
:10B65000782F892F99272091210A422F50E0CB0182
:10B660004617570708F4CA019C012C0F3D1F1AC04A
:10B67000A901481B590BCA0160911F0A0E94921D23
:10B68000672F782F892F99272091220A422F50E087
:10B69000CB014617570708F4CA019E01281B390B36
:10B6A00001C09E01C9018C1B9D0B9093C30A80931E
:10B6B000C20AE901CE01DF91CF91089582958F7082
:10B6C000E4E5FEE1E80FF11DE4918E2F0895E82FE7
:10B6D000F0E0EF70F070EC5AF14EE4918E2F089587
:10B6E000823118F0E5E6FEE104C0E82FF0E0EC5A04
:10B6F000F14E84910895282F66E10E940BC694E1D3
:10B70000899F302D1124822F0E940BC6992311F49A
:10B710008DE00895913011F48AE00895E92FF0E06A
:10B72000E753F54FE30FF11D319780810895282FDE
:10B7300090E0877090708959914EFC019491269504
:10B7400026952695E22FF0E0E65EF44F808189236E
:10B7500008958091640A982F92959F709A95F1F7B9
:10B76000A99A8F708A95F1F7A9980895F89495B3DE
:10B770009F70906895BB9698969A78940000F8947C
:10B7800095B3282F207F9F70292B25BB2091640A19
:10B79000322F32953F70932F9A95F1F7A99A2F7017
:10B7A000922F9A95F1F7A99878940000F89495B3A0
:10B7B0008295807F9F70982B95BB3A95F1F7A99A57
:10B7C0002A95F1F7A99878940000F89485B38F70C2
:10B7D00085BB9698969A78940895982F862F8F5FB8
:10B7E0008093260B803510F01092260B262F30E028
:10B7F000D901A753B54F11968C911197891791F0E4
:10B8000011969C93669566956695A62FB0E0277075
:10B8100030702959314EF9018491A65EB44F9C9144
:10B82000892B8C930895CF93DF93EC0126C0462F8C
:10B830004F5F4093260B403511F41092260B262FB4
:10B8400030E0D901A753B54F11968C911197891704
:10B8500091F011969C93669566956695A62FB0E03B
:10B86000277030702959314EF9018491A65EB44F8A
:10B870009C91892B8C932196642F603518F49881C4
:10B880009923A9F6DF91CF910895AC01862F8F5FA0
:10B8900057FF28C08093260B803510F01092260B9E
:10B8A000262F30E0D901A753B54F11968C911197EF
:10B8B0008D3299F08DE211968C936695669566951A
:10B8C000A62FB0E0277030702959314EF9018491CC
:10B8D000A65EB44F9C91892B8C9322273327241B7F
:10B8E000350B24C08093260B803510F01092260B68
:10B8F000262F30E0D901A753B54F11968C9111979F
:10B900008B3299F08BE211968C93669566956695CD
:10B91000A62FB0E0277030702959314EF90184917B
:10B92000A65EB44F9C91892B8C939A01C90108950E
:10B93000FF920F931F93CF93DF938C01E4E022E0FB
:10B94000F22E40E350E020E43CE9CEE0D0E00217E4
:10B95000130720F0021B130B4E0F511DCE018370F5
:10B960009070892B29F036952795E695762F2AC079
:10B97000762F7F5F262F30E0D901A753B54F119660
:10B980008C911197841791F011964C93669566955A
:10B990006695A62FB0E0277030702959314EF90115
:10B9A0008491A65EB44F9C91892B8C93EF2DF0E08F
:10B9B000EE0FFF1FE159F14EFA9425913491E8E022
:10B9C00040E350E02197FFEFCF3FDF0711F0672FF3
:10B9D000BECF902F905D872F8F5F8093260B803591
:10B9E00010F01092260B272F30E0F901E753F54FA6
:10B9F0008181891789F09183769576957695A72F21
:10BA0000B0E0277030702959314EF9018491A65E5B
:10BA1000B44F9C91892B8C93DF91CF911F910F9103
:10BA2000FF900895CF93DF93DC014BC0E42FF0E04B
:10BA3000EE0FFF1FE159F14E85919491A817B907B8
:10BA400018F420E330E004C0A81BB90B28E330E071
:10BA500096958795A817B90720F0A81BB90B2C5FFE
:10BA60003F4F96958795A817B90720F0A81BB90BEB
:10BA70002E5F3F4F96958795A817B90720F0A81B12
:10BA8000B90B2F5F3F4F922F562F5F5F262F30E06D
:10BA9000F901E753F54F8181891789F09183669504
:10BAA00066956695C62FD0E0277030702959314EC3
:10BAB000F9018491C65ED44F9881892B88834150C7
:10BAC000652F47FFB3CF862F8F5FAA30B105A0F057
:10BAD0008093260B803510F01092260B262F30E035
:10BAE000D901A753B54F11968C9111978D3A41F119
:10BAF0008DEA11968C9314C09A2F905D8093260B3B
:10BB0000803510F01092260B262F30E0D901A75374
:10BB1000B54F11968C911197891791F011969C93BE
:10BB2000669566956695A62FB0E027703070295906
:10BB3000314EF9018491A65EB44F9C91892B8C9370
:10BB4000DF91CF910895A998F89495B3807F9F7065
:10BB5000982B95BB8091640A982F92959F709A9527
:10BB6000F1F7A99A8F708A95F1F7A99878940895BA
:10BB7000F89495B3282F207F9F70292B25BB209107
:10BB8000640A322F32953F70932F9A95F1F7A99A54
:10BB90002F70922F9A95F1F7A99878940000F89455
:10BBA00095B38295807F9F70982B95BB3A95F1F75E
:10BBB000A99A2A95F1F7A9987894089581E00E94AE
:10BBC000B85D08951092250B82E00E94B85D109236
:10BBD000260B0895813011F48CE001C088E06130BB
:10BBE00009F48260413009F481600E94B85D0895D3
:10BBF00080680E94B85D08951F93182F8C3310F051
:10BC0000885E07C0883210F0845103C0843108F088
:10BC1000845D0E94F85D1093240B1F91089580931A
:10BC2000260B08958091260B0895982FE091260BFE
:10BC30008E2F8F5F8093260B803510F01092260B8D
:10BC40002E2F30E0D901A753B54F11968C91119743
:10BC5000891791F011969C93E695E695E695AE2F9F
:10BC6000B0E0277030702959314EF9018491A65EF9
:10BC7000B44F9C91892B8C930895CF93DF93EC0163
:10BC800003C00E94155E219688818823D1F7DF9139
:10BC9000CF910895CF93DF93EC0102C00E94155E0F
:10BCA000FE01219684918823C9F7DF91CF910895F1
:10BCB0001F93CF93DF93EC01162F03C011500E9406
:10BCC000155EFE0121968491882311F01123B1F7AE
:10BCD000DF91CF911F9108954091260B50E220C033
:10BCE0004F5F403508F040E02E2F30E0D901A753D8
:10BCF000B54F11968C911197803291F011965C930B
:10BD0000E695E695E695AE2FB0E02770307029599C
:10BD1000314EF9019491A65EB44F8C91892B8C938E
:10BD2000E42F842F81508F34D8F24093260B08954E
:10BD3000582F4091260B60E220C04F5F403509F438
:10BD400040E02E2F30E0D901A753B54F11968C91CA
:10BD50001197803291F011966C93E695E695E695F1
:10BD6000AE2FB0E0277030702959314EF90194910F
:10BD7000A65EB44F8C91892B8C93E42F442319F445
:10BD80001092260B0895541710F04035B0F24093EE
:10BD9000260B0895E091260BEC3310F050E509C016
:10BDA000E83210F05CE305C0E43110F454E101C066
:10BDB00058E26E2F70E223C04E2F4F5F403508F0DF
:10BDC00040E02E2F30E0D901A753B54F11968C914A
:10BDD0001197803291F011967C93E695E695E69561
:10BDE000AE2FB0E0277030702959314EF90184919F
:10BDF000A65EB44F9C91892B8C936F5FE42F6517DF
:10BE0000D8F2E093260B08950F931F93CF93DF93FF
:10BE1000082F10E8C0E0D0E0812F802311F480E3E8
:10BE200001C081E30E94155E16952196C830D105A8
:10BE300099F7DF91CF911F910F9108951F93CF93A1
:10BE4000DF93182F82958F70C4E5DEE1FE01E80FC5
:10BE5000F11DE4918E2F0E94155E1F70C10FD11D40
:10BE6000FE0184910E94155EDF91CF911F9108958C
:10BE70000F931F93082F843690F46AE00E940BC63C
:10BE8000182F805D0E94155E005D86EF9FEF189F62
:10BE9000102D1124812F800F0E94155E04C089E7A8
:10BEA0009EE10E944A5E1F910F910895EF92FF92CA
:10BEB0000F931F937C0123E0883E9207A0F564E670
:10BEC00070E00E9417C68B01862F805D0E94155E70
:10BED00084E690E09C01029FC001039F900D129F99
:10BEE000900D11248701081B190BC8016AE070E04E
:10BEF0000E9417C6F62EE72E862F805D0E94155EE3
:10BF00008F2D9E2D9C0153E0220F331F5A95E1F790
:10BF1000880F991F280F391F021B130B802F805D7C
:10BF20000E94155E04C085E79EE10E944A5E1F9153
:10BF30000F91FF90EF900895A19AA09A0895EAE1D9
:10BF4000FBE08FEF81939BE0E432F907D9F7808320
:10BF500008958FEF8093240B8CEF8093C90A089586
:10BF6000EAECFAE081938F5F9BE0EA31F907D1F7C1
:10BF70008FEF81939BE0E432F907D9F7808308952E
:10BF8000F8948FE084BBA998A89A9091640A292F0D
:10BF900022952F70822F8A95F1F7A99A9F70892F89
:10BFA0008A95F1F783B3A9982A95F1F7A99A9A95FA
:10BFB000F1F7A998A8989FEF94BB7894807808959A
:10BFC000CF93DF938091630A80FF05C00E94C05F1A
:10BFD000882309F071C02091250B822F86958695C4
:10BFE0008695C82FD0E0C65ED44F3881A22FB0E02E
:10BFF000FD01E770F070E959F14E9491892F832388
:10C0000051F18091240B821711F590959323988319
:10C01000A753B54F1196EC91982F9F5F9093250BE6
:10C02000903510F01092250B8091630A81FD08C0B5
:10C030009093240B943121F0983211F09C3319F431
:10C040008FEF8093240B8E2F0E94B65B35C0822F1A
:10C050000E94FC5D31C0822F8F5E86958695869505
:10C060008A3008F080E09AE00CC0915031F4880FDB
:10C07000880F880F8093250B1FC08F5F8A3009F4CB
:10C0800080E0E82FF0E0E65EF44FE081EE2369F314
:10C09000982F990F990F990F8E2F807F19F49C5F1D
:10C0A000E295E07F8E2F807C19F49E5FEE0FEE0FFD
:10C0B000E7FF9F5F9093250BDF91CF9108951F932A
:10C0C000CF93DF93EC01162F97FF08C08DE20E94FB
:10C0D000155E882799278C1B9D0B04C08BE20E945C
:10C0E000155ECE016091260B412F0E94125DDF91FB
:10C0F000CF911F9108958091700AE82FF0E083FF9F
:10C1000020C0E770F070EE0FFF1FEE5AF24F8081F3
:10C11000918125E08535920770F48091290B81503B
:10C120008093290B8F5F69F484E00E94296B8FE074
:10C130008093290B08958B5A9A4018F082E08093DF
:10C14000290B0895CF93DF939091C90A9F5F909335
:10C15000C90A9150973F31F1983F70F4943FE1F054
:10C16000953F20F4933F09F095C016C0953FA1F08C
:10C17000963F09F08FC012C09A3F59F19B3F30F4AF
:10C18000983F91F0993F09F085C021C09B3F19F17C
:10C190009C3F09F07FC05AC080E301C080E20E944A
:10C1A000A35D8DC088E210C08091630A84FF87C0C0
:10C1B0002091650A8FEF90E0821B9109F6E095953A
:10C1C0008795FA95E1F780680E94B85D78C08CE0A9
:10C1D000FBCF86E0F9CF0E94DE5D8FEF8093240BCA
:10C1E0001092260B8091630A83FF2DC06091650A2F
:10C1F00060932A0B60932B0BF8948091920B909193
:10C20000930BCCB5DDB5D093930BC093920BC817AD
:10C21000D90748F48091940B9091950B01969093D7
:10C22000950B8093940B7894CE010E94921D672FFA
:10C23000782F892F992770932E0B60932D0BD09315
:10C24000300BC0932F0B1092C90A39C02091240BD8
:10C250002F5F2093240B822F86958F3711F09093B8
:10C26000C90A20FF14C0E82FF0E080FF06C0EF707D
:10C27000F070EC5AF14E849107C082958F70E82FD0
:10C28000F0E0EC5AF14E84910E94B65B18C00E9417
:10C29000F85D15C09D3F98F08091260B8F5F8093CD
:10C2A000260B882319F09093C90A09C0EAE1FBE044
:10C2B0008FEF81939BE0E432F907D9F78083DF9118
:10C2C000CF910895CF93DF938093C90A1092250BE5
:10C2D0001092260B8091630A83FF2DC06091650A3E
:10C2E00060932A0B60932B0BF8948091920B9091A2
:10C2F000930BCCB5DDB5D093930BC093920BC817BD
:10C30000D90748F48091940B9091950B01969093E6
:10C31000950B8093940B7894CE010E94921D672F09
:10C32000782F892F992770932E0B60932D0BD09324
:10C33000300BC0932F0BEAECFAE080E281939BE094
:10C34000EA31F907D9F78FEF81939BE0E432F907DF
:10C35000D9F780839FB7F894A19AA09AA998A89832
:10C3600084B3806F84BB9FBFDF91CF91089589ED27
:10C370000E9462610895FC01108208951F93CF937B
:10C38000DF93EC01142F88818F3108F04BC0582FB8
:10C390005F5F58831FC0852F90E0FC01EE0FFF1FE9
:10C3A000E80FF91FEC0FFD1FB283A1830196DC019A
:10C3B000AA0FBB1FA80FB91FAC0FBD1FC901019663
:10C3C000FC01EE0FFF1FE80FF91FEC0FFD1F80812E
:10C3D0008C93542F513091F0452F4695242F30E007
:10C3E000F901EE0FFF1FE20FF31FEC0FFD1FA181FC
:10C3F000B281CB018A1B9B0B97FDCDCF852F90E09F
:10C40000FC01EE0FFF1FE80FF91FEC0FFD1F7283F9
:10C4100061830196FC01EE0FFF1FE80FF91FEC0F7F
:10C42000FD1F1083DF91CF911F910895EF92FF922E
:10C430000F931F93CF93DF93EC012881222309F4FC
:10C440007EC0E22EEA94E882EE2009F478C030E063
:10C45000F901EE0FFF1FE20FF31FE80FF91F8181B3
:10C4600092819D838C832F5F3F4FF901EE0FFF1F59
:10C47000E20FF31FEC0FFD1F80818E8351E0452FEB
:10C48000440FE41608F45BC0F42EF394EF14D8F0D4
:10C490008F2D90E0DC01AA0FBB1FA80FB91FAC0FB6
:10C4A000BD1F842F90E0FC01EE0FFF1FE80FF91F66
:10C4B000EC0FFD1F11968D919C9112972181328175
:10C4C000821B930B97FFF42E652F70E0DB01AA0F00
:10C4D000BB1FA60FB71FAC0FBD1F11960D911C916E
:10C4E00012974F2D50E0FA01EE0FFF1FE40FF51FDA
:10C4F000EC0FFD1F21813281C801821B930B97FD38
:10C500001EC012963C932E93119712830183CB0188
:10C510000196DC01AA0FBB1FA80FB91FAC0FBD1FEE
:10C520002C91CA010196FC01EE0FFF1FE80FF91FC5
:10C53000EC0FFD1F80818C9320835F2DA0CFDF91B6
:10C54000CF911F910F91FF90EF900895EF92FF927E
:10C550000F931F93CF93DF93EC017D836C834E8306
:10C56000E88051E0452F440FE41608F45BC0F42E38
:10C57000F394EF14D8F08F2D90E0DC01AA0FBB1FCD
:10C58000A80FB91FAC0FBD1F842F90E0FC01EE0F68
:10C59000FF1FE80FF91FEC0FFD1F11968D919C9165
:10C5A000129721813281821B930B97FFF42E652F06
:10C5B00070E0DB01AA0FBB1FA60FB71FAC0FBD1F9A
:10C5C00011960D911C9112974F2D50E0FA01EE0F2C
:10C5D000FF1FE40FF51FEC0FFD1F21813281C80101
:10C5E000821B930B97FD1EC012963C932E931197BE
:10C5F00012830183CB010196DC01AA0FBB1FA80F98
:10C60000B91FAC0FBD1F2C91CA010196FC01EE0FA2
:10C61000FF1FE80FF91FEC0FFD1F80818C93208313
:10C620005F2DA0CFDF91CF911F910F91FF90EF90E1
:10C63000089525B32F70962F9F78282B992331F0DA
:10C640006077262B25BB9698969A0895262B25BBB6
:10C65000809165008B7F8093650080916500846088
:10C660008093650008950F931F93382F20918F01B9
:10C67000222399F090918E01892F82958F708217D5
:10C6800048F4985890938E01809155018062809370
:10C69000550125C0995890938E01809155018F7D49
:10C6A00080935501E32FF0E0E851FE4F60898091BF
:10C6B0007A0A80FD02C000E801C000E03F3F79F047
:10C6C000162F1877802F612F0E94196380917A0AA4
:10C6D00081FF05C01051802F612F0E9419631F91A7
:10C6E0000F9108950F931F93982FE82FF0E0E851D2
:10C6F000FE4F608980917A0A80FD02C000E001C08F
:10C7000000E89F3F79F0162F1877802F612F0E9445
:10C71000196380917A0A81FF05C01051802F612F23
:10C720000E9419631F910F910895E82F20919E0197
:10C73000222391F08091910186FF0EC090918E018D
:10C74000892F82958F70821720F4985890938E01CC
:10C7500007C0995890938E018091520180FF06C0C6
:10C76000809155018062809355010895F0E0E85171
:10C77000FE4F90818091A201892B8093A2012BB35F
:10C78000892F809582238BBB8AB3982B9ABB0895FF
:10C7900080B5816880BD109289001092880014BC19
:10C7A0001DBC1CBC80B58F7780BD08959C01462FB1
:10C7B0008091920B9091930B6CB57DB57093930B18
:10C7C0006093920B6817790748F48091940B9091CD
:10C7D000950B01969093950B8093940B620F731FAA
:10C7E00081E39BE050E00E94BE6108959C01462FCA
:10C7F0008091920B9091930B6CB57DB57093930BD8
:10C800006093920B6817790748F48091940B90918C
:10C81000950B01969093950B8093940B620F731F69
:10C8200080914E01882331F081E39BE050E00E942B
:10C83000BE61089581E080934E0181E39BE050E06A
:10C840000E94A66208959C01462F8091920B9091C0
:10C85000930B6CB57DB57093930B6093920B681737
:10C86000790748F48091940B9091950B01969093E1
:10C87000950B8093940B620F731F81E39BE050E054
:10C880000E94A66208959C01462F81E39BE0B901B6
:10C8900050E00E94A66208959C01462F80914E01AF
:10C8A000882339F081E39BE0B90150E00E94BE612A
:10C8B000089581E080934E0181E39BE0B90150E04F
:10C8C0000E94A6620895AF92BF92CF92DF92EF923C
:10C8D000FF920F931F93CF93DF930091310B8CEF57
:10C8E000A82E8FEFB82E27C01091370B812F8F7095
:10C8F000880F90E08458914EFC0125913491812F4E
:10C9000082958F70F90109950091310B002399F000
:10C910008091370B181779F48091350B9091360B75
:10C92000C817D90741F48091BF0B85FD04C081E38E
:10C930009BE00E9416628091920B9091930B4CB5F4
:10C940005DB55093930B4093920B4817590748F4E9
:10C950008091940B9091950B01969093950B8093F9
:10C96000940B9A012F5F3F4F002349F0C091350B84
:10C97000D091360BCE01821B930B97FDB5CF8091E2
:10C98000960B381741F03093960B809139058062F1
:10C9900080933905D0CF232F2F5F002349F0F22E4B
:10C9A000EE24C7018860BE01681B790B77FD04C0C7
:10C9B000D22ECC24E601C5602CB53DB53093930B47
:10C9C0002093920B2417350748F48091940B909193
:10C9D000950B01969093950B8093940BC501821B48
:10C9E000930B8C0F9D1F97FDA6CFD0937900C0931A
:10C9F000780081E080937C00DF91CF911F910F91AF
:10CA0000FF90EF90DF90CF90BF90AF90089583E0BC
:10CA10008EBDEDE7F0E080818160808310924E0151
:10CA200081E39BE00E94BB61109289001092880014
:10CA30001DBC1CBC1092930B1092920B0E9463645D
:10CA400008951F920F920FB60F920BB60F921124FA
:10CA50002F933F934F935F936F937F938F939F9306
:10CA6000AF93BF93EF93FF930E946364FF91EF91A5
:10CA7000BF91AF919F918F917F916F915F914F91F6
:10CA80003F912F910F900BBE0F900FBE0F901F90F4
:10CA9000189581E39BE00E9416620895833021F18E
:10CAA000843028F4813091F08230B8F408C08530A9
:10CAB00049F1853000F1863009F0D4C02BC02091B7
:10CAC0009201309193014091A20A2AC020919401D1
:10CAD0003091950140919F0923C02091C30130916D
:10CAE000C40140915D091CC02091B9013091BA0187
:10CAF0004091A40A15C02091C3013091C401409116
:10CB00005D0906C02091B9013091BA014091A40A93
:10CB1000405F06C0209117053091180540913D09EE
:10CB20008091920B9091930B821B930B499708F085
:10CB300099C0542F5F70242F207F523009F472C0A7
:10CB4000533030F4552359F0513009F08BC028C0D0
:10CB5000563009F46EC0573009F084C06EC0822F81
:10CB600090E08077907044E0959587954A95E1F73D
:10CB7000E82F27FF03C00E94956374C0F0E0E851DE
:10CB8000FE4F90812091A201892F8095822380936E
:10CB9000A2018BB3892B8BBB8AB3982B9ABB62C043
:10CBA000822F90E08077907034E0959587953A9544
:10CBB000E1F7382F8230E8F427FF0DC0209165009F
:10CBC00081E090E002C0880F991F3A95E2F7282B88
:10CBD0002093650047C02091650081E090E002C08D
:10CBE000880F991F3A95E2F780958223809365001C
:10CBF00039C027FF0BC028B381E090E002C0880F46
:10CC0000991F3A95E2F7282B28BB2CC028B381E066
:10CC100090E002C0880F991F3A95E2F78095822331
:10CC200088BB20C08091520181FD1CC0E5E6F0E088
:10CC300006C08091520182FD15C0E2E3F0E085B3A9
:10CC40008F70282B25BB908121E030E002C0220F9D
:10CC5000331F5A95E2F7822F809598239083808125
:10CC6000822B808381E39BE00E941662089580E21C
:10CC700080937C00EDE7F0E080818062808381E337
:10CC80009BE00E941662089580E286BF87B78062AB
:10CC900087BF81E39BE00E941662089581E39BE0D9
:10CCA0000E941662089581E39BE00E941662089537
:10CCB00080E00E94726381E39BE00E941662089507
:10CCC000AB9880916B0D805F80936B0D81E39BE04F
:10CCD0000E9416620895982F6091690D70916A0DF7
:10CCE0008FEF6F3F7807B1F0AB9A80916B0D8F702B
:10CCF000806180936B0D9093660D8091920B909163
:10CD0000930B680F791F81E39BE04DE050E00E9498
:10CD1000A662089581E39BE00E9416620895813027
:10CD200009F45FC0813020F0823009F0ACC07EC0D1
:10CD3000E091B908F091BA08309709F4A4C0809145
:10CD4000920B9091930B4CB55DB55093930B409320
:10CD5000920B4817590748F48091940B9091950BCA
:10CD600001969093950B8093940B8091A2018095EE
:10CD70009091E8018923C9F08091520180FF06C09B
:10CD8000809155018062809355010FC020919001E0
:10CD90008091A201822B8093A2019BB3822F809568
:10CDA00089238BBB8AB3822B8ABBBA016E0F7F1F8C
:10CDB0007093BC086093BB0820918A0130918B016D
:10CDC000C90143968E179F0710F04BE204C0B901CA
:10CDD000640F751F4BE181E39BE050E00E94BE6150
:10CDE00052C08091A2019091E801892309F44BC0BF
:10CDF0008091520180FF06C080915501806280932E
:10CE0000550109C0809190019BB3809598239BBBED
:10CE10009AB389238ABB6091BB087091BC0881E3F7
:10CE20009BE04BE250E00E94A66208954091BB084F
:10CE30005091BC088091920B9091930B2CB53DB50D
:10CE40003093930B2093920B2817390748F4809165
:10CE5000940B9091950B01969093950B8093940B66
:10CE6000421B530B57FF0FC0209190019091A201DC
:10CE7000822F809589238093A2018BB3822B8BBB59
:10CE80008AB3822B8ABB81E39BE00E9416620895DD
:10CE9000682FE82FF0E0EE0FFF1FEE0FFF1FE754A3
:10CEA000F74F428153818091920B9091930B2CB557
:10CEB0003DB53093930B2093920B2817390748F414
:10CEC0008091940B9091950B01969093950B809384
:10CED000940B421B530B57FF12C0E62FF0E0E851B2
:10CEE000FE4F90812091A201892F8095822380930B
:10CEF000A2018BB3892B8BBB8AB3982B9ABB81E39E
:10CF00009BE00E9416620895482FA82FB0E0FD0113
:10CF1000E851FE4F90818091A201892329F481E399
:10CF20009BE00E94166208958091520180FF06C026
:10CF30008091550180628093550107C08BB3909515
:10CF400089238BBB8AB398239ABBAA0FBB1FAA0F56
:10CF5000BB1FA554B74F6D917C914295407F465FB2
:10CF600081E39BE050E00E94A6620895DF92EF9279
:10CF7000FF920F931F93CF93DF93D82EC82FD0E04B
:10CF8000CC0FDD1FCC0FDD1FC754D74FE880F980D1
:10CF9000E114F10429F481E39BE00E94166242C08F
:10CFA0008091920B9091930B0CB51DB51093930B40
:10CFB0000093920B0817190748F48091940B9091F5
:10CFC000950B01969093950B8093940B8091A20101
:10CFD000ED2DF0E0E851FE4F80959081892321F0FE
:10CFE0008D2D0E94956381E04D2D4295407F9801E3
:10CFF0002E0D3F1D3B832A8360918A0170918B0126
:10D00000882349F0CB0143968E159F0520F4600FCD
:10D01000711F475F02C0465FB90181E39BE050E0AA
:10D020000E94A662DF91CF911F910F91FF90EF9028
:10D03000DF90089580914E01882329F481E39BE0DD
:10D040000E941662089510924E0108958091310B4E
:10D050008730A8F40E94C0C5BC018EE36138780710
:10D0600038F071708091920B9091930B680F791F3B
:10D0700081E39BE046E050E00E94A662089581E3D0
:10D080009BE00E94166208951F93CF93DF93182FA1
:10D0900080917A0A85FF04C0812F0E94726309C0C3
:10D0A00083B1806383B981E880938B00812F0E94D4
:10D0B00033638091C00B86FF1CC08091920B9091CE
:10D0C000930B4CB55DB55093930B4093920B48175F
:10D0D000590748F48091940B9091950B0196909389
:10D0E000950B8093940B83EF99E266E028E00E9411
:10D0F0005E248091F20981FF03C088E00E941DA593
:10D10000C091940BD091950BA091920BB091930B81
:10D110008B2F9C2F8456904090936C0180936B01D1
:10D12000809177018823D9F08091700D811729F0C3
:10D130008091720D8F5F8093720D80916B0D82FFD5
:10D140000EC08091670D9091680DA80FB91F1295C0
:10D15000107F145F81E39BE0BD01412F52C080919D
:10D160007701E12FF0E0E959F14EE491E095E823F1
:10D17000E093770140917501242F30E0F901E851E7
:10D18000FE4F8085803809F040C090917701B90149
:10D190006959714EFB018491892309F43AC08B2FA0
:10D1A0009C2F2091880130918901830F911D9093CC
:10D1B0006C0180936B0180917B0AE42FE1508E1704
:10D1C00008F4E82FE09375018091540187FF06C0B1
:10D1D00080919D01F0E0E55EFA4F808380917701B8
:10D1E000FB01949190959823909377014295407F0D
:10D1F00060918801709189016A0F7B1F4F5F81E305
:10D200009BE050E00E94A66204C081E39BE00E9484
:10D210001662DF91CF911F9108951F93182F80916F
:10D220007A0A85FF04C0812F0E94336312C0812FC8
:10D230000E94726384E690E0909383008093820062
:10D240008BE990E090938500809384008DEA809331
:10D250008B00A091920BB091930B8091940B9091C5
:10D26000950B9C018B2F922F20917A0130917B019D
:10D27000830F911D90936C0180936B018091700DD1
:10D28000811729F08091710D8F5F8093710DE0916E
:10D290007601F0E0E851FE4F8085803819F5409125
:10D2A000760190917B0A842F8150981708F4892F7A
:10D2B0008093760180917701E42FF0E0E959F14EF7
:10D2C000E491E82BE09377016091880170918901E6
:10D2D0006A0F7B1F4295407F81E39BE050E00E94F4
:10D2E000A66225C081E39BE00E94166280916F0ACE
:10D2F0008430E8F420916D0A80916B0A81FF02C0AE
:10D30000922F12C0203211F494E20EC084FF03C0A9
:10D31000922F9F5F02C0922F9E5F80916C0A84FDC6
:10D3200002C0243008F4990F892F0E94167B1F91A8
:10D33000089521B180915101822782FF09C0809117
:10D340005001853000F190E08D33F0F491E01CC085
:10D3500022FF07C01092500190E020935101892FC5
:10D360000895809150018F3FD1F08F5F80935001DD
:10D37000883CA9F480914F0180FD11C081608093A9
:10D380004F0192E0EACF90E01092500180914F015E
:10D390008E7F80934F0120935101892F089590E053
:10D3A00020935101892F089591B1809151018927CE
:10D3B00082FF19C080915001853088F18D3378F556
:10D3C0001092500180914F018E7F80934F01909376
:10D3D00051018091B40B8F5F8093B40B833048F17F
:10D3E0001092B40B089592FF05C0109250019093D3
:10D3F00051010895809150018F3FC9F38F5F809351
:10D400005001883CA1F780914F0180FDF0CF8160F1
:10D4100080934F01909351010E94E9430895109227
:10D42000500180914F018E7F80934F019093510165
:10D43000089508958DB78093EA0D8EB78093EB0D14
:10D440008CE293E09093B60B8093B50B1092B80BDF
:10D450008FEF8093BA0B089540E050E008C02FEFA3
:10D460003FEF420F531F21503040D9F701970097EB
:10D47000B1F7CA010895882311F48DE00895813031
:10D4800011F48AE00895282F2250322F36953695D0
:10D490003695E0913B08F0E053E0EE0FFF1F5A9500
:10D4A000E1F7E05CF74F832F90E0880F991F019020
:10D4B000F081E02DE80FF91F9081818127702330E2
:10D4C000B1F0243028F4213071F0223070F409C01A
:10D4D0002530A1F0253070F0263059F0273089F43E
:10D4E0000CC080E2089584E50895832F07C08DE382
:10D4F0000895892F0E945E5B0895892F0E94675BC3
:10D50000089585E60895882311F48DE0089581300B
:10D5100011F48AE00895982F9250292F2695269588
:10D52000269580913B08A82FB0E0FD0173E0EE0F37
:10D53000FF1F7A95E1F7E05CF74F0190F081E02D55
:10D54000E20FF11DE081892F8770833081F08430F4
:10D5500028F4813081F08230C0F40BC08530C9F0EE
:10D560008530A8F08630B9F08730E9F418C08DE333
:10D57000089580E2089563E0AA0FBB1F6A95E1F762
:10D58000A45CB74F16968C910895822F09C080E055
:10D5900003C080E005C08E2F0E945E5B08958E2F31
:10D5A0000E94675B089585E608958091BA0B80FF1D
:10D5B00005C08BE79BE568E50E9431248091BA0B9A
:10D5C00082FF07C083E89AE66CE441E35BE00E94D7
:10D5D000BD2408959091B80B992391F08091B90BD7
:10D5E0008F5F8093B90B891728F01092B90B0E94B6
:10D5F000D56A08959F3F21F40E94D56A1092B80B16
:10D6000008950895089508950895582F742F422F6E
:10D61000281788F4282F30E0842F90E0871B910989
:10D62000860F911D281739071CF4852F841B089538
:10D63000862F871B089580E008959FEF9093C60B77
:10D640008093C70B7093CA0B6093C90B1092C80BE1
:10D650000895582F4091C50B242F30E08BE290E0C5
:10D66000851B91098217930728F0252F240F2093FB
:10D67000C50B089520E02093C50B08959091C50B2C
:10D68000981718F0981B9093C50B089594E1899F03
:10D69000802D11240E940F5E08950F931F93809197
:10D6A000C60B8F3F09F455C0082F02950F70182F35
:10D6B0001F708091C50B800F8C32F0F08EE190E2EC
:10D6C000FC012591349121153105F9F0812F90E06D
:10D6D000880F991FFC01E20FF31F85919491009729
:10D6E000E1F0FC0109951F5F0295007F100F109378
:10D6F000C60B1F910F910895E82FF0E0EE0FFF1F6A
:10D700008EE190E2E80FF91FDCCFFC012591349106
:10D7100000E010E080E090E0DDCF0330E8F4902FEF
:10D720009F5F84E1989F90011124022F192F129579
:10D73000107F8091260B90E08217930711F00E94D2
:10D74000CA5E802F0E940F5E1093C60B1F910F912F
:10D75000089500E010E0ADCF20E030E000E010E000
:10D76000E8CF0E94CA5E0895FF920F931F93E62FA1
:10D77000E81BF0E0EE0FFF1FE758FA4F25913491B8
:10D7800050E0481B5109440F551FCA01880F991FCB
:10D79000880F991F880F991F480F591F329522959E
:10D7A0002F7023273F702327249FC001259F900DB2
:10D7B000349F900D1124929582958F7089279F70C8
:10D7C0008927092FF92E10E008C01F1591F08DE26E
:10D7D0000E94155E1F5F123141F01017B1F78AE207
:10D7E0000E94155E1F5F1231C1F71F910F91FF90CC
:10D7F00008958EE50E94155EEDCF0F931F93681B71
:10D80000E62FF0E0EE0FFF1FE758FA4F2591349115
:10D8100050E0481B5109440F551FCA01880F991F3A
:10D82000880F991F880F991F480F591F329522950D
:10D830002F7023273F702327429FC001439F900DE5
:10D84000529F900D1124929582958F7089279F7019
:10D850008927092F10E006C08DE20E94155E1F5F28
:10D86000123141F01017C1F78AE20E94155E1F5F66
:10D870001231C1F71F910F9108950F931F93681BE9
:10D88000E62FF0E0EE0FFF1FE758FA4F2591349195
:10D8900050E0481B5109440F551FCA01880F991FBA
:10D8A000880F991F880F991F480F591F329522958D
:10D8B0002F7023273F702327429FC001439F900D65
:10D8C000529F900D1124929582958F7089279F7099
:10D8D0008927092F10E006C083E20E94155E1F5FB2
:10D8E000123141F00117C0F78FE50E94155E1F5FEE
:10D8F0001231C1F71F910F9108958091550182FD5A
:10D9000010C08091540181FD10C08091A80B87FF49
:10D9100004C080916B0A81FF0CC080E20E94155EFA
:10D92000089585E40E94155E089582E40E94155EC4
:10D93000089583E50E94155E08958091530181FD4D
:10D940002AC08091540185FD22C08091540184FD3C
:10D9500026C08091530182FD26C08091540182FD32
:10D9600024C08091530187FD24C08091530184FD20
:10D970001EC08091530185FD1EC08091540183FD1E
:10D980001CC08091530180FD1AC08FE501C081E465
:10D990000E94155E089583E40E94155E089583E653
:10D9A0000E94155E089587E7F3CF8FE4F1CF81E6FB
:10D9B000EFCF89E6EDCF84E6EBCF8FE6E9CF80E2CB
:10D9C000E7CF80E20E94155E089580E20E94155E16
:10D9D00080916A0C81FF12C087E50E94155E8091DC
:10D9E0006A0C82FF12C080E50E94155E80916A0C6D
:10D9F00084FD12C080E20E94155E089580E20E94BC
:10DA0000155E80916A0C82FDEECF80E20E94155E69
:10DA100080916A0C84FFEECF86E40E94155E089523
:10DA200083E60E94155E80E20E94155E089587E8F5
:10DA300090E20E944A5E089580E990E20E944A5E68
:10DA400008958AE990E20E944A5E089585EA90E28C
:10DA50000E944A5E089580916A0C80FD05C08CEC9E
:10DA600090E20E944A5E089580ED90E20E944A5E34
:10DA700008958CEE90E20E944A5E089583EF90E252
:10DA80000E944A5E089588EF90E20E944A5E0895DF
:10DA90008CEF90E20E944A5E08958091530187FDC9
:10DAA00005C086E091E20E944A5E08958EE091E210
:10DAB0000E944A5E089586E191E20E944A5E0895BE
:10DAC0008BE191E20E944A5E089581E291E20E9418
:10DAD0004A5E08958BE291E20E944A5E08958FE2C9
:10DAE00091E20E944A5E089584E391E20E944A5EB8
:10DAF00008958091F30981FD05C085E491E20E94BB
:10DB00004A5E08958BE491E20E944A5E089584E59E
:10DB100091E20E944A5E089589E591E20E944A5E80
:10DB200008958EE591E20E944A5E089580E691E2B2
:10DB30000E944A5E089586E691E20E944A5E089538
:10DB400088E691E20E944A5E08958DE691E20E9485
:10DB50004A5E08958DE691E20E944A5E08958DE640
:10DB600091E20E944A5E089583E791E20E944A5E34
:10DB700008950F931F9303E711E2C8010E944A5EC4
:10DB8000C8010E944A5E1F910F91089586E791E2B5
:10DB90000E944A5E08958BE791E20E944A5E0895D2
:10DBA00080E20E94155E86E991E20E944A5E8FE85B
:10DBB00091E20E944A5E089580E20E94155E80E232
:10DBC0000E94155E80E20E94155E80E20E94155E52
:10DBD00080E20E94155E81EA91E20E944A5E089509
:10DBE000CF92DF92EF92FF920F931F93CF93DF9329
:10DBF0007C01EB01142FD22EC02E222329F500E048
:10DC0000123048F08981F70191917F01891B0E94B0
:10DC10001E5F22961250112349F4DF91CF911F917C
:10DC20000F91FF90EF90DF90CF9008950F5F01303C
:10DC300039F48CE30E94155E1150123008F7EDCFD5
:10DC40000023E1F08C2DF6CF00E0123048F08981FE
:10DC5000F70191917F01891B0E941E5F229612504D
:10DC60001123D9F20F5F0D1539F08C2D0E94155E2E
:10DC70001150123050F7D1CF8EE3F8CF8EE3DACFC8
:10DC8000EF92FF920F931F93CF93DF93EC01162F28
:10DC9000F42EE22E4423F1F400E0123020F08991BA
:10DCA0000E941E5F1250112339F4DF91CF911F9112
:10DCB0000F91FF90EF9008950F5F013039F48CE3DE
:10DCC0000E94155E1150123040F7EFCF0023B9F0DB
:10DCD0008E2DF6CF00E0123020F089910E941E5F59
:10DCE0001250112311F30F5F0F1539F08E2D0E9482
:10DCF000155E1150123078F7D8CF8EE3F8CF8EE34F
:10DD0000DFCF85EB90E20E944A5E8091760D0E9403
:10DD10001E5F8091750D0E941E5F80EB90E20E9455
:10DD20004A5E8091770D0E941E5F80E20E94155E20
:10DD30008091780D0E941E5F80E20E94155E8091A6
:10DD4000720D0E941E5F089588EB90E20E944A5E69
:10DD50008091740D0E941E5F8091730D0E941E5F62
:10DD600080E20E94155E8091650D0E941E5F80E238
:10DD70000E94155E80916B0D0E941E5F08958FEBCF
:10DD800090E20E944A5E8091680D0E941E5F809121
:10DD9000670D0E941E5F8BEB90E20E944A5E8091AD
:10DDA0006A0D0E941E5F8091690D0E941E5F08959A
:10DDB00080E20E94155E80916F0C0E941E5F809130
:10DDC0006E0C0E941E5F80E20E94155E8091720CB4
:10DDD0000E941E5F089580916D0C0E941E5F8091CD
:10DDE0006C0C0E941E5F80E20E94155E8091760C92
:10DDF0000E941E5F8CE20E94155E089580916D0C5A
:10DE00000E941E5F80916C0C0E941E5F80E20E9447
:10DE1000155E80916F0C0E941E5F80916E0C0E94B7
:10DE20001E5F80E20E94155E8091760C0E941E5F4C
:10DE3000089584ED90E20E944A5E8091720C0E94E7
:10DE40001E5F08958AED90E20E944A5E8091760CF2
:10DE50000E941E5F089580EE90E20E944A5E8091CB
:10DE60006F0C0E941E5F80916E0C0E941E5F0895D1
:10DE700088EE90E20E944A5E80916D0C0E941E5FC7
:10DE800080916C0C0E941E5F089580E70E94155ED1
:10DE90008091A80B0E941E5F08951F931091560158
:10DEA00087E50E94155E812F90E08F709070892B1E
:10DEB00029F480E00E941E5F1F910895812F8295B2
:10DEC0008F700E941E5F1F91089581E60E94155E6B
:10DED0008091A1089091A208969587950E941E5F57
:10DEE0008DE20E94155E08958DE60E94155E2091D8
:10DEF0005801309159018091660A8F70823091F0FB
:10DF000083E02C3F380790F4369527953695279572
:10DF1000822F0E941E5F8DE20E94155E80E20E94A9
:10DF2000155E089587E0283F380710F08FEFF1CF96
:10DF3000369527953695279536952795822FE9CFE3
:10DF400082E70E94155E809165010E941E5F8DE24E
:10DF50000E94155E80E20E94155E089580E00E9496
:10DF60001E5F80E00E941E5F089580E20E94155EA1
:10DF7000809191010E941E5F08958091B50A0E94D0
:10DF8000675B0E94155E82E50E94155EE091B50A0E
:10DF9000EE2309F045C08FEF0E941E5F80E20E94D1
:10DFA000155E8091B30A0E94675B0E94155E8BE448
:10DFB0000E94155E8091B30A882309F44FC0E09156
:10DFC000B20AF0E0E25EFC4F9081E82FF0E0E25E02
:10DFD000FC4F608140915801509159018091660A2F
:10DFE0008F70823071F183E04C3F5807A8F5569549
:10DFF000479556954795892F0E942E1E0E941E5FB9
:10E0000080E20E94155E8091B8080E94675B0E94C2
:10E01000155E84E50E94155E8AEA0E941E5F0895DF
:10E0200040916501A091B40AB0E0A25FBC4FF0E05E
:10E03000E25FFC4F8C9160810E942E1E0E941E5F49
:10E04000ADCF87E0483F580738F456954795569529
:10E05000479556954795CFCF4FEFCDCF8FEF0E9485
:10E060001E5FCECFCF92DF92EF92FF920F931F935E
:10E07000DF93CF9300D0CDB7DEB77C01DC011696DD
:10E080000C9116970295007F17968C91082BC02E45
:10E09000DD249601220F331F21593B4EF901859152
:10E0A00094919A838983892B09F04EC010E0225005
:10E0B00030401F5FF901859194910097C1F39A83D5
:10E0C000898384E890E20E944A5E802F811B0E942F
:10E0D0001E5F8FE20E94155E812F0E94675B0E9487
:10E0E000155E8DE30E94155ED7011396ED91FC91AC
:10E0F0001497EC0DFD1D80810E941E5F80E20E943E
:10E10000155E8091BF0B87FD12C0CE01019666E4BB
:10E110000E94585E0E946C5E0F900F90CF91DF912D
:10E120001F910F91FF90EF90DF90CF900895CE0157
:10E13000019662E30E94585E8BE30E94985E0E9403
:10E14000BD6F0E946C5EE8CF10E0BBCF80915E0196
:10E1500090915F0127E28031920710F080E090E01B
:10E160006091260B42E00E94125D089580915C014F
:10E1700090915D0127E28031920710F080E090E0FD
:10E180006091260B42E00E94125D089585E990E2BD
:10E190000E944A5E80915801909159016091260B2E
:10E1A00041E00E94125D0895809131059091320501
:10E1B0009695879596958795969587956091260B68
:10E1C00041E00E94125D0895CF93DF938BEA90E2C5
:10E1D0000E944A5E2091730D3091740D8091750DEF
:10E1E0009091760D8217930778F0EC01C21BD30B48
:10E1F0008DE20E94155ECE016091260B41E00E94E7
:10E20000125DDF91CF910895E901C81BD90B8BE214
:10E210000E94155EF0CFCF93DF93C0917301D09130
:10E220007401D695C795D695C795C034D10570F4BD
:10E230008DE20E94155E80E48C1B90E06091260BBD
:10E2400040E00E94125DDF91CF9108958BE20E9421
:10E25000155E9E012054822FF0CFCF93DF93C091A3
:10E26000C20AD091C30AD7FD0DC08BE20E94155E91
:10E270008C2F90E06091260B41E00E94125DDF91AF
:10E28000CF9108958DE20E94155E9E012195822F07
:10E29000F0CF84E60E94155E8091C70A90E06091FD
:10E2A000260B40E00E94125D08958091B70A90E02D
:10E2B0006091260B41E00E94125D089580E20E9469
:10E2C000155E8091BE0A90E06091260B41E00E94AD
:10E2D000125D0895809160018F3FC1F080916001CF
:10E2E00029E1829FC00111240024880F991F001C7E
:10E2F000880F991F001C892F902D6091260B40E0FC
:10E300000E94125D85E20E94155E089587E291E207
:10E310000E944A5E08958091600190E06091260B12
:10E3200041E00E94125D0895809158019091590139
:10E3300096958795969587956091260B41E00E946A
:10E34000125D08950F931F93182F8436D8F0082F6D
:10E350000456043668F480E20E94155E802F90E037
:10E360006091260B40E00E94125D1F910F9108956D
:10E37000802F90E06091260B41E00E94125D1F917A
:10E380000F9108958DE20E94155E04E6011BE6CF11
:10E39000EF92FF92CF93DF93C0916701D091680114
:10E3A00087E2C031D807A8F08EE30E94155E7E0197
:10E3B0008F2D8695869590E06091260B40E00E9417
:10E3C000125D8BE60E94155EDF91CF91FF90EF907A
:10E3D0000895CE016091260B42E00E94125DDF910C
:10E3E000CF91FF90EF900895409160018CEB95E004
:10E3F00068E00E9441200E941E5F89E60E94155E2F
:10E40000809198010E941E5F0895CF92DF92EF9253
:10E41000FF920F931F936C01937064E60E94921D0C
:10E420007B018C018D2D8695869590E06091260B61
:10E4300040E00E94125D8EE20E94155EFAE01695A1
:10E440000795F794E794FA95D1F78E2D90E06091B7
:10E45000260B40E00E94125D1F910F91FF90EF90FC
:10E46000DF90CF90089580917A0190917B0166E6CC
:10E470000E94921DDC01CB01892F9A2FAB2FBB2765
:10E480006091260B41E00E94125D08958091B908C9
:10E490009091BA0868E30E94921D20916701309123
:10E4A000680140E050E00E94ECC5DC01CB018B2FFD
:10E4B0009927AA27BB276091260B41E00E94125D95
:10E4C00085E20E94155E08958091B9089091BA087E
:10E4D00066E60E94921DDC01CB01892F9A2FAB2F9B
:10E4E000BB276091260B42E00E94125D0895809147
:10E4F000A1089091A20864E60E94921DDC01CB0164
:10E50000892F9A2FAB2FBB2790E06091260B41E01B
:10E510000E94125D089589E60E94155E8091B80AF6
:10E520009091B90A62E00E945F6008950F931F9373
:10E5300080916701909168010091BE0A2AE0029FD4
:10E5400080011124081B190B85E60E94155EC80185
:10E5500062E00E945F601F910F91089580E26CE17C
:10E560000E94ED5B08951F93943600F5492F50E00B
:10E5700090709C01220F331F220F331F220F331F75
:10E58000880F991F280F391F132F105DCA01609142
:10E59000260B40E00E94125D8EE20E94155E812FE4
:10E5A0006091260B0E94ED5B1F91089543E650E0B9
:10E5B00019E3ECCF1F93CF93DF939C01A0E0B0E071
:10E5C000AC01BD0152956295729540EF7627742398
:10E5D0007627652764236527CB01182F8A30A8F09A
:10E5E00099E3C3E6D0E0892F6091260B0E94ED5B92
:10E5F0008EE20E94155ECE016091260B40E00E94E3
:10E60000125DDF91CF911F910895C9019F7064E65B
:10E610000E94921D9B01AC0132954295529520EFCC
:10E62000542752235427432742234327CA01912FBB
:10E63000905DC82FD0E0D7CFCF93DF93C091580122
:10E64000D0915901D695C795D695C795C636D105AF
:10E6500028F58DE20E94155E85E690E08C1B9D0BEF
:10E6600024E630E0AC01429FC001439F900D529FD1
:10E67000900D112463E00E94921DDC01CB01EAE0C1
:10E68000B695A79597958795EA95D1F76091260B52
:10E6900040E00E94125DDF91CF910895C556D040B1
:10E6A0008EE0BE010E94BD1E6091260B41E00E94DB
:10E6B000125DDF91CF9108958DE890E20E944A5E4D
:10E6C00080915C0190915D0127E28031920710F00A
:10E6D00080E090E06091260B42E00E94125D089578
:10E6E0008091240A85FF2EC08091210890912208F4
:10E6F000969587959695879596958795880F8436F4
:10E7000008F083E690E06091260B40E00E94125DE5
:10E7100080E20E94155E8091A1089091A20864E6B3
:10E720000E94921DDC01CB01892F9A2FAB2FBB27B2
:10E7300090E06091260B41E00E94125D80E20E9411
:10E74000155E089580911508909116089695879505
:10E750009695879596958795D1CF89E391E20E940A
:10E760004A5E8091A1089091A20864E60E94921DE1
:10E77000DC01CB01892F9A2FAB2FBB2790E0609152
:10E78000260B41E00E94125D08958FE391E20E9402
:10E790004A5E8091A1089091A20864E60E94921DB1
:10E7A000DC01CB01892F9A2FAB2FBB2790E0609122
:10E7B000260B41E00E94125D08950F931F938CE792
:10E7C0000E94155E8091580190915901E1E9F6E0AF
:10E7D00045915491969587959695879596958795A9
:10E7E00090E00A97880F991F9C01220F331F220F78
:10E7F000331F220F331F820F931F529542954F7084
:10E8000045275F7045279C01249FC001259F900DDF
:10E81000349F900D1124929582958F7089279F7057
:10E820008927092F10E006C083E20E94155E1F5F52
:10E83000123141F00117C0F78FE50E94155E1F5F8E
:10E840001231C1F78CE70E94155E1F910F91089558
:10E850000F931F93009157018EE1089F80011124AF
:10E86000812F90E06091260B40E00E94125D8EE2C5
:10E870000E94155E1070C801880F991F880F991F9C
:10E88000880F991F000F111F800F911F892F805D26
:10E890006091260B0E94ED5B86E50E94155E1F913C
:10E8A0000F9108951F93CF93DF9366E40E94921D0A
:10E8B000672F782F892F9927CB01A0E0B0E09C012A
:10E8C000AD0132954295529520EF5427522354279B
:10E8D000432742234327CA01182F8A30A8F099E31F
:10E8E000C3E6D0E0892F6091260B0E94ED5B8EE29B
:10E8F0000E94155ECE016091260B40E00E94125DE1
:10E90000DF91CF911F910895CB019F7064E60E9423
:10E91000921D9B01AC0132954295529520EF5427F0
:10E9200052235427432742234327CA01912F905D46
:10E93000C82FD0E0D7CF0F931F93CF93DF93C09111
:10E94000800CD091810C8CE70E94155E8091800C28
:10E950009091810C8F5F9F4FF1F58DE20E94155EC3
:10E960008DE20E94155E8DE20E94155E8DE20E948E
:10E97000155E8DE20E94155E8DE20E94155E8DE2AD
:10E980000E94155E8DE20E94155E8FE30E94155E67
:10E990008FE30E94155E8DE20E94155E8DE20E945B
:10E9A000155E8DE20E94155E8DE20E94155E8DE27D
:10E9B0000E94155E8DE20E94155E8DE20E94155E3A
:10E9C0008DE20E94155E8CE70E94155EDF91CF916B
:10E9D0001F910F910895E9EDF5E045915491CC0F09
:10E9E000CD2FCC1FDD0BD1958C2F90E08D55904015
:10E9F000880F991F9C01220F331F220F331F220FF4
:10EA0000331F820F931F529542954F7045275F70B9
:10EA100045279C01249FC001259F900D349F900D98
:10EA20001124929582958F7089279F708927092FCD
:10EA300010E007C083E20E94155E1F5F123109F4E7
:10EA4000C2CF0117B8F78FE50E94155EF6CFDF92AF
:10EA5000EF92FF920F931F93CF93DF93F62EE42E46
:10EA6000890194E1899F802D11240E940F5ECF2D92
:10EA7000D0E0FE01E25EFC4F80810E941E5F8AE3CF
:10EA80000E94155EF80186818F1509F450C0DD24BF
:10EA9000DA948091B30A8F1509F446C080E2F82E0B
:10EAA000F8018181843601F1C295D295D07FDC27AF
:10EAB000C07FDC27EC0EC381D481CE0DD11DDD20BB
:10EAC000D9F400E011E1123020F089910E941E5F1C
:10EAD0001250112349F00F5F013011F58CE30E94B1
:10EAE000155E1150123078F7DF91CF911F910F9181
:10EAF000FF90EF90DF90089500E011E1123020F0D8
:10EB000089910E941E5F1250112371F30F5FD0167E
:10EB100091F08F2D0E94155E1150123078F7E4CFDE
:10EB2000002359F08F2DDBCFBDE2FB2EB9CFF801CA
:10EB3000D780DE18AECF8EE3EDCF8EE3D0CF0F932C
:10EB40001F9310915A01143608F1012F0456043610
:10EB500080F480E20E94155E802F90E06091260B89
:10EB600040E00E94125D83E40E94155E1F910F91A8
:10EB70000895802F90E06091260B41E00E94125D85
:10EB800083E40E94155E1F910F9108958DE20E940B
:10EB9000155E04E6011BE0CF0F931F9310915B01FC
:10EBA0001436D8F0012F0456043668F480E20E942F
:10EBB000155E802F90E06091260B40E00E94125D70
:10EBC0001F910F910895802F90E06091260B41E0F6
:10EBD0000E94125D1F910F9108958DE20E94155EB3
:10EBE00004E6011BE6CF1F938091850C9091860C63
:10EBF000009731F48FE491E20E944A5E1F910895DC
:10EC00009695879563E30E94921D672F782F892F31
:10EC10009927743608F5472F50E0CB0190709C017E
:10EC2000220F331F220F331F220F331F880F991F0C
:10EC3000280F391F132F105DCA016091260B40E089
:10EC40000E94125D8EE20E94155E812F6091260B5C
:10EC50000E94ED5B1F91089543E650E019E3ECCF6D
:10EC6000CF92DF92EF92FF920F931F93CF93DF9398
:10EC700082EC90E20E944A5E0E946499EC018FEF60
:10EC8000CF3FD80759F1CE01937064E60E94921DE0
:10EC90007B018C016E018D2D8695869590E06091AB
:10ECA000260B40E00E94125D8EE20E94155EAAE0F3
:10ECB00016950795F794E794AA95D1F78E2D90E0D5
:10ECC0006091260B40E00E94125DDF91CF911F9171
:10ECD0000F91FF90EF90DF90CF9008958FE30E9407
:10ECE000155E83E791E20E944A5E83E791E20E940B
:10ECF0004A5EEBCFCF92DF92EF92FF920F931F937A
:10ED0000CF93DF9387EC90E20E944A5EC091800C23
:10ED1000D091810C8FEFCF3FD80759F1CE0193707E
:10ED200064E60E94921D7B018C016E018D2D8695FB
:10ED3000869590E06091260B40E00E94125D8EE285
:10ED40000E94155EBAE016950795F794E794BA9578
:10ED5000D1F78E2D90E06091260B40E00E94125D6D
:10ED6000DF91CF911F910F91FF90EF90DF90CF90A7
:10ED700008958FE30E94155E83E791E20E944A5E48
:10ED800083E791E20E944A5EEBCFCF92DF92EF924F
:10ED9000FF920F931F93CF93DF93C091800CD0917C
:10EDA000810C8FEFCF3FD80759F1CE01937064E605
:10EDB0000E94921D7B018C016E018D2D869586959A
:10EDC00090E06091260B40E00E94125D8EE20E946E
:10EDD000155E8AE016950795F794E7948A95D1F722
:10EDE0008E2D90E06091260B40E00E94125DDF9135
:10EDF000CF911F910F91FF90EF90DF90CF900895EA
:10EE00008FE30E94155E83E791E20E944A5E83E7EA
:10EE100091E20E944A5EEBCFDF92EF92FF920F9356
:10EE20001F93CF93DF93C091C90BD091CA0B8981F7
:10EE3000883609F471C0893608F469C08C3609F443
:10EE40006BC08E3609F468C08A3609F465C088E064
:10EE500091E060E00E94135C89810E94155E8EE75C
:10EE600090E20E944A5E8F810E941E5F88E790E2D6
:10EE70000E944A5E8F81EB81FC81E80FF11D808149
:10EE80000E941E5F0E946C5E84E10E940F5E5F81A3
:10EE90004A81533008F489C04F5F252F30E0842F1A
:10EEA00090E041500597281739070CF4B1C0042FA2
:10EEB0000650802F90E0EB80FC80E80EF91E842F36
:10EEC00090E00196BC01660F771F680F791F6150B3
:10EED00084E10E94B61F182FDF80D01A09F06FC09E
:10EEE00000E0123030F0F70181917F010E941E5F37
:10EEF0001250112309F441C00F5F013009F05BC0CB
:10EF00008CE30E94155E1150123058F736C08336DC
:10EF100071F1843609F09BCF2091C60B2430A8F5FF
:10EF20006E816230C0F1862F90E00C970CF041C0EA
:10EF300061504F81433098F510E0213009F477C0DB
:10EF4000213008F055C088E091E060E00E94135C39
:10EF500089810E94155E812F90E04091B50A411B86
:10EF6000825F9C4F61E120E20E94406E06C080E01B
:10EF70000E940F5ECE010E943270DF91CF911F91EF
:10EF80000F91FF90EF90DF9008951092C60B20E054
:10EF90006E81623040F660E04F81433068F2842F2A
:10EFA00090E00C97D4F11AE0C8CF00E080E090E048
:10EFB00082CF6BE0BECF0023C9F080E2A2CF00E099
:10EFC000123030F0F70181917F010E941E5F1250D4
:10EFD000112399F20F5FD01639F080E20E94155E7E
:10EFE0001150123068F7C9CF8EE3F8CF8EE389CF86
:10EFF0002230B1F0233009F0C0CF8A8580FF1DC0D8
:10F000008BE30E94985E0E94BD6F0E946C5EB5CF3C
:10F01000052F0250802F90E04ECF142F12508DCF2D
:10F020006F5F82E0412F9E010E942775A6CF81E08D
:10F03000412F9E010E942775A0CF6E5F83E0412F74
:10F040009E010E94277599CF1F93CF93DF938091E4
:10F05000F30981FF39C08091800C9091810C2FEFD2
:10F060008F3F920709F45AC066E40E94921D672FF1
:10F07000782F892F9927CB01A0E0B0E09C01AD014A
:10F0800032954295529520EF542752235427432717
:10F0900042234327CA01182F8A3008F44AC099E353
:10F0A000C3E6D0E0892F6091260B0E94ED5B8EE2D3
:10F0B0000E94155ECE016091260B40E00E94125D19
:10F0C000DF91CF911F9108958091240A85FD1BC087
:10F0D0008091150890911608969587959695879535
:10F0E00096958795880F843608F083E690E06091C6
:10F0F000260B40E00E94125D86E50E94155EDF91BE
:10F10000CF911F91089580912108909122089695A2
:10F1100087959695879596958795E4CF8091850CF0
:10F120009091860C0097E1F48FE491E20E944A5E90
:10F13000C7CFCB019F7064E60E94921D9B01AC017A
:10F1400032954295529520EF542752235427432756
:10F1500042234327CA01912F905DC82FD0E0A2CF50
:10F160009695879563E30E94921D672F782F892FCC
:10F170009927743600F5472F50E0CB0190709C0121
:10F18000220F331F220F331F220F331F880F991FA7
:10F19000280F391F132F105DCA016091260B40E024
:10F1A0000E94125D8EE20E94155E812F6091260BF7
:10F1B0000E94ED5B85CF43E650E019E3EDCF8091EF
:10F1C000C70B8130D9F0813070F48091940B90910D
:10F1D000950B099728F181E08093C70B0E94DE5DB3
:10F1E0000E949F5F0895823009F008958091C60BB8
:10F1F0008F5F8093C60B0E940C7708958091940BCB
:10F2000090E08F739070892B81F18091260B80584C
:10F210009091250B891B893A40F70E944D6B089508
:10F2200080E00E940F5E80E20E94155E80E20E94F4
:10F23000155E80E20E94155E80E20E94155E80E20B
:10F240000E94155E81EA91E20E944A5E84E10E947A
:10F250000F5E80E20E94155E86E991E20E944A5E9E
:10F260008FE891E20E944A5E08950E949F5FCDCF91
:10F27000AF92BF92CF92DF92EF92FF920F931F93C4
:10F280009B01AC01E090A90BF090AA0B0091AB0B95
:10F290001091AC0B6093A90B7093AA0B8093AB0BEE
:10F2A0009093AC0B809154018160809354018091C4
:10F2B00064018E3F20F081508093640181C02E193B
:10F2C0003F09400B510B60916201709163013093D3
:10F2D000630120936201842F80936401C9018158E6
:10F2E0009F4F8617970710F48FEF0BC0CB01815803
:10F2F0009F4F8217930710F480E003C0862F805839
:10F30000821B80939D016091F10962956F7070E09E
:10F310006F5F7F4F882777FD8095982F0E94ECC5FF
:10F320007B018C0116950795F794E794A090B301A3
:10F33000B090B401C090B501D090B60120912209DF
:10F3400030E020503F4F442737FD4095542FC801EF
:10F35000B7010E94ECC5672F782F892F99276A0D76
:10F360007B1D8C1D9D1D6093C5017093C60180930C
:10F37000C7019093C801A090B301B090B401C090B0
:10F38000B501D090B6012091660930E020503F4F82
:10F39000442737FD4095542FC801B7010E94ECC5A2
:10F3A000672F782F892F99276A0D7B1D8C1D9D1D36
:10F3B0006093C9017093CA018093CB019093CC01F3
:10F3C0001F910F91FF90EF90DF90CF90BF90AF9083
:10F3D00008958093560108959FEF9093A80B81E0C4
:10F3E0008093A40B80916B0A86FF02C090939C01CE
:10F3F0001FBC80FD02C093E801C093EC8EB5982B32
:10F400009EBD80916C0A282F30E0C9018A709070EF
:10F41000892B19F087B7806287BF80E286BF809111
:10F420007A0A85FF05C081E880938B0089E80FC0C8
:10F4300083B1806383B991E890938B008DEA8093C8
:10F440008B0083B1806383B990938B0081E820FFA8
:10F4500006C024FF03C025FF01C00F9B806480937A
:10F460008A0021FD05C080917D00806280937D002F
:10F4700080E280937C000895EF92FF920F931F9398
:10F48000CF93DF93E090980BF090990B00919A0B3B
:10F4900010919B0B4091A301442321F45091D20978
:10F4A000577002C0542F5150252F30E08091D2095F
:10F4B00090E087709070821793070CF450E050939F
:10F4C000A301A42FB0E0FD01EE0FFF1FEE0FFF1F01
:10F4D000E754F74F80819181009709F4A0C02091F3
:10F4E000A5013091A6018217930710F0B70105C05E
:10F4F000B701681B790B620F731F8091920B90917B
:10F50000930B2CB53DB53093930B2093920B28179A
:10F51000390748F48091940B9091950B0196909344
:10F52000950B8093940BCB01821B930B97FF6FC0BD
:10F53000C42FD0E0CC0FDD1FCC0FDD1FC754D74F39
:10F54000E880F980E114F10409F469C00CB51DB537
:10F550001093930B0093920B0217130748F48091BA
:10F56000940B9091950B01969093950B8093940B2F
:10F57000A851BE4FEC918091A20180958E2371F12C
:10F5800020919E01222391F08091910186FF0EC06F
:10F5900090918E01892F82958F70821720F4985850
:10F5A00090938E0107C0995890938E0180915201DB
:10F5B00080FF06C0809155018062809355010DC087
:10F5C0008091A2018E2B8093A2019BB38E2F8095F8
:10F5D00089238BBB8AB3E82BEABB81E04295407F4D
:10F5E000B8016E0D7F1D7B836A8320918A01309163
:10F5F0008B01882351F0C90143968E159F0528F48D
:10F60000B901600F711F475F05C0465F03C0429597
:10F61000407F485F81E39BE050E00E94BE61DF9144
:10F62000CF911F910F91FF90EF900895EF92FF926D
:10F630001F93CF93DF9320918201E0917601F0E058
:10F64000E851FE4F9085203809F461C0920F88235D
:10F6500011F403C0981B9817E8F78091A80B98172E
:10F6600009F061C0E090980BF090990B90918201A5
:10F6700080918301981749F4C0918601D091870148
:10F68000D0938501C093840104C0C0918401D091BE
:10F690008501809183018093820180918601909100
:10F6A0008701909385018093840110917601909158
:10F6B0007B0A812F8150981708F4892F8093760157
:10F6C000E12FF0E0E851FE4F808D882329F090E093
:10F6D0000E94FB4CE80EF91E80917701E12FF0E0CB
:10F6E000E959F14EE491E82BE0937701CE0DDF1D4F
:10F6F0001295107F81E39BE0BE01412F50E00E94F4
:10F70000BE618091B10B81608093B10B0CC0809180
:10F71000830180938201809186019091870190936B
:10F72000850180938401DF91CF911F91FF90EF902D
:10F7300008952F923F924F925F926F927F928F9295
:10F740009F92AF92BF92CF92DF92EF92FF920F9370
:10F750001F93DF93CF9300D0CDB7DEB7AC01E0901D
:10F76000940BF090950B8091920B9091930B8417D2
:10F77000950718F40894E108F108C701A0E0B0E08B
:10F780004C0177246624CA01A0E0B0E0682A792AF7
:10F790008A2A9B2A80915301816080935301809132
:10F7A000C00B882339F086FF05C085E39AE262E04A
:10F7B0000E94BD248091980B9091990BA0919A0B77
:10F7C000B0919B0B13012401281A390A4A0A5B0ADB
:10F7D0001092B10B80916B0A282F30E03A83298375
:10F7E00081FF83C2C901827A9070823A910509F043
:10F7F0009CC16092980B7092990B80929A0B909298
:10F800009B0B80916C0A84FD1DC020919B0191B1DE
:10F81000907880FD9058992311F490EC10C0922FAD
:10F820009F5F923C60F08091A80B87FF03C010920D
:10F83000A80BCEC4809155018865809355019093A3
:10F840009B01CEC18091090984FF7BC0842D882350
:10F8500021F0EE24EA94FE2C01C071010091AD0B61
:10F860001091AE0B398133FD12C00E151F05A0F4A7
:10F8700034FD02C0980103C0980136952795C70151
:10F88000801B910B2817390738F480E006C0C701A8
:10F89000B8010E9429A101C081E040919C01909192
:10F8A0009B01292F30E0882381F42F7730702E328E
:10F8B00031050CF078019E3021F410929C018EE805
:10F8C00001C08EE080939B01C2C02F703070232B4B
:10F8D00059F4925F90939B019E50413009F074C09F
:10F8E000903109F071C06AC09F3F21F09F5F9093F3
:10F8F0009B019150F092AE0BE092AD0B8091090903
:10F9000083708295807F815F981709F09CC4413095
:10F9100009F099C4930180919C0B90919D0BB301C8
:10F92000681B790B7093B2016093B1018091A00BB9
:10F930009091A10B281B390B3093B8012093B7018C
:10F9400082C480916D0A8C3008F486C0842D88238F
:10F9500021F0EE24EA94FE2C01C071010091AD0B60
:10F960001091AE0B798173FD12C00E151F05A0F426
:10F9700074FD02C0980103C0980136952795C70110
:10F98000801B910B2817390738F480E006C0C701A7
:10F99000B8010E9429A101C081E090919C01409191
:10F9A0009B018823C1F44E3208F078018EE08093E9
:10F9B0009B01403108F04BC0992331F080915501F3
:10F9C00088658093550143C080916C0A84FD3FC0D7
:10F9D0001092A80B3CC0842F90E08F709070892B00
:10F9E00021F4425F40939B0132C04F3520F44F5FBA
:10F9F00040939B014150F092AE0BE092AD0B809191
:10FA0000A80B8530F0F48091090983708295807F7E
:10FA1000815F4817B1F4930180919C0B90919D0BED
:10FA2000D301A81BB90BB093B201A093B10180918F
:10FA3000A00B9091A10B281B390B3093B801209398
:10FA4000B7014E3309F0FFC310929C01FCC3F09242
:10FA5000AE0BE092AD0BC4C080919C0190916F0AF7
:10FA6000882359F010929C01891728F08091550144
:10FA700088658093550120E003C020919B012F5F92
:10FA8000913019F4233008F0235020939B01B98161
:10FA9000B3FD32C0933040F18091A90A90E08F709D
:10FAA0009070892BE1F0909165018091B7098917D9
:10FAB000B0F010928701109286018091860190919A
:10FAC0008701909385018093840180917A019091C0
:10FAD0007B0190937D0180937C0182E001C081E0F5
:10FAE000281709F0B0C37CC0822F63E00E940BC6C8
:10FAF000913009F0A8C374C06091AD0B7091AE0B4A
:10FB0000842D882321F0EE24EA94FE2C01C071019B
:10FB1000F092AE0BE092AD0B76956795C7010E940F
:10FB200029A1813009F08FC35BC080916C0A86FFE8
:10FB300057C080919C0B90919D0BA0919E0BB09112
:10FB40009F0B64015301A81AB90ACA0ADB0A842D63
:10FB5000823020F0EE24EA94FE2C07C0D201C101CD
:10FB6000B695A795979587957C016091A80A6295AF
:10FB70006F70605FC7010E94921D9B01AC0194E011
:10FB800056954795379527959A95D1F7CA01AA2793
:10FB9000BB27882319F06FEF7FEF01C0B901CB01BC
:10FBA000A0E0B0E08A159B05AC05BD05C8F06091EA
:10FBB000A80A6F70C7010E94921D04E09695879570
:10FBC000779567950A95D1F780E090E0A616B7067D
:10FBD000C806D90628F080915501886580935501A3
:10FBE0004091A80B47FD3BC090916D0A491721F445
:10FBF00081E18093560140E08091550186FD0AC065
:10FC0000142F1F5F80916C0A84FDC4C1191709F07D
:10FC1000C1C1BFC1292F2150809155018F7B809395
:10FC20005501421709F4B5C181E4809356012B3385
:10FC300018F02695421789F08091090985FFA9C11E
:10FC4000242F30E0892F90E002972817390709F018
:10FC5000A0C18091550180FF9CC1142FEBC0809101
:10FC6000550186FF2EC0809155018F7B80935501F1
:10FC700080916B0A90E0827A90708232910531F423
:10FC80004F3B79F14B3B69F416E02CC0823A910569
:10FC900061F480916D0A863041F4403C11F14C3B97
:10FCA000F1F080EC8093A80B93C28091090985FF45
:10FCB00018C08091550180FF14C010916D0A115039
:10FCC00011C080916C0A84FF0CC080916B0A827A0B
:10FCD000823209F07DC241504093A80B79C215E0F1
:10FCE00001C010E01093A80B55C1842D882321F08A
:10FCF000EE24EA94FE2C01C071016091AD0B70916D
:10FD0000AE0BE981E3FD12C06E157F0598F4E4FDAA
:10FD100002C09B0103C09B0136952795C701861B36
:10FD2000970B2817390730F480E005C0C7010E94FF
:10FD300029A101C081E01091A80B17FD84C090910A
:10FD40006D0A882321F0813009F076C073C080915C
:10FD5000B10B80648093B10B903239F51232D1F03F
:10FD6000133240F41F30A1F01E3191F01C3009F025
:10FD70004DC00EC0133361F0143320F4103309F07A
:10FD800045C006C0123421F0163409F03FC002C04D
:10FD90001E5F4DC08091550186FF53C28091550171
:10FDA0008F7B8093550114E242C080916C0A84FFDE
:10FDB0001CC08091550186FF0DC0809155018F7B3D
:10FDC00080935501212F291B80916B0A84FD17C058
:10FDD000215015C080916B0A84FD02C083E001C0F0
:10FDE00082E0212F2F5F180F0BC0212F2F5F94303F
:10FDF00030F4143010F414E003C0212F235010E02D
:10FE00002917A9F0921718F481E102C020E081E2DD
:10FE10008093560130E0892F90E001972817390729
:10FE200031F08091550184608093550108C0F694AB
:10FE3000E794B0C01F5FAEC081E6809356018FEF9C
:10FE40008093A80B99C0173F08F08DC090916D0A60
:10FE5000882309F07EC0F694E7948FEF80936401C5
:10FE60008091B10B80648093B10B9032E9F5809161
:10FE700055018B7F809355011C3AE9F01D3A18F427
:10FE80001B3A71F523C0163B69F0173B49F5809189
:10FE90007B0A815080937601809176018093750171
:10FEA00011E178C080917B0A809376018091760180
:10FEB000809375016EC080917B0A8150809376019A
:10FEC00080917601809375011EE064C080917B0A69
:10FED00080937601809176018093750110E25AC07B
:10FEE00088EB8093A80B56C080916C0A84FF2BC0CE
:10FEF0008091550186FF0FC0809155018B7B8093C7
:10FF00005501133808F445C08091910A8F3F09F4D8
:10FF100040C016EF3FC0113C38F080915501877A00
:10FF20008093550180EC8CCF809155018B7F80931D
:10FF3000550180916B0A84FD02C022E001C021E0DE
:10FF4000122F190F27C0809155018B7F8093550187
:10FF500020C0903221F0812F8258843708F411504C
:10FF60001093A80B09C0812F81508093A80B8D3F5F
:10FF700018F08FEF80936401F092AE0BE092AD0B1E
:10FF80006092980B7092990B80929A0B90929B0BB7
:10FF90001FC110E08091F20987FF09C080916B0AB0
:10FFA00080FF03C0849903C04EC184994CC1F09274
:10FFB000AE0BE092AD0B6092980B7092990B809211
:10FFC0009A0B90929B0B1093A80B80916401803147
:10FFD00008F0ACC000916D0A80916B0A81FD15C0DC
:10FFE000003211F404E211C084FF03C0902F9F5F20
:10FFF00002C0902F9E5F80916C0A84FD04C0043083
:020000021000EC
:1000000010F0092F02C0092F000F802F0E94167BCD
:10001000E0917501F0E0E851FE4F908580918001FC
:10002000803809F477C0980F002311F403C0901BA7
:100030009017E8F78091A80B981709F05EC0E09040
:100040007C01F0907D0100917501E02FF0E0E85116
:10005000FE4F808D882329F090E00E94FB4CE80E33
:10006000F91E80917701E02FF0E0E959F14EE4911B
:10007000E823A1F12091980B3091990B40919A0BB4
:1000800050919B0B832F942F8F0D911D90936C019A
:1000900080936B0180917B0AE02FE1508E1708F46A
:1000A000E82FE09375018091540187FF06C080918D
:1000B0009D01F0E0E55EFA4F80830295007FE20E3D
:1000C000F31E0F5F81E39BE0B701402F50E00E94D9
:1000D000BE618091B10B82608093B10B80918101F0
:1000E0008093800180917E0190917F0190937D01AA
:1000F00080937C011092B20B19C090918001809185
:100100008101981799F08091B20B81508093B20BC6
:10011000882361F4809181018093800180917E0128
:1001200090917F0190937D0180937C0106B605FE3E
:100130000BC080916B0A86FF07C080E286BF80916A
:100140009C01815080939C01112349F580916C0A98
:1001500084FF25C01092A30180916B0A827A823AB3
:10016000B1F0930180919C0B90919D0BA301481BD2
:10017000590B5093B2014093B1018091A00B909123
:10018000A10B281B390B3093B8012093B701609263
:10019000B3017092B4018092B5019092B601809142
:1001A0006B0A827A823A31F480916D0A8C3010F4B5
:1001B00081E006C080916F0A882321F001C0181BDE
:1001C0001817E8F7112321F4C401B3010E9438790C
:1001D000598152FF2FC0842D8529882359F4B101FC
:1001E0007695679583E16938780720F48B010C5385
:1001F000104002C008E813E18091B10B86FF02C0F5
:10020000169507956091920B7091930B600F711F7B
:1002100081E39BE042E050E00E94BE61812F99277C
:10022000892B29F48091B10B84608093B10B87B73F
:100230008F7D87BF8091B10B877129F00E94636425
:1002400002C010E0F4CD0F900F90CF91DF911F917D
:100250000F91FF90EF90DF90CF90BF90AF909F9065
:100260008F907F906F905F904F903F902F90089568
:100270001F920F920FB60F920BB60F9211248F920E
:100280009F92AF92BF92CF92DF92EF92FF920F9325
:100290001F932F933F934F935F936F937F938F930E
:1002A0009F93AF93BF93CF93DF93EF93FF9380918F
:1002B0006B0A86FF54C080919C01823018F081E067
:1002C00080939C018091550186FF03C081E3809358
:1002D0005601809155018865809355012091940BBA
:1002E0003091950B8091920B9091930BECB5FDB5ED
:1002F000F093930BE093920BE817F90740F42F5F0C
:100300003F4F3093950B2093940B21503040C901FF
:10031000A0E0B0E0DC01992788279F0140E050E091
:10032000822B932BA42BB52B80939C0B90939D0B2E
:10033000A0939E0BB0939F0B8091C00B86FFABC127
:1003400083EF99E266E0AF0122E00E945E24809193
:10035000F20981FFA0C182E00E941DA59CC180918D
:10036000920B9091930BCCB5DDB5D093930BC093CA
:10037000920BC817D90748F48091940B9091950B74
:1003800001969093950B8093940B80916C0A83FD5A
:1003900004C0CE010E94997B7EC10091940B109104
:1003A000950B8091C00B882349F086FF07C083EF2F
:1003B00099E266E0AE0122E00E945E248091F2099B
:1003C00081FF03C082E00E941DA5C801A0E0B0E04B
:1003D0008C01FF24EE24CE01A0E0B0E0E82AF92A47
:1003E0000A2B1B2B80916C0A682F70E086FF15C0CA
:1003F0008091F20981FF03C082E00E941DA58091D7
:100400009C018F5F80939C01E0929C0BF0929D0B6E
:1004100000939E0B10939F0B3EC1E4E0CE2ED12C97
:10042000C622D72282FF1FC080919C0B90919D0B0A
:10043000A0919E0BB0919F0BA8019701281B390B2F
:100440004A0B5B0B842F852B882349F4C9019695B1
:10045000879523E18938920710F4CC9702C088E889
:1004600093E1C80FD91F90918A008091F209582F0B
:1004700086FF07C096FF03C00F9B0DC102C00F99F6
:100480000AC180916401803108F049C064FF47C00F
:100490008091C5019091C601A091C701B091C8019A
:1004A00047015801881A990AAA0ABB0A8B2D87FFAF
:1004B00011C08091C9019091CA01A091CB01B09166
:1004C000CC0147015801881A990AAA0ABB0A8B2D48
:1004D000813828F19091A80B20916D0A80916B0AC8
:1004E00084FD02C082E001C081E0820F19F406C0E1
:1004F000920F02C0282F21959817D0F78091910A6A
:10050000981768F481E5809356019091090996FF48
:10051000BCC08FEF809364018093A80BB6C040E00D
:10052000E0929C0BF0929D0B00939E0B10939F0BFF
:1005300064FF94C080916B0AE82FF0E0CF01827ACB
:1005400090708232910539F0823A9105A9F4809138
:100550006D0A863089F49091A80B80916D0A8630DF
:1005600019F025E030E002C024E030E0892F90E06F
:100570008217930709F478C065FF09C08091530181
:1005800081FF05C080918A0090E4892709C060FF3F
:1005900004C080918A00806403C080918A008F7BB0
:1005A00080938A00442321F08091090987FD5CC073
:1005B0003091910A3F3FD9F48091550186FF08C0E0
:1005C00081E38093560151FF03C089E00E941DA57D
:1005D00080915501886580935501849B04C080916A
:1005E0005501816019C0809155018E7F15C0909191
:1005F000A80B97FF14C08091550186FD35C08091EE
:100600006D0A831710F481E802C08E57831B809314
:10061000A80B8091550188658093550125C02091D4
:100620006D0AE4FD02C082E001C081E0820F19F48E
:1006300006C0920F02C0282F21959817D0F7931764
:1006400098F48091550186FFE4CF81E380935601B1
:1006500051FFDFCF89E00E941DA5DBCF80918A008A
:1006600090E4892780938A00CD28A9F080917D00AD
:100670008F7D80937D0081E39BE0BE0143E050E0ED
:100680000E94BE610E94636406C097FF02C041E001
:100690004FCF41E045CFFF91EF91DF91CF91BF91D7
:1006A000AF919F918F917F916F915F914F913F910A
:1006B0002F911F910F91FF90EF90DF90CF90BF90FF
:1006C000AF909F908F900F900BBE0F900FBE0F902A
:1006D0001F9018951F920F920FB60F920BB60F92A4
:1006E00011242F933F934F935F936F937F938F9337
:1006F0009F93AF93BF93EF93FF9390916B0A96FFF5
:1007000010C080919C01882321F0815080939C012E
:1007100022C097FD02C082E002C08091A90A8093A6
:100720009C012091920B3091930B8CB59DB59093C9
:10073000930B8093920B8217930748F48091940B4C
:100740009091950B01969093950B8093940B86B5A1
:1007500097B50E94997BFF91EF91BF91AF919F91C7
:100760008F917F916F915F914F913F912F910F905A
:100770000BBE0F900FBE0F901F901895809112091D
:1007800090E09C012074307086FF06C08AB78061BB
:100790008ABF8AB78F7D02C08AB780638ABF80E430
:1007A00088BF89B7806489BF10925307232B49F013
:1007B00080916A00816080936A0080916A008D7FD9
:1007C00008C080916A00826080936A0080916A000C
:1007D0008E7F80936A0081E088BF89B7816089BF7E
:1007E0001092180208951F920F920FB60F920BB637
:1007F0000F921124DF92EF92FF920F931F932F938A
:100800003F934F935F936F937F938F939F93AF9398
:10081000BF93CF93DF93EF93FF9380911E0281509C
:1008200080931E028F5F09F094C08091130A829515
:100830008F7080931E02D0901D02DD2019F084E09D
:10084000D81621F489B78E7F89BF83C08091920B1F
:100850009091930BCCB5DDB5D093930BC093920BD5
:10086000C817D90748F48091940B9091950B019685
:100870009093950B8093940B0091940B1091950B92
:100880008091C00B86FF07C083EF99E266E0AE015E
:1008900027E00E945E248091F20981FF03C087E077
:1008A0000E941DA581E0D81611F482E050C0C80155
:1008B000A0E0B0E08C01FF24EE24CE01A0E0B0E087
:1008C000E82AF92A0A2B1B2B82E0D81651F4E09271
:1008D0001902F0921A0200931B0210931C0283E08B
:1008E00036C08091190290911A02A0911B02B0911A
:1008F0001C02A8019701281B390B4A0B5B0B62E015
:1009000056954795379527956A95D1F7E092190244
:10091000F0921A0200931B0210931C02C90143E0DB
:10092000880F991F4A95E1F7A0E0B0E08093250277
:1009300090932602A0932702B093280281E292E0CE
:10094000B9010E94681D80912902843011F48093BE
:100950001D02FF91EF91DF91CF91BF91AF919F91D8
:100960008F917F916F915F914F913F912F911F9147
:100970000F91FF90EF90DF900F900BBE0F900FBE86
:100980000F901F9018951F920F920FB60F920BB6F3
:100990000F921124DF92EF92FF920F931F932F93E8
:1009A0003F934F935F936F937F938F939F93AF93F7
:1009B000BF93CF93DF93EF93FF93809159078150BB
:1009C000809359078F5F09F090C08091130A8F7050
:1009D00080935907D09058078D2D8150833020F097
:1009E00089B78F7B89BF81C08091920B9091930BC7
:1009F000CCB5DDB5D093930BC093920BC817D90734
:100A000048F48091940B9091950B01969093950BDF
:100A10008093940B0091940B1091950B8091C00BD7
:100A200086FF07C083EF99E266E0AE0126E00E94F0
:100A30005E248091F20981FF03C086E00E941DA51B
:100A400081E0D81611F482E04EC0C801A0E0B0E009
:100A50008C01FF24EE24CE01A0E0B0E0E82AF92AC0
:100A60000A2B1B2B82E0D81651F4E0925407F09227
:100A70005507009356071093570783E034C08091C1
:100A8000540790915507A0915607B0915707A801B8
:100A90009701281B390B4A0B5B0BE2E056954795F3
:100AA00037952795EA95D1F7E0925407F0925507CC
:100AB0000093560710935707842F882319F06FEF80
:100AC0007FEF01C0B90180915A0790915B076817C9
:100AD000790708F4BC018CE597E00E94681D8091BD
:100AE0006407843011F480935807FF91EF91DF91F0
:100AF000CF91BF91AF919F918F917F916F915F91B6
:100B00004F913F912F911F910F91FF90EF90DF90A8
:100B10000F900BBE0F900FBE0F901F9018951F9354
:100B2000182F80916501E82FF0E0EE0FFF1FE758C6
:100B3000FA4F8591949162E30E94921DDC01CB01F2
:100B4000892F9A2FAB2FBB27612F0E94921D9B01EB
:100B5000AC01842F882319F06FEF7FEF01C0B9013A
:100B6000660F672F661F770B7195EFEFF8E030E0A7
:100B70002181808190E0820F911D6817790710F420
:100B8000832F05C03F5F3196353091F785E0809324
:100B9000A0011F910895EF92FF920F931F93CF939F
:100BA000DF93EC01ED84FE840F85188972E01695C1
:100BB0000795F794E7947A95D1F7E62FF0E0EE0FDA
:100BC000FF1FE758FA4F859194916FE50E94921D9F
:100BD000970140E050E00E942BC68091120986FFE9
:100BE00002C0369527952F3F310519F010F02FEFF1
:100BF00030E028831D82DF91CF911F910F91FF90EC
:100C0000EF900895CF93DF93EC01F8948091920BCD
:100C10009091930B2CB53DB53093930B2093920B91
:100C20002817390748F48091940B9091950B019601
:100C30009093950B8093940B78948091940B909162
:100C4000950BA0E0B0E0DC019927882740E050E058
:100C5000822B932BA42BB52B29813A814B815C816C
:100C6000821B930BA40BB50B9C01AD01842F8695C1
:100C7000869541F1188237E0C335D30729F41092E5
:100C8000A0018091FE0802C080914309E82FF0E0A6
:100C9000EE0FFF1FE758FA4F859194916FE50E9480
:100CA000921D21E031E040E050E00E94ECC5BC0123
:100CB000882799278091120986FF02C0660F771F47
:100CC00078876F838D818823A1F581E08D83CE01A4
:100CD00009960E945B1DC355D74079F48091120993
:100CE00086FF03C08AB78F7D02C08AB780628ABF41
:100CF00080E488BF89B780641BC08091120986FF99
:100D000009C080916A00816080936A0080916A00C6
:100D10008D7F08C080916A00826080936A00809114
:100D20006A008E7F80936A0081E088BF89B7816006
:100D300089BFDF91CF91089525B32F70962F9F78AB
:100D4000282B992331F06077262B25BB9698969A0D
:100D50000895262B25BB809165008B7F80936500CD
:100D6000809165008460809365000895982FFB0151
:100D70008A3320F4803378F090530AC0815486304F
:100D800010F4975305C0892F8156863020F497556B
:100D9000908381E0089580E00895FC01228185819F
:100DA000882329F09091B30A5091B50A02C0968128
:100DB0005781822F82958F70891740F12F702517E8
:100DC00028F1892F90E030E02F5F3F4F829FF001A4
:100DD000839FF00D929FF00D1124E50FF11DE60F9A
:100DE000F71F8081552747FD5095480F511D852FCE
:100DF0009927009741F08F3F910519F04FEF50E090
:100E000002C040E050E0408381E0089580E0089512
:100E1000FC0160831582178216828AE681838CE248
:100E200093E0948383838FED828308952BEF3FEFCC
:100E300041E050E06FEF7FEF4BBFF90187916827EA
:100E4000862F82958627082E869586958025082EE2
:100E5000869580258770062E672F8695079487953F
:100E6000702D68270694879570256827215030409B
:100E700040405040253F8FEF380781E0480780E031
:100E8000580709F0D9CFCB0108951F93CF93DF9373
:100E9000EC013A818D81882329F09091B30A209149
:100EA000B50A02C09E812F81832F82958F7089178A
:100EB000C8F1132F1F701217A8F11F5F199F902DF3
:100EC00011241150920FEB81FC81E90FF11D608319
:100ED0008981833699F4993829F0923B79F40E94FC
:100EE000B7610CC060913C0A70E096E0660F771F16
:100EF0009A95E1F78FE89CE00E941C9F8F818117F3
:100F000018F48F5F8F830CC08981833649F49E81EA
:100F10008A8182958F70981718F49F5F9E831F8235
:100F200081E001C080E0DF91CF911F9108950F9380
:100F30001F93482F809375018093760180917601ED
:100F400090917B0A8150981708F4892F809376013D
:100F5000F89480917A0A382F85FF38C020918F014C
:100F6000222399F090918E01892F82958F7082179C
:100F700048F4985890938E01809155018062809337
:100F800055014EC0995890938E01809155018F7DE7
:100F900080935501E42FF0E0E851FE4F608930FD69
:100FA00002C000E801C000E04F3FD1F1162F1877D2
:100FB000802F612F0E949C8680917A0A81FF30C029
:100FC0001051802F612F0E949C862AC0E42FF0E0F0
:100FD000E851FE4F608980FD02C000E001C000E8DA
:100FE0004F3F79F0162F1877802F612F0E949C8633
:100FF00080917A0A81FF05C01051802F612F0E94D5
:101000009C8684E690E090938300809382008BE935
:1010100090E090938500809384008DEA80938B000C
:1010200078940000F8948091920B9091930B6CB59A
:101030007DB57093930B6093920B6817790748F412
:101040008091940B9091950B01969093950B8093C2
:10105000940B80917A0190917B01680F791F81E355
:101060009BE041E050E00E94BE610E94636478947E
:101070001F910F910895FF920F931F93DF93CF93CA
:101080000F92CDB7DEB78C01F62EDC018C918D303E
:1010900011F40C94FC928E3068F5863009F43FC54B
:1010A0008730A0F4823009F4F0C0833040F4882304
:1010B00009F4CCC0813011F00C946C94DAC0843007
:1010C00009F4DEC1853008F007C219C1893009F47E
:1010D00069C58A3040F4873009F431C5883011F091
:1010E0000C946C9454C58B3009F47DC58C3008F099
:1010F000EBC569C5843111F40C944C928531B0F480
:10110000803109F4B2C6813148F48E3011F40C9468
:10111000B4938F3011F00C946C945BC6823109F457
:1011200089C7833110F00C94799156C7883111F436
:101130000C947792893150F4853111F40C945992C2
:10114000863111F00C946C940C946492813209F401
:10115000C2C08F3F31F0893111F00C946C940C9423
:101160007B921092B50DB3E56B1739F48EE092E2E5
:101170006AE10E9431240C946F94862FBE016F5F48
:101180007F4F0E94B686882391F0809181089091CC
:10119000820824E0880F991F2A95E1F72981820FA0
:1011A000911D90938208809381080C946F946FEF47
:1011B0007FEF2BEF3FEF41E050E04BBFF90187910C
:1011C0006827862F82958627082E86958695802506
:1011D000082E869580258770062E672F86950794A2
:1011E0008795702D6827069487957025682721506C
:1011F000304040405040253FEFEF3E07E1E04E07D2
:10120000E0E05E0709F0D9CF8091810890918208D3
:101210006817790759F4D8011C9281EF92E266E0D1
:1012200043E252E20E94BD240C946F9481EF92E25B
:1012300068E04AE152E20E94BD2483E093E26CE060
:1012400040EF5FEF0E94BD240C946F94BDE46B17D8
:1012500059F480917D08882339F481E0F801808376
:101260001092B50D0C946F948F2D0E94ED2B0C9461
:101270006F94F1E66F1729F482E0D8018C930C94F7
:101280006F94F80110820C946F94F7E66F17C1F019
:101290008EE6681721F0A3E66A17C9F40CC083E054
:1012A000F801808381EF92E268E041E152E20E941E
:1012B000BD240C946F948EE1D8018C930C946F94A0
:1012C00010929A0881E2F80180830C946F94D801FF
:1012D0001C920C946F94862F0E9457BF813011F09E
:1012E0000C946F94809105098E3D11F060E001C06F
:1012F0006FEF8BEC9BE00E9408870C946F94B6E72D
:101300006B1709F498C0B61750F1E9E66E1709F4A7
:1013100079C0E61770F0F3E66F1709F469C084E648
:10132000681709F46AC0A2E66A1711F00C946F946A
:101330005AC0B1E76B1709F483C0B61730F0ECE67A
:101340006E1711F00C946F9462C0F3E76F1709F4F5
:1013500063C084E7681711F00C946F9462C0A0E931
:101360006A17E9F0A61768F0B8E76B1709F45EC0D2
:101370006B1708F473C0EAE86E1711F00C946F94C1
:1013800018C0F2E96F1781F06F17C0F083EF68178C
:10139000D1F0ABEF6A1711F00C946F941DC084E08C
:1013A0000E943E6B0C946F9484E00E94296B0C9415
:1013B0006F9481E00E943E6B0C946F9481E00E94D8
:1013C000296B0C946F9482E0B8010E941D6B85E03C
:1013D000F80180830C946F948BE79BE568E50E948D
:1013E00031240C946F9488E0D8018C930C946F9402
:1013F00083E1F80180830C946F9480E1D8018C9391
:101400000C946F9487E1F80180830C946F948FE0C3
:10141000D8018C930C946F9489E1F80180830C942B
:101420006F9484E0D8018C930C946F948CE0F80155
:1014300080830C946F9488E1D8018C930C946F9402
:10144000F8018181833611F00C946F94638174816B
:10145000C80141E00E94CD860C946F94D80111968A
:101460008C911197833611F00C946F9413966D91B3
:101470007C911497C8014FEF0E94CD860C946F9415
:1014800083E0F8018083F4E76F17E9F083EF6817D2
:10149000D1F0A6E66A1711F00C946F94F8018181DF
:1014A0008A3631F08E3621F08C3611F00C946F9420
:1014B000D80113968D919C9114979093B60B8093BD
:1014C000B50B0C946F9482E0B8010E941D6B85E00F
:1014D000F80180830C946F948AE0D8018C93BEE667
:1014E0006B1709F468C2B617A8F1E6E66E1709F49F
:1014F000ACC1E617C0F0F3E66F1709F45EC1F6174A
:1015000048F083E4681709F47CC1A2E66A1709F081
:1015100002C39FC2B4E66B1709F42FC2E5E66E174B
:1015200009F0F9C2DFC2FAE66F1709F4D9C1F6175C
:1015300048F087E6681709F499C1A8E66A1709F028
:10154000EAC2B3C1BCE66B1709F4E4C1B61708F4EC
:10155000A1C0F9C1E8E76E1709F41BC1E617C0F096
:10156000F2E76F1709F45CC2F61748F080E76817D6
:1015700009F440C2A1E76A1709F0CDC294C0B4E7EC
:101580006B1709F47FC2E7E76E1709F0C4C2ECC01D
:10159000FAE86F17B9F0F61748F089E7681709F409
:1015A00088C2AAE76A1709F0B6C2ADC0B1E96B17E5
:1015B000C1F0E2E96E1709F445C0F0E96F1709F0D0
:1015C000AAC223C0D80116968C911697882319F0C9
:1015D000815016968C9385E0F801808315820C94D7
:1015E0006F94D80116969C91169712968C9112972B
:1015F00082958F70981718F49F5F16969C9385E0DC
:10160000F801808315820C946F94D80117968C9101
:101610001797882321F0815017968C930BC0F801FF
:101620008181833639F48681882321F08150868335
:101630008FE08783D80115961C92159785E08C93CF
:101640000C946F94F80147815281242F30E0852F4C
:1016500090E08F709070281739071CF44F5F478314
:1016600013C0D80111968C911197833669F41696A0
:101670008C91169752955F70851730F48F5F169690
:101680008C93169717961C92F801158285E080833B
:101690000C946F9481E0B8010E941D6B83E0D80127
:1016A0008C930C946F9485E0F801808381818A3655
:1016B00011F08E36A9F4D8011696EC911697F0E049
:1016C00004E0EE0FFF1F0A95E1F717968C91E80FE3
:1016D000F11DE25DFD4F80818F5F80830C946F94DC
:1016E000833641F08C3631F0823621F0843711F0A8
:1016F0000C946F94F80163817481C80141E00E94E9
:10170000CD860C946F9485E0D8018C9311968C91C2
:101710008A3611F08E36A9F4D8011696EC911697F8
:10172000F0E014E0EE0FFF1F1A95E1F717968C9189
:10173000E80FF11DE25DFD4F8081815080830C94A4
:101740006F94833641F08C3631F0823621F0843745
:1017500011F00C946F94F80163817481C8014FEF0C
:101760000E94CD860C946F9485E0D8018C931196DD
:101770008C918A3631F08E3621F08C3611F00C9433
:101780006F94C80165E677E041E00E94CD860C9435
:101790006F9485E0F801808381818A3631F08E363E
:1017A00021F08C3611F00C946F94C80165E677E057
:1017B0004FEF0E94CD860C946F94D80111966C93D4
:1017C000119783EB99E014969C938E9313978FEF68
:1017D00012968C93129715961C92159716968C91CB
:1017E0001697803118F08FE016968C93F801878158
:1017F00090E0409714F40C946F948FE087830C94DE
:101800006F94D80111966C93119789EE98E0149615
:101810009C938E9313978FEB12968C931297159639
:101820001C92159716968C9116978C3018F08BE0B9
:1018300016968C93F801878190E0409714F40C94ED
:101840006F948FE087830C946F94D80111968C91DC
:101850008A3621F08E3611F08C3619F480E8F801C2
:10186000858385E0D8018C930C946F9486E0F80111
:10187000808315824281942F92959F70868198175C
:1018800008F49683D80117962C91179730E0842F8F
:1018900090E08F7090708217930714F00C946F94FF
:1018A0004F7017964C930C946F94F801618388EEF7
:1018B00091E09483838387E582838681863010F06C
:1018C00085E08683D80117968C91179790E008974A
:1018D00014F40C946F9487E017968C930C946F9487
:1018E000F80161838CE293E0948383838FED82839C
:1018F00086818E3010F08DE08683D80117968C910A
:10190000179790E0409714F40C946F948FE017961B
:101910008C93E5C7F80161838CE293E09483838321
:1019200087E782838681883010F087E08683D8013C
:1019300017968C91179790E008970CF4D0C787E022
:1019400017968C93CCC78BE6F80181838EE193E0E8
:10195000948383838DE0828315828681181608F430
:101960001682D80117968C91179790E00E970CF479
:10197000B6C78DE017968C93B2C785E0F8018083D7
:101980008AE681838CE293E0948383838FED828364
:1019900086818E3010F08DE08683D80117968C9169
:1019A000179790E040971CF08FE017968C9384E691
:1019B000F801818394C7D80111966C93119785E63D
:1019C00097E014969C938E9313978BEB12968C93BF
:1019D000129716968C9116978C3018F08BE016960D
:1019E0008C93F801878190E00C970CF478C78BE01A
:1019F000878375C7D80111968C918A3631F08E365F
:101A000021F08C3611F0843639F48091B30AF80154
:101A100086838091B50A878385E0D8018C935FC760
:101A2000F80161838EE093E0948383838FE0828367
:101A300015828681181608F41682D80117968C91A3
:101A4000179790E040970CF44AC78FE017968C9355
:101A500046C7F801618384EC95E0948383838BED22
:101A6000828386818E3010F08DE08683D8011796B0
:101A70008C91179790E00C970CF431C78BE0179678
:101A80008C932DC7F80161838CEB95E0948383835D
:101A900087E08283868181111682D80117968C9106
:101AA000179790E008970CF41AC787E017968C9365
:101AB00016C7F80161838BEA96E0948383838BEBEE
:101AC000828386818C3010F08BE08683D801179654
:101AD0008C91179790E00C970CF401C78BE0179648
:101AE0008C93FDC6F80161838CE194E09483838339
:101AF00087E9828386818A3010F089E08683D80165
:101B000017968C91179790E008970CF4E8C687E039
:101B100017968C93E4C685E0F8018083E0C6B8018F
:101B2000685F7F4F8F2D0E94B686882321F087E063
:101B3000D8018C93D4C685E0F8018083D0C685E0B7
:101B4000D8018C93B801695F7F4F8F2D0E94B686B4
:101B5000882309F4C4C6F8018085868315824281F2
:101B6000942F92959F70981708F49683D801179632
:101B70002C91179730E0842F90E08F70907082172F
:101B800093070CF0ACC64F7017964C93A8C6B9E7F4
:101B90006B1721F489E0F8018083A1C683E0D801A6
:101BA0008C939DC6B5E66B1751F4F801108281EF56
:101BB00092E265E04BE052E20E94BD2490C683E0D1
:101BC000D8018C938CC6B801685F7F4F8F2D0E941F
:101BD000B686882321F08BE0F801808380C685E0FB
:101BE000D8018C937CC685E0F8018083862FBE01E6
:101BF0006F5F7F4F0E94B686882309F465C0D801C5
:101C000018966C9118976295607F8981682B69831B
:101C100011968C918A3661F18B3680F4833601F10E
:101C2000843630F4833401F1823609F058C63CC062
:101C30008536D1F1883609F052C63AC08E36E1F1C8
:101C40008F3630F48B3661F18C3609F048C62CC0E3
:101C5000843751F1893741F1823709F040C630C0ED
:101C6000C8010E9445873BC6C8010E94458737C608
:101C7000F801F780C8010E944587882309F42FC620
